:020000024000BC
:10000000F0650220E1250400592604009D2004002B
:100010009D2004009D2004009D2004009D200400DC
:100020009D2004009D2004009D2004006120040008
:100030009D2004009D2004001D2004009D2004003C
:10004000C5200400C5200400C5200400C52004000C
:10005000C5200400C5200400C5200400C5200400FC
:10006000C5200400C5200400C5200400C5200400EC
:10007000C5200400C5200400C5200400C5200400DC
:10008000C5200400C5200400C5200400C5200400CC
:10009000C5200400C5200400C5200400C5200400BC
:1000A000C5200400C5200400C5200400C5200400AC
:1000B000AD310400CF310400C5200400C520040088
:1000C000C5200400C5200400C5200400C52004008C
:1000D000C5200400C5200400C5200400C52004007C
:1000E000C5200400C5200400F1310400C52004002F
:1000F000C5200400C5200400C5200400C52004005C
:10010000C5200400C5200400C5200400C52004004B
:10011000C5200400C5200400C5200400C52004003B
:10012000C5200400C5200400C5200400C52004002B
:10013000C5200400C5200400C5200400C52004001B
:10014000C52004007BB972B90029BEBF00204FF062
:10015000004106E008BF00281CBF6FF000414FF0CF
:10016000FF3000F0C7B9ADF1080C6DE904CE0029ED
:1001700009DB002B1ADB00F04DF8DDF804E0DDE9C7
:10018000022304B07047404261EB4101002B1BDBAE
:1001900000F040F8DDF804E0DDE9022304B040425D
:1001A00061EB4101524263EB43037047524263EB00
:1001B000430300F02FF8DDF804E0DDE9022304B08A
:1001C000404261EB41017047524263EB430300F050
:1001D00021F8DDF804E0DDE9022304B0524263EBCC
:1001E0004303704753B94AB9002908BF00281CBF10
:1001F0004FF0FF314FF0FF3000F07CB9ADF1080C4B
:100200006DE904CE00F006F8DDF804E0DDE9022334
:1002100004B070472DE9F0478C46089D04468A4695
:10022000002B4AD18A42174662D9B2FA82F64EB101
:10023000C6F1200E01FA06F3B740B44020FA0EFED4
:100240004EEA030A4FEA1748230C1FFA87F9BAFB54
:10025000F8FE08FB1EAA0EFB09F243EA0A439A4283
:100260000BD9FB180EF1FF312CBF012000209A4260
:1002700002D9002800F02A818E469A1AA3B2B2FB56
:10028000F8F008FB102200FB09F943EA0244A145FB
:1002900007D93C1900F1FF3302D2A14500F21081C9
:1002A0001846A4EB090440EA0E4000211DB1F440B9
:1002B0000023C5E90043BDE8F0878B4208D9002D33
:1002C00000F0F2800021C5E9000C0846BDE8F08787
:1002D000B3FA83F100294ED16345C0F0E880824231
:1002E00040F2E5800846002DE5D0C5E9004AE2E786
:1002F00002B9FFDEB2FA82F6002E40F099808B1A26
:100300004FEA124E1FFA82F801214FEA144CB3FB58
:10031000FEF20EFB123008FB02F94CEA004CE145FC
:1003200008D917EB0C0C02F1FF3302D2E14500F2C1
:10033000CA801A46ACEB090CA3B2BCFBFEF00EFB64
:1003400010CC08FB00F843EA0C44A0450ED93C1938
:1003500000F1FF332CBF4FF0010C4FF0000CA04513
:1003600003D9BCF1000F00F0A8801846A4EB0804E4
:1003700040EA02409AE7C1F120048B4002FA01FEF4
:100380000CFA01F6E24020FA04F72CFA04FC00FA19
:1003900001F813433E431F0C320C1FFA83F9BCFBD8
:1003A000F7F007FB10CC00FB09FA42EA0C4CE245DF
:1003B00008D913EB0C0C00F1FF3202D2E24500F237
:1003C00089801046ACEB0A0CB6B2BCFBF7FA07FB0F
:1003D0001ACC0AFB09F946EA0C42914506D99A184B
:1003E0000AF1FF3601D291457AD8B2464AEA004076
:1003F000A2EB0902A0FB0E67BA42B446B94602D38B
:1004000007D1B04505D2B6EB0E0C67EB03030138FC
:100410009946002D6BD0B8EB0C0362EB090202FA8F
:1004200004F4CB40CA4000211C43C5E9004242E726
:10043000B740C6F1200201FA06F3B44021FA02FCEB
:100440004FEA174E20FA02F21FFA87F8BCFBFEF1C2
:100450001A430EFB11CC01FB08F0130C43EA0C4CC1
:10046000604507D917EB0C0C01F1FF3301D2604551
:1004700033D81946ACEB000C92B2BCFBFEF00EFB7D
:1004800010CC00FB08F342EA0C4C634507D917EB8C
:100490000C0C00F1FF3201D2634525D81046ACEBBD
:1004A000030340EA014130E72946284603E7841A5E
:1004B0006CEB030301209A4615E702383C4455E7EC
:1004C00002383C44EDE6023ABC4433E7AEF1020E9A
:1004D0003B44D2E602389C4474E70239BC44C9E785
:1004E000AAF1020A1A4481E70238BC44D7E7294638
:1004F000E1E600BF704700BF30B44FF0000310F8D2
:10050000014B11F8015B013A84EA050443EA040354
:10051000F5D1A3F101034FEAD37030BC70474FF01F
:10052000000310F8012B013943EA0203F9D1A3F1CA
:1005300001034FEAD37070472DE9F00791E8F807FF
:10054000B2E802105B1854EB0C04B2E802104D4103
:1005500056EB0C06B2E802104F4158EB0C08B2E81B
:10056000021059EB01095AEB0C0A8941B3F1FF3330
:1005700074F1FF3475F1FF3576F1000677F100076D
:1005800078F1000879F101097AF1FF3A51F100019F
:100590004A425B184C414D4156F1000657F10007A5
:1005A00058F1000859EB02095AEB010A80E8F807F4
:1005B000BDE8F00770472DE9F00791E8F807B2E8C9
:1005C00002105B1A74EB0C04B2E802108D4176EB5A
:1005D0000C06B2E802108F4178EB0C08B2E802106A
:1005E00079EB01097AEB0C0A89414A425B184C41CC
:1005F0004D4156F1000657F1000758F1000859EB3C
:1006000002095AEB010A80E8F807BDE8F0077047D5
:100610000A462DE9F04F41EC140A92EC080A91E8E1
:10062000390010EE101AA0FB01784FF00009E3FB2F
:1006300001894FF0000AE4FB019A4FF0000BE5FB43
:1006400001AB12EE101A4FF0000CE0FB01BC4FF0B2
:10065000000EE3FB01CE4FF00002E4FB01E24FF09D
:100660000006E5FB012605EE107A10EE901A4FF019
:100670000007E0FB018719EB07094FF0000747EB84
:100680000707E3FB01971AEB070A4FF0000747EB58
:100690000707E4FB01A71BEB070B4FF0000747EB35
:1006A0000707E5FB01B712EE901A1CEB070C4FF0A1
:1006B000000747EB0707E0FB01C71EEB070E4FF0F3
:1006C000000747EB0707E3FB01E7D2194FF00007EC
:1006D00047EB0707E4FB0127F6194FF0000747EB4C
:1006E0000707E5FB016705EE908A11EE101A4FF03F
:1006F0000008E0FB01981AEB080A4FF0000848EBED
:100700000808E3FB01A81BEB080B4FF0000848EBBF
:100710000808E4FB01B81CEB080C4FF0000848EB9C
:100720000808E5FB01C813EE101A1EEB080E4FF087
:10073000000848EB0808E0FB01E812EB08024FF064
:10074000000848EB0808E3FB012816EB08064FF009
:10075000000848EB0808E4FB016817EB08074FF0B6
:10076000000848EB0808E5FB017806EE109A11EE48
:10077000901A4FF00009E0FB01A91BEB090B4FF0A9
:10078000000949EB0909E3FB01B91CEB090C4FF027
:10079000000949EB0909E4FB01C91EEB090E4FF002
:1007A000000949EB0909E5FB01E913EE901A12EB88
:1007B00009024FF0000949EB0909E0FB012916EB9A
:1007C00009064FF0000949EB0909E3FB016917EB42
:1007D00009074FF0000949EB0909E4FB017918EB1F
:1007E00009084FF0000949EB0909E5FB018906EE0C
:1007F00090AA14EE901A01F1100191E8390010EE60
:10080000101A4FF0000AE0FB01BA1CEB0A0C4FF083
:10081000000A4AEB0A0AE3FB01CA1EEB0A0E4FF07C
:10082000000A4AEB0A0AE4FB01EA12EB0A024FF063
:10083000000A4AEB0A0AE5FB012A12EE101A16EB2F
:100840000A064FF0000A4AEB0A0AE0FB016A17EBBE
:100850000A074FF0000A4AEB0A0AE3FB017A18EB99
:100860000A084FF0000A4AEB0A0AE4FB018A19EB76
:100870000A094FF0000A4AEB0A0AE5FB019A07EE63
:1008800010BA10EE901A4FF0000BE0FB01CB1EEBFC
:100890000B0E4FF0000B4BEB0B0BE3FB01EB12EBE2
:1008A0000B024FF0000B4BEB0B0BE4FB012B16EB99
:1008B0000B064FF0000B4BEB0B0BE5FB016B12EE45
:1008C000901A17EB0B074FF0000B4BEB0B0BE0FBF9
:1008D000017B18EB0B084FF0000B4BEB0B0BE3FB12
:1008E000018B19EB0B094FF0000B4BEB0B0BE4FBEF
:1008F000019B1AEB0B0A4FF0000B4BEB0B0BE5FBCC
:1009000001AB07EE90CA11EE101A4FF0000CE0FB9D
:1009100001EC12EB0C024FF0000C4CEB0C0CE3FB67
:10092000012C16EB0C064FF0000C4CEB0C0CE4FB0E
:10093000016C17EB0C074FF0000C4CEB0C0CE5FBBB
:10094000017C13EE101A18EB0C084FF0000C4CEB66
:100950000C0CE0FB018C19EB0C094FF0000C4CEB7C
:100960000C0CE3FB019C1AEB0C0A4FF0000C4CEB57
:100970000C0CE4FB01AC1BEB0C0B4FF0000C4CEB34
:100980000C0CE5FB01BC08EE10EA11EE901A4FF0DA
:10099000000EE0FB012E16EB0E064FF0000E4EEBA4
:1009A0000E0EE3FB016E17EB0E074FF0000E4EEB41
:1009B0000E0EE4FB017E18EB0E084FF0000E4EEB1E
:1009C0000E0EE5FB018E13EE901A19EB0E094FF097
:1009D000000E4EEB0E0EE0FB019E1AEB0E0A4FF0DE
:1009E000000E4EEB0E0EE3FB01AE1BEB0E0B4FF0B9
:1009F000000E4EEB0E0EE4FB01BE1CEB0E0C4FF096
:100A0000000E4EEB0E0EE5FB01CE54EC173A18EE3D
:100A1000101A13EB0A0354EB0B0451EB0C0152EBCD
:100A20000E02002040F1000013EB0B0354EB0C040A
:100A300051EB0E0152EB0E0246410020474158EBAC
:100A4000000859EB0A0940F10000B3EB0E0374F102
:100A5000000471F1000172EB0A0276EB0B0677EBF2
:100A60000C0778EB0A0879EB0C0960F10000B2EB97
:100A70000B0276EB0C0677EB0E0778EB0B0879EBA5
:100A80000E0960F100005FEAE07C7FEA0C0CDCF10B
:100A9000000EB3EB0C0374EB0C0471EB0C0172F160
:100AA000000276F1000677F1000778EB0E0879EB8B
:100AB0000C0960F100005FEAE07CDCF1000E13EB52
:100AC0000C0354EB0C0451EB0C0152F1000256F1F3
:100AD000000657F1000758EB0E0859EB0C0940F1DE
:100AE00000005FEAE07CDCF1000E13EB0C0354EB3A
:100AF0000C0451EB0C0152F1000256F1000657F1C3
:100B0000000758EB0E0859EB0C095BEC15AA5EECDC
:100B100016CA1AEB060A5BEB070B5CEB080C5EEBE4
:100B2000090E002040F100001AEB070A5BEB080BEE
:100B30005CEB090C5EEB090E43410020444141414E
:100B4000724140F10000BAEB090A7BF1000B7CF125
:100B5000000C7EEB060EBB4174EB0804B14172EB56
:100B6000080260F10000BEEB070E73EB080374EBA4
:100B70000904B94172EB090260F100005FEAE07814
:100B80007FEA0808D8F10009BAEB080A7BEB080BEA
:100B90007CEB080C7EF1000E73F1000374F100048D
:100BA00071EB090172EB080260F100005FEAE07886
:100BB000D8F100091AEB080A5BEB080B5CEB080C98
:100BC0005EF1000E53F1000354F1000451EB0901F2
:100BD00052EB080240F100005FEAE078D8F100092A
:100BE0001AEB080A5BEB080B5CEB080C5EF1000EDD
:100BF00053F1000354F1000451EB090152EB0802D8
:100C000014EE100AA0E8005C18C080E80600BDE8F9
:100C1000F08F00BF70B491E87800B2E802105B1862
:100C200054EB0C04B2E802104D4156EB0C0680E880
:100C300078008041013070BC704770B491E8780052
:100C4000B2E802105B1A74EB0C04B2E802108D419A
:100C500076EB0C0680E878008041404270BC70471B
:100C60002DE9F00791E8F807B2E802105B1854EBA1
:100C70000C04B2E802104D4156EB0C06B2E802102B
:100C80004F4158EB0C08B2E8021059EB01095AEB3E
:100C90000C0A80E8F80780410130BDE8F007704792
:100CA0002DE9F00791E8F807B2E802105B1A74EB3F
:100CB0000C04B2E802108D4176EB0C06B2E802108B
:100CC0008F4178EB0C08B2E8021079EB01097AEB5E
:100CD0000C0A80E8F80780414042BDE8F007704701
:100CE0002DE9F007524290E87800B1E880071740FC
:100CF000DB1918EA020854EB080419EA020955EB5B
:100D000009051AEA020A56EB0A0678C090E878004C
:100D1000B1E8800717407B4118EA020854EB080449
:100D200019EA020955EB09051AEA020A56EB0A0606
:100D300078C080410130BDE8F00770472DE9F00729
:100D4000524290E87800B1E880071740DB1B18EAB0
:100D5000020874EB080419EA020975EB09051AEA9E
:100D6000020A76EB0A0678C090E87800B1E88007BE
:100D70001740BB4118EA020874EB080419EA02099B
:100D800075EB09051AEA020A76EB0A0678C080417B
:100D90004042BDE8F007704790E8300091E8C0009D
:100DA000A31B1340E41AF618EB1B1340ED1AFF18AF
:100DB00030C0C0C17047F0B55242FFF7EDFFFFF7FA
:100DC000EBFFFFF7E9FFFFF7E7FFF0BD2DE9F007C5
:100DD0003AC91668A1FB069A4FF0000CE3FB06AC7B
:100DE0004FF00007E4FB06C74FF00008E5FB06786C
:100DF00040F8049B56684FF00009E1FB06A91CEB84
:100E0000090C4FF0000949EB0909E3FB06C917EB90
:100E100009074FF0000949EB0909E4FB067918EBD3
:100E200009084FF0000949EB0909E5FB068940F87C
:100E300004AB96684FF0000AE1FB06CA17EB0A07FD
:100E40004FF0000A4AEB0A0AE3FB067A18EB0A089D
:100E50004FF0000A4AEB0A0AE4FB068A19EB0A097A
:100E60004FF0000A4AEB0A0AE5FB069A40F804CB69
:100E7000D6684FF0000CE1FB067C18EB0C084FF035
:100E8000000C4CEB0C0CE3FB068C19EB0C094FF03F
:100E9000000C4CEB0C0CE4FB069C1AEB0C0A4FF01C
:100EA000000C4CEB0C0CE5FB06AC80E88017BDE8B1
:100EB000F00770470A462DE9F04F41EC140A92EC16
:100EC000080A91E8390010EE101AA0FB01784FF0E3
:100ED0000009E3FB01894FF0000AE4FB019A4FF09F
:100EE000000BE5FB01AB12EE101A4FF0000CE0FB1B
:100EF00001BC4FF0000EE3FB01CE4FF00002E4FB1B
:100F000001E24FF00006E5FB012605EE107A10EE37
:100F1000901A4FF00007E0FB018719EB07094FF02B
:100F2000000747EB0707E3FB01971AEB070A4FF0AF
:100F3000000747EB0707E4FB01A71BEB070B4FF08C
:100F4000000747EB0707E5FB01B712EE901A1CEB11
:100F5000070C4FF0000747EB0707E0FB01C71EEB4C
:100F6000070E4FF0000747EB0707E3FB01E7D21935
:100F70004FF0000747EB0707E4FB0127F6194FF096
:100F8000000747EB0707E5FB016705EE908A11EEC6
:100F9000101A4FF00008E0FB01981AEB080A4FF016
:100FA000000848EB0808E3FB01A81BEB080B4FF017
:100FB000000848EB0808E4FB01B81CEB080C4FF0F4
:100FC000000848EB0808E5FB01C813EE101A1EEBF9
:100FD000080E4FF0000848EB0808E0FB01E812EBB0
:100FE00008024FF0000848EB0808E3FB012816EB65
:100FF00008064FF0000848EB0808E4FB016817EB0F
:1010000008074FF0000848EB0808E5FB017806EEFA
:10101000109A11EE901A4FF00009E0FB01A91BEBAA
:10102000090B4FF0000949EB0909E3FB01B91CEB7F
:10103000090C4FF0000949EB0909E4FB01C91EEB5B
:10104000090E4FF0000949EB0909E5FB01E913EE30
:10105000901A12EB09024FF0000949EB0909E0FB75
:10106000012916EB09064FF0000949EB0909E3FBDA
:10107000016917EB09074FF0000949EB0909E4FB87
:10108000017918EB09084FF0000949EB0909E5FB64
:10109000018906EE90AA14EE901A01F1100191E870
:1010A000390010EE101A4FF0000AE0FB01BA1CEBF9
:1010B0000A0C4FF0000A4AEB0A0AE3FB01CA1EEBD6
:1010C0000A0E4FF0000A4AEB0A0AE4FB01EA12EBAF
:1010D0000A024FF0000A4AEB0A0AE5FB012A12EE67
:1010E000101A16EB0A064FF0000A4AEB0A0AE0FB58
:1010F000016A17EB0A074FF0000A4AEB0A0AE3FB02
:10110000017A18EB0A084FF0000A4AEB0A0AE4FBDE
:10111000018A19EB0A094FF0000A4AEB0A0AE5FBBB
:10112000019A07EE10BA10EE901A4FF0000BE0FB98
:1011300001CB1EEB0B0E4FF0000B4BEB0B0BE3FB4D
:1011400001EB12EB0B024FF0000B4BEB0B0BE4FB34
:10115000012B16EB0B064FF0000B4BEB0B0BE5FBDB
:10116000016B12EE901A17EB0B074FF0000B4BEBD5
:101170000B0BE0FB017B18EB0B084FF0000B4BEB6C
:101180000B0BE3FB018B19EB0B094FF0000B4BEB47
:101190000B0BE4FB019B1AEB0B0A4FF0000B4BEB24
:1011A0000B0BE5FB01AB07EE90CA11EE101A4FF0E6
:1011B000000CE0FB01EC12EB0C024FF0000C4CEBCE
:1011C0000C0CE3FB012C16EB0C064FF0000C4CEB67
:1011D0000C0CE4FB016C17EB0C074FF0000C4CEB14
:1011E0000C0CE5FB017C13EE101A18EB0C084FF009
:1011F000000C4CEB0C0CE0FB018C19EB0C094FF0D4
:10120000000C4CEB0C0CE3FB019C1AEB0C0A4FF0AE
:10121000000C4CEB0C0CE4FB01AC1BEB0C0B4FF08B
:10122000000C4CEB0C0CE5FB01BC08EE10EA11EED7
:10123000901A4FF0000EE0FB012E16EB0E064FF059
:10124000000E4EEB0E0EE3FB016E17EB0E074FF098
:10125000000E4EEB0E0EE4FB017E18EB0E084FF075
:10126000000E4EEB0E0EE5FB018E13EE901A19EBFD
:101270000E094FF0000E4EEB0E0EE0FB019E1AEB36
:101280000E0A4FF0000E4EEB0E0EE3FB01AE1BEB11
:101290000E0B4FF0000E4EEB0E0EE4FB01BE1CEBEE
:1012A0000E0C4FF0000E4EEB0E0EE5FB01CE14EED1
:1012B000100AA0EC075A80E8C45FBDE8F08F00BFB9
:1012C00008B5094801F030FF084801F02DFF012161
:1012D000002002F0DDFB20B1BDE80840044801F029
:1012E00023BF02F01DFCFCE7300B05004C0B050092
:1012F0006A0B050008B50446084611461A46A04781
:1013000003F072FC01F048F970B50C254D43C66836
:1013100090F90B0074198842A8BF21464FF02004B1
:1013200092FBF4F4B8BF715902F01F0001EB840185
:10133000196070BD07B501ABFFF7E6FF0123019A05
:1013400003FA00F013680343136003B05DF804FB75
:1013500007B501ABFFF7D8FF0123019A03FA00F0AC
:10136000136823EA0003136003B05DF804FB10F078
:10137000010005D04FF02003EFF3118083F31188B3
:1013800070472DE9F8430446FF2200214FF00C0E70
:101390004368058900685D4394F80AC02844E272F6
:1013A0008C4505DC00252389AB4222DCBDE8F883AF
:1013B000B5FBF3F20EFB01F7D4F80C801F2A08EB03
:1013C0000706C8BF1F324FEA930306F10409C8BFDE
:1013D000520903F10303C6E9019923F00303D4BFC3
:1013E000E17248F8070001F10101C8BF00EB82007B
:1013F000D6E76268E3686A4320681E1D811886503C
:101400009A6820464A609A68116099602A460021CD
:10141000FFF790FF0135C6E72DE9F04F8BB0867AD4
:1014200000AFC7E90232B3000A3303F4FF63ADEB48
:10143000030DE9464A4643680446033323F0030399
:1014400042F804394FF0FF3500234FF00C0C581EC2
:101450009E42786209DD2BB110688008033020F0CD
:1014600003005060506888420BD27B6A013314D16C
:1014700000236FF00B003A6D13602C37BD46BDE8BA
:10148000F08FE06804320CFB030000F1040E4068AA
:10149000704518BF1D460133D9E76E1CE8D0207C8B
:1014A000FFF765FF0C236B431A1DE3683862134492
:1014B0001E68B34277D0D6E900131960316859F835
:1014C00025204B6023682946F31A93FBF2F220464D
:1014D000FFF73EFFA9EB890305F1010B3B6109EB27
:1014E00085057A6A0BF1FF339A4216DC237CD90713
:1014F00002D53B6A83F31188FB6800201A467B6A99
:1015000013607A6A236859F82220F31A93FBF2F3E6
:10151000BA6813603B6D1E60AFE7236855F8042B73
:10152000F31A93FBF2F34FF0010A9B003A69BB6197
:1015300005EB450313447B61D5F8008059460AFB4F
:1015400008F3FB61F3187B60BB6920460AEB0302DA
:10155000FFF7F0FE7B68226808F1FF389844A8EB9B
:101560000208218962684A4390450AD2E268796993
:10157000F8690A44111D31509168596091680B60F7
:1015800093600AF1010ABAF1040FD5D1237CD80780
:1015900002D53B6A83F31188207CFFF7E8FE0BF14C
:1015A000010B38629DE7013D6A1CA6F10C037FF434
:1015B0007FAF00269AE72DE9F04F87B0837A00AF1E
:1015C0009B000A3303F4FF63ADEB030DE946436868
:1015D00004464D460120033323F00303C9F80030CD
:1015E00081426ED2207C0D461646FFF7C0FE804633
:1015F00059F82530324603FB06FBFB602368294679
:10160000204603EB0B0ABB60FFF794FE0C23E26855
:1016100003FB0522BB68111D43F80B109368CAF841
:1016200004309368C3F800A0C2F808A0237CDA074E
:1016300001D588F31188207CFFF799FE8046002DA4
:1016400048D007F11403324629462046FFF75CFED6
:10165000042390FBF3F07A6983001068D84000F00F
:101660000F000F2836D14FF0000A26F00303BB60AD
:10167000FB68013BBA68F968524401FB02FBB4F80D
:1016800008C0616803EB0B0001FB0CF188420FD22C
:10169000294620467B60FFF75BFE22687B6802EBF1
:1016A0000B0152F80B004968086052F80B2051609A
:1016B0000AF1010ABAF1040FDCD1013D96FBFAF6FA
:1016C00096E72B6801309B08033323F0030345F8AA
:1016D000043F85E7237CDB0701D588F311881C379D
:1016E000BD46BDE8F08F0020704700000B68013355
:1016F0000B60014B1B681847306F02202DE9F04F3B
:1017000085B00E9C9B46012CB8BF0124012B0CBF59
:101710003023202315468046894601260A270022C9
:10172000DFF870A0019402930AF101040AB9AA45F6
:101730001ED2B5FBF4F049463030C04701220136D5
:10174000B5FBF4F10A23013F012F04FB1155BAFB4D
:10175000F3FAE9D1494605F13000C047BBF1030F68
:1017600003D1019B9C1B002C0FDC05B0BDE8F08F62
:10177000019BBB42E4DBBBF1020FE1D84946029872
:1017800003920136C047039ADAE749462020C04752
:10179000013CE8E7FFC99A3B014B1860704700BF66
:1017A000306F02202DE9F04F4FF0000A06460F4639
:1017B0004FF0FF39D04689B01C46531E04930025D4
:1017C00005E06DB9252800F011813946B047049B2A
:1017D00013F8010F04930028F3D109B0BDE8F08F8E
:1017E000642861D019D839280AD8312850D22D2838
:1017F0003CD030283DD0252808D13946B047DEE717
:10180000582800F08880632800F0EA8039462520B7
:10181000B047049B39461878F0E7702871D006D895
:10182000692841D06C283CD06828D0D0EEE77528D4
:1018300057D017D87328E9D1236804F1040B1C464C
:10184000254615F8010B002840F0BF80B8F1030FC2
:1018500040F0D580E41AA9EB0404002C00F3BB800F
:101860005C46ACE7782856D07A28DEE74FF00308CC
:10187000ADE7B9F1000F0EDAB8F1000F00F0BC804F
:10188000A0F13009B8F1000F08BF4FF002089EE741
:10189000B9F1000FF4DB0A2303FB0909A9F13009B0
:1018A000F0E70AF1010A92E7BAF1010FC5BF073468
:1018B00024F0070325681D68D4BF043403F108042D
:1018C000002D05DA39462D20B0476D4209F1FF3968
:1018D00043462A46CDF8009039463046FFF70EFFC2
:1018E0006DE7BAF1010FC5BF073424F00703226882
:1018F0001A68CCBF03F108040434CDF800904346C5
:10190000EAE739463020B04739467820B0474FF0F3
:1019100008094FF001080822BAF1010FC5BF0734CA
:1019200024F00703236803F10804CABF1B6805936A
:1019300005934FF000039346D8BF043403930793F5
:101940000BF1FF3B059B4FEA8B0023FA00F010F0F0
:101950000F0009D1079B13B9BBF1000F24D14FF041
:10196000300C07E0069AEBE709288CBF4FF0570CC4
:101970004FF0300C394660440692B047039B079500
:1019800001330393BBF1000FECD1B8F1030F7FF4E7
:1019900016AF039BC3EB4905002D7FF710AF394607
:1019A0002020B047013DF7E7531E91450693E9DB40
:1019B000B8F1010F03D139463020B047E2E7B8F162
:1019C000020FDFD139462020F7E7394603932C4632
:1019D000B047039B34E739462020B047013C3CE741
:1019E0002068251D3946B0472C46E8E6AA46A84699
:1019F0004FF0FF390125EAE64FF00108E7E65C46C3
:101A00000546E4E6002313B502AC44F8043D024663
:101A10000B4603482146FFF7C5FE02B010BD00BFCC
:101A2000ED1604000FB407B504A951F8040B019199
:101A3000FFF7E8FF03B05DF804EB04B070477047B0
:101A400010B54FF02003EFF3118483F3118800F0F9
:101A500011F80122054BC3F840254FF0FF32044B2B
:101A60009A62DA6284F31188002010BD009003406E
:101A700000ED00E0074AD2F8883043F47003C2F862
:101A80008830BFF34F8FBFF36F8F034B034A1A6049
:101A9000704700BF00ED00E0346F02200090D003DB
:101AA0002DE9F041064604792420404D00FB045006
:101AB00090F82000002877D108683368471C0BD0C5
:101AC00001274FF0030EDFF8F4C08740CCF8087010
:101AD00000F180074CF827E0D1F804C0BCF1FF3FCB
:101AE0001FBF4FF00008DFF8D4E00CF180074EF87C
:101AF00027808F6991F814E0C3F824754F7DBEF1FB
:101B0000010F4EEA0707C3F86C75C3F80C05C3F85C
:101B100014C520D18F68781C1FBF4FF0000EDFF86E
:101B20009CC007F180004CF820E0C868B0F1FF3F8E
:101B30000DD04FF0010C4FF00308DFF880E00CFAF5
:101B400000FCCEF808C000F1800C4EF82C80C3F8E1
:101B50000805C3F81075242363430969E818426037
:101B6000E95082B100233068C0F81031C0F820314C
:101B7000C0F82431C0F844310D4BC0F8043340F3B1
:101B8000073000F031FC082233680A48C3F800250A
:101B90002423002203FB0453C3E906225A610122D5
:101BA00083F82020BDE8F0810348FBE70000022015
:101BB000100302000000AD0B0500AD0B00258440B2
:101BC00001F06043B3F1005FF0B529D12424057919
:101BD000164F04FB0574666926BB03686261C3F88F
:101BE0002061C3F85861C3F84415C3F848250122A1
:101BF000A1609A606268BAB9D3F82011D3F858216D
:101C000041B9002AF8D00A48242303FB05750023B4
:101C10006B61F0BD0648074B002A08BF1846F3E782
:101C20000548F6E70548F4E70248F2E7000002201D
:101C30000800AD0B0000AD0B0A00AD0B0B00AD0BA7
:101C4000014B1860704700BF304702200A2838B5A2
:101C50000446074D04D128680D2143685B68984706
:101C60002868E1B243685B689847204638BD00BFEA
:101C70002400022010B5044C204601F043FA20460F
:101C8000BDE81040FFF788BD4D1C040008B50448AE
:101C900002F004FC034B1860FFF7ECFF002008BDC6
:101CA000C30B05002400022010B54FF02003EFF312
:101CB000118283F31188114C237823B982F31188A0
:101CC0006FF0440010BD013BDBB2237023B182F3FF
:101CD00011886FF00F00F5E7094B0121187828B142
:101CE000217082F311886FF00A00EBE7197082F31C
:101CF0001188044A11601870E4E700BF2A0002202E
:101D0000290002200450004010B54FF02002EFF3EC
:101D1000118382F31188114C207880B183F31188EC
:101D20000F4AD2F81C34D2F8182403F0030343F40A
:101D30008033934314BF6FF04300002010BD012295
:101D4000227083F31188064BC3F80401C3F81815F9
:101D50000221C3F804139A60E2E700BF28000220C2
:101D600000500040174B30B5D3F80851D3F8042386
:101D7000D3F8004102F00102D3F80413D3F80401B0
:101D800015B10025C3F8085194B10024C3F80041EF
:101D90001AB101220B4BC3F8082340B10022094BB2
:101DA000C3F804218A0702D50222C3F8082330BDF4
:101DB000002AF2D0D3F80C3403F00113B3F1011F61
:101DC000EBD1E6E70050004008B5002201210520D4
:101DD00000F02EFB052000F007FB002008BD0000EE
:101DE000F8B54FF02002EFF3118382F31188254AF2
:101DF0001078441C147068B183F31188224BD3F817
:101E00000C3403F00113B3F1011F0CBF00206FF07D
:101E1000430007E01D4D2F782FB1107083F3118818
:101E20006FF00A00F8BD01262E7083F31188164C5E
:101E300021B3052000F0E8FAC4F80071D4F80433A7
:101E4000C4F804632660D4F800219AB10022DB07AD
:101E500058BF0123C4F800214FF0200258BFC4F836
:101E600008330B4B0520C3F8802100F0BDFA002396
:101E70002B70C3E720BF40BF20BFE4E7C4F80011C8
:101E80002660F4E72A0002200050004029000220CA
:101E900000E100E070474FF02003EFF3118083F37F
:101EA0001188704700230D4A10B5C2F84031FFF782
:101EB000F2FFD2F8043540F2471209490C681B1BA7
:101EC00023F07F43B3FBF2F302FB03420A6080F38B
:101ED00011881846BDE8104003F01CB800500140BE
:101EE0002C00022038B51B4802F0D8FA70B34368C2
:101EF00001211B689847002440F24713164D4FF408
:101F00000012C5F80845C5F840354FF48033C5F8D0
:101F10004433C5F80433114B01211C60104B1520CC
:101F2000C3F88021224600F083FA152000F05CFA05
:101F3000012320460B4A13602B60D5F8043503F2C9
:101F4000471323F07F43C5F8403538BD4FF0FF30CD
:101F5000FBE700BFE40B0500005001404051014089
:101F600000E100E00850014070B54CF66905B0F1A1
:101F7000FF3F14BF02462A46FFF78DFF124B134C5A
:101F80001E68531EAB42A8BF2B4640F24715D4F83B
:101F9000041523EAE3738A1B22F07F4202F5A37241
:101FA00005FB0323B3FBF5F305FB0363591A21F08B
:101FB0007F411F2998BF5B1923F07F43C4F8403548
:101FC00080F3118870BD00BF2C000220005001403A
:101FD00008B5FFF760FF084B084AD3F804351268CC
:101FE0009B1A40F2471223F07F43B3FBF2F380F3D6
:101FF0001188184608BD00BF005001402C00022087
:1020000004488168406A884203D003494FF08052F7
:102010000A607047604B022004ED00E0202080F34E
:1020200011880D498A684FF028001044EFF3098C9D
:1020300080E8F01F094F4FF000664A6A8A603E60F0
:10204000506E0023536680F3118802F1280090E857
:10205000F01F8CF309887047604B022004ED00E00C
:102060001EF0040F0CBFEFF30880EFF309808169C5
:1020700031F8021C11F0FF010229FFD000B500F079
:102080005BFA00BD014910220A60704710ED00E0C4
:10209000404080F3118830BF704700BF404080F35C
:1020A0001188DFF81CC0DCF800C01CF4006C0CBF09
:1020B000EFF30880EFF3098000B500F027F900BDC9
:1020C00004ED00E000B572B60B4A106A00281EBF8E
:1020D0000021116202F00EFA62B6EFF30580A0F162
:1020E00010004FEAC0000549014409C998475DF84E
:1020F00004EB034800470000604B0220780805000D
:1021000001200400002320210348C2180133412B81
:1021100082F80013F9D1704700E100E0084A09494C
:10212000936809685866996607494B6843F080537D
:102130004B60002383F311889368986E704700BF4B
:10214000604B02204411050000ED00E038B5194C49
:1021500005461948FFF766FCA36AD90602D5174859
:10216000FFF760FCA36A1A0702D51548FFF75AFC6F
:10217000A36A9B070ED51348FFF754FC616BA36A53
:10218000180607D51048FFF74DFC1DB1A36A23F0D0
:102190008003A362074CA26AD20702D50B48FFF75F
:1021A00041FCA36A9B0602D50948FFF73BFC0020CF
:1021B00038BD00BF00ED00E0530D05006A0D0500BD
:1021C0007C0D0500900D0500A90D0500C00D050052
:1021D000E00D050038B51E4C05461E48FFF722FCF1
:1021E000A36AD80409D51C48FFF71CFC184A002034
:1021F000936A43F47F43936238BDA36A190501D5FE
:102200001648F1E7A36A9A0514D51548FFF70AFCAA
:10221000A16BA36A1B0407D51248FFF703FC1DB18D
:10222000A36A23F40043A362094B9B6A5805DDD5DA
:102230000D48D9E7A36A5905FAD4A36ADA0501D58E
:102240000A48D1E7A36A9B04D0D50948CCE700BF70
:1022500000ED00E0040C05006A0D05007C0D050092
:102260001B0C0500350C05004B0C0500670C050028
:10227000E00D050010B51C4C1C48FFF7D3FBA36A0A
:102280009A0102D51A48FFF7CDFBA36ADB0102D5FC
:102290001848FFF7C7FBA36ADC0202D51648FFF710
:1022A000C1FB114CA36A180302D51448FFF7BAFB0F
:1022B000A36A590302D51248FFF7B4FBA36A9A0335
:1022C00002D51048FFF7AEFB074CA36ADB0302D52B
:1022D0000D48FFF7A7FBA36A00206FEA03436FEAEC
:1022E0001343A36210BD00BF00ED00E0100E050017
:1022F000290E05003D0E0500580E05006A0E05006A
:10230000890E0500AF0E0500CA0E050038B5274C32
:1023100005466368C3F30803DA1E092A3AD8DFE8E2
:1023200002F0053335303939393939372048FFF76C
:1023300079FBE36A9A0703D51E48FFF773FB02E0B7
:10234000E36A5B0005D400202946BDE8384000F070
:10235000C1B81948FFF766FB184B1B782BB1012059
:10236000FFF7F4FE0628EFD138BD154B1B781BB1E3
:102370000120FFF72FFFF5E7124B1B889BB2002BC4
:10238000E1D0FFF777FFEDE70020E9E70020F0E775
:102390000D48D2E70D480E49A3F110020F2BD8BF0C
:1023A00001460C48FFF73EFBCDE700BF00ED00E023
:1023B000AE0C0500C60C0500E80C050028ED00E099
:1023C00029ED00E02AED00E0080D0500800C050075
:1023D000950C05003F0D0500024A536943F01003B8
:1023E0005361704700ED00E043B2002B08DB01228F
:1023F00000F01F0002FA00F0024A5B0942F82300D5
:10240000704700BF00E100E043B2002B0DDB01226A
:1024100000F01F0002FA00F05B09044A203342F882
:102420002300BFF34F8FBFF36F8F704700E100E0D1
:1024300043B2002B01F10101A8BF03F160434FEA51
:102440004111B8BF054BC9B2ABBF03F5614300F002
:102450000F0083F800131954704700BF14ED00E01B
:10246000FFF71CBE08B572B6044B186A18B10022FB
:102470001A6202F03FF862B608BD00BF604B02204E
:1024800070470000F8B516460C461F4604220A9B0A
:102490000999054602F092FC0023A6F168010C4A56
:1024A000214421F0070122F00102C5E91333C5E9F7
:1024B00016468A61069A0F604A60079A8A60089AEF
:1024C000CA604FF08072CA61A9646B66F8BD00BF34
:1024D000F512040038B504460D4605281AD8DFE881
:1024E00000F00319191315170D48FFF79BFA02F0B6
:1024F0007BFBAA6901460B48FFF794FA2946204660
:10250000BDE8384000F01CB80748EEE70748ECE7A4
:102510000748EAE701460748FFF784FAE7E700BF04
:10252000F60E0500940F0500160F05003C0F050080
:10253000560F0500710F050001460068FFF7CABF7E
:10254000052810B50CD002F081FB60B102F07EFBD3
:102550000C490D4B002808BF19460C48FFF762FADA
:10256000FFF796FDFCE702F081FB0028EED1084C56
:102570000848A168FFF756FAA068BDE8104000F0CF
:102580000BB800BFD00F0500D40F0500E50F050004
:10259000604B02200510050038B505464FF02003BA
:1025A000EFF3118483F3118802F09AFB0A4B9B68C6
:1025B000AB420BD1094B5A68C2F3080212B920464C
:1025C000FFF7ACFD5A6842F080525A602046BDE8E1
:1025D000384002F0E5B900BF604B022000ED00E09A
:1025E000202080F3118806484FF40061401880F3E2
:1025F0000988022080F31488BFF36F8F00F006F87B
:102600003067022030BFFFF7FDBF00BF104A08B59A
:10261000104B22F07F029A60BFF34F8FBFF36F8F92
:10262000D3F8882042F47002C3F888204FF00042AB
:10263000C3F83422BFF36F8FB0EE400ABFF36F8F41
:1026400001F072FF01F07AFFFFF75CFD01F09AFFE5
:102650000000040000ED00E008B5FFF7D3FFBDE87F
:102660000840FFF7CDBC00000522034B5A60BFF3C2
:102670004F8FBFF36F8F704790ED00E0BFF35F8F18
:102680000022014B5A60704790ED00E0184919484C
:102690000B6870B50468C3F307239C4225D8FFF785
:1026A000EDFF4FF6AA73426800200B63844202F1EB
:1026B000100603D1FFF7D8FF002070BD157A56F839
:1026C000103C05F01F0223F01F031A4356F8043C88
:1026D0006D0923F01F0343F0010343EA45038860BB
:1026E000CA6001300B613246E0E74FF0FF30E4E7AB
:1026F00090ED00E08C0B0500C9B2027803468A42D7
:1027000000F1010004D0002AF7D1002918BF0023EE
:102710001846704702460346981A13F8011B002911
:10272000FAD170470138013910F8013F11F8012F33
:10273000934202D1002BF7D11A46981A704730B550
:102740000024A24208D0035D0D5DAB4202D10134EA
:10275000002BF6D1581B00E0002030BD431A9342F5
:1027600010B500EB020308D3024601399A420BD0A0
:1027700011F8014F02F8014BF8E70A4412F8014D35
:102780008A4203F8014DF9D110BDF0B581EA000489
:10279000A50703460BD0013B0A4491421DD1F0BD71
:1027A000002AFCD011F8014B013A03F8014B9C07B9
:1027B000F6D10C461D1F8F183E1B032E08D86FF054
:1027C0000305940805FB0422A40023442144E2E706
:1027D00054F8046B45F8046FEEE711F8014B03F869
:1027E000014FDAE70346F0B5C9B29C070FD11D4689
:1027F00041EA012444EA04449F187E1B032E0CD8AE
:10280000940803EB840413449C4209D1F0BD002AD0
:10281000FCD003F8011B013AE7E745F8044BECE76D
:1028200004F8011BF0E770B50446B1FBF2F602FBB9
:1028300016110929CDB28CBF27210021303529443A
:1028400004F8011B3146002EEFD13021221A9342A9
:1028500007DC2346002103F80119834204D81046FF
:1028600070BD04F8011BF1E71978047803F80149F9
:1028700000F8011BF1E7D0E900232DE930485FEAB9
:10288000530C4FEA320B002502F001041BEB04024B
:102890004CEB0503C0E90023BDE830880521D0E9F1
:1028A00000232DE9F04F12F1020843F10009B9FBB2
:1028B000F1F5002601FB05F7B8EB060869EB0709FF
:1028C0004FEAD80646EA4976B6FBF1FC0024C24638
:1028D0004FEACC06A6FB0189A2194FEA5C7745EBCB
:1028E00007031446BAEB0802B2FBF1F21D46A41826
:1028F00045F10005C0E90045BDE8F08F0B682DE902
:102900001048002B13DD013B0B600A21026844686C
:10291000A2FB01BC5A4601FB04CC2CF07043C0E979
:1029200000234FEA1C713031C8B2BDE81088302155
:10293000FAE700002DE9F04F1F4600239346C9B087
:10294000CDE90C0104939BF800000BF1010548B19F
:10295000252879D0DDE90C319847013006D14FF0B8
:10296000FF330493049849B0BDE8F08FAB46049B55
:102970000133CDE90437059FE5E7232C5DD052D81C
:10298000002CEFD0202C08BF4FF001095D46AB466C
:102990001BF8014BBD482146FFF7AEFE0028ECD1E5
:1029A0002A2C59D13A683B1D002A0392BEBF5242DD
:1029B000039201221F466C78B8BF069205F1020B04
:1029C000039BC92B28BFC82303932E2C69D19BF8E6
:1029D00000302A2B62D13D680BF1010B0437C92D61
:1029E000A8BF4FF0FF359BF800400BF1010B2146CB
:1029F000A748FFF781FE18B19BF800400BF1010BCF
:102A0000672C7CDC652C80F2E080472C4CDC452C6C
:102A100080F2DB80002CA5D0252C00F03583C82C5B
:102A200040F33C839BE72D2C0BD0302C07D02B2C74
:102A3000079B08BF01230793A8E70126A6E7029496
:102A4000A4E701230693A1E74FF000092023CDE975
:102A5000069902934E469AE7A4F13003092B03909E
:102A6000B3D80A22AB461BF8010BA0F13003092BA7
:102A70000446A5D8039B5D4602FB0300A0F130038A
:102A80000393EFE7934600FB0535303D5A4612F8B5
:102A9000013BA3F130010929F4D9A0E700250A2060
:102AA000F4E74FF0FF35A2E7632C6FD032DC582CEF
:102AB000B5D13B1D05933968002E00F0DC8247F646
:102AC00030030DF15607ADF854302B46102238462E
:102AD000FFF7A9FE582C06D10DF1530212F8013F61
:102AE000002B40F0CA820DF15408002EA7EB080815
:102AF000404414BF4FF002094FF0000929E0702C48
:102B000000F094822BDC6E2C00F0538200F357828D
:102B1000692C84D13C683B1D002C059342DA2D239F
:102B2000B4F1004F8DF8543041D061420DF1550899
:102B30002B4640460A22FFF776FE079B804415A8E5
:102B4000A8EB0000002B3DD1B9F1000F01D14FEAF5
:102B5000D4790135029B18BF2023029380E0752CA5
:102B600000F08082782CA4D0732C7FF458AF00261C
:102B70003B1D396805938B5D002B00F066820136A2
:102B8000C82EF8D1002D80F2628266E23B1D0593CB
:102B90003B6801268DF8543000238DF855304FF0F6
:102BA00000091CE2079B23B12B238DF854302146EA
:102BB000BCE7B9F1000F01D02023F6E721460DF163
:102BC0005408B5E7DDF81C90C3E7073727F007077F
:102BD00007F108030593D7E900C7FB0243EA5C53FA
:102BE00023F000410B464FEACC22CDE9102340F2FE
:102BF000FF731046C7F30A589845CDE900016046B7
:102C000048D1DDE90012002877F10003B8BF2D2379
:102C100015A8AEBF03468DF854300DF155030A4395
:102C2000A4F1410403F1030825D1192C1DD8492230
:102C30001A704E225A7046229A700022DA70079B50
:102C4000A8EB0000002B40F05582B9F1000F07D12E
:102C50009DF85410A1F12D03D3F1000949EB0309AC
:102C6000C8283FF77CAE0646B9E169221A706E2289
:102C70005A706622E0E7192C99BF4E2241216E223C
:102C8000612194BF1A701A705970D5E72A10050097
:102C900030100500462CDDE9002342EA080243EA31
:102CA000E87308BF6624134343D0DDE900230028FE
:102CB00043F00043CDE9102377F10003A8F2FE387A
:102CC00039DA2D238DF854300DF1550A0023009385
:102CD00018F1020F3EDBB8F1000F79DC10A808F103
:102CE0000108FFF7C8FDB8F1040FF7D1002D24F05B
:102CF0002003B8BF0625472B40F09780002E40F0F8
:102D000092802B1C18BF01230893009B033304DB24
:102D1000009A6B1C9A4240F38D80672C0CBF65248F
:102D2000452405F10108102398450F93A8BF984644
:102D300089E04FF00008079B0BB12B23C2E7B9F1E4
:102D4000000F01D02023BDE70DF1540ABEE710A803
:102D5000FFF791FDDDE9107C00230B930023CDF8F4
:102D600028C0A94ADDE90A018B4208BF824208F166
:102D70000108ECD30522A7FB0201CDE90801099B5C
:102D800002FB0C334FF0000C0993DDE90823CDE979
:102D90001023009B013B0093002300216FF00040B3
:102DA000099A994208BF904207D2BCF1000F8FD018
:102DB000DDE90823CDE910238AE7DDE9082392182D
:102DC0005B41CDE9082308F1FF384FF0010CE3E740
:102DD00010A8FFF763FD4FF0000C009B08F1FF38CF
:102DE00001330093DDE91023CDE9082300230021FE
:102DF0006FF00040099A994208BF904208D2BCF196
:102E0000000F3FF468AFDDE90823CDE9102362E746
:102E1000DDE9082392185B41CDE9082308F1FF386A
:102E20004FF0010CE2E700236EE70023662C0893C5
:102E30007FF477AF009B13EB05084BD51023662476
:102E40004FF000080F9300224FF0006348A961E99A
:102E5000362318F1FF383FD2DDE91023DDE91201F6
:102E6000171843EB01083A464346CDE910230023E7
:102E700008F07042134308D010A8FFF70FFD10A808
:102E8000FFF7F9FC009B01330093662C0AF101085F
:102E900040D1009B002B29DD534498460FA910A870
:102EA000FFF72CFD0AF8010BC245F7D10023009370
:102EB00006B95DB12E2346464FF0300A88F800303F
:102EC00008EB0503B34215D10135A844089B002B3C
:102ED00039D160E0662426E708460A91FFF7DEFC58
:102EE0000A990846FFF7C7FC0A99B2E730238AF827
:102EF0000030DDE7009A2AB1013286F801A0009285
:102F00000136DFE70FA910A80A93FFF7F7FC0A9B29
:102F10007070F5E70FA910A8FFF7F0FC302818BF74
:102F2000009B8AF800001CBF03F1FF33009306B931
:102F30003DB12E230AF102088AF801304544454587
:102F40002ED1089B43B118F8012C08F1FF33302A29
:102F50002DD02E2A08BF984624F02003452B1AD1E5
:102F6000009B0A22002BBBBF5B4200932B232D2327
:102F700088F80130009B88F8004093FBF2F303F1DE
:102F8000300188F80210009908F1040802FB1317B9
:102F9000303708F8017C002315A888F800304EE689
:102FA0000FA910A8FFF7AAFC08F8010BC7E798467D
:102FB000C9E73B1D0593049A3B681A60DBE43B1D9F
:102FC0000593396816B330238DF8543059BB013559
:102FD000029B18BF202389468DF855100293039B4E
:102FE000B34240F38580069B15AD002B58D02023BB
:102FF000039AAB550136B242FAD1DDE9033215AC82
:1030000013441D46A41A6FE03233333315A80DF173
:1030100054082B460822A0EB0808FFF704FC4044A4
:103020004FF0000995E50DF15500F0E73B1D0593C4
:1030300047F630033968ADF85430102208230DF1FB
:103040005600FFF7F0FB0230EAE7002D02DBAE424C
:10305000A8BF2E46002E3FF48EAC324615A8FFF7CF
:1030600094FB9CE53B1D05930A222B46396815A865
:10307000FFF7D9FBD4E715AF27E5A3F161011929C3
:103080009CBF203B137029E50D9920460C9B984767
:1030900001303FF464AC049B0133049305976AE468
:1030A000039B721C9C1B28192946FFF757FB069BA4
:1030B000029A202A18BF4B4606931C44069BA34243
:1030C0009BDA069B1A46029BAB54134601330693C8
:1030D000F4E7049B0D99E05C0C9B984701303FF4AA
:1030E0003EAC049B01330493049BAB42F1D142E418
:1030F000039682E7DDF81C90B2E500BF4FF0FF3089
:1031000070470000014B1860704700BF386F022005
:10311000022902D1024B1B6818474FF0FF3070475D
:10312000386F0220FFF7F4BF0FB407B504AB53F8B4
:10313000042B022104480193FFF7FCFB03B05DF868
:1031400004EB04B0704700BF253104007047000055
:103150008279044B03EB4213DB69C01A024BC010A7
:103160005843704798700220ABAAAAAA10B5094B21
:10317000827903EB42139B690A685C6823689A4270
:1031800094BF0A600B60FFF7E3FFD4E9002302FB62
:10319000003010BD98700220002208B511462A2088
:1031A000FFF746F901F044FF002008BD684620F013
:1031B00007018D4601B5FFF763F904F0B5FAFFF793
:1031C00051F9FEF71DFFBDE801408546704768468E
:1031D00020F007018D4601B5FFF752F902F052F8D1
:1031E000FFF740F9FEF70CFFBDE801408546704748
:1031F000684620F007018D4601B5FFF741F902F05E
:1032000039FCFFF72FF9FEF7FBFEBDE801408546CC
:103210007047002070472F2810B504460CD023DCDF
:10322000162809D012DC092806D009DC022803D0B0
:10323000052801D001283BD101F056F9046010BDEA
:103240000D28F9D00E28F7D00C28F4E72A28F3D05F
:1032500005DC232830D02928EED01828EBE72C28CD
:10326000EAD02EDB2D28E6E7692832D00EDC36289E
:10327000E2D005DC322828D03328DDD03028DAE748
:103280003928D9D03C28D7D03828D4E77E282CD06C
:1032900009DC732821D07D2823D0702808D101F0C3
:1032A00023F943230BE0802829D023DB81282BD06E
:1032B00001F01AF9162302E001F016F90B2303605E
:1032C000BDE701F011F92B23F9E701F00DF93E23D9
:1032D000F5E701F009F93723F1E701F005F9442397
:1032E000EDE701F001F94823E9E701F0FDF840F2CC
:1032F000D173E4E701F0F8F840F2D273DFE701F0B0
:10330000F3F840F2D373DAE701F0EEF840F2D47349
:10331000D5E700004FF08052014BC3F80021704701
:1033200000E100E04FF08052014BC3F8802170476C
:1033300000E100E04FF00052014BC3F8002170475C
:1033400000E100E04FF00052014BC3F880217047CC
:1033500000E100E008B51D2000220621FFF768F813
:10336000BDE808401D20FFF73FB808B51C2000222B
:103370000621FFF75DF8BDE808401C20FFF734B8D0
:1033800030B589B06C46074D0FCD0FC495E80F00DE
:1033900084E80F00002269460348FEF781FB09B06C
:1033A00030BD00BF100B05006410050008B5FFF725
:1033B000DCFFFFF7E5FFBDE80840FFF7CBBF0000EB
:1033C0002DE9F04107460D460C46DFF8248014B97C
:1033D0002046BDE8F081FF2C264628BFFF26291B8A
:1033E000324639444046FEF7EBFBA41BEFE700BF33
:1033F000641005000138052812D8DFE800F0030743
:10340000090B0D0F02230B60002070470523FAE71C
:103410000623F8E70723F6E70423F4E70123F2E79E
:103420004FF0FF30704710F0400318BF02238207AF
:1034300048BF43F0080318467047112814D005DC34
:10344000C0B1062815D06FF02A00704740F2111362
:1034500098420BD040F2012398420BD0B0F5817F07
:10346000F1D14FF482707047022070474FF487709B
:10347000704701207047000008B50248FEF7E0FBE6
:10348000002008BD6C10050038B5044604B938BDED
:103490006069E56901F0D4F9204601F0D1F92C46C4
:1034A000F4E738B524230B7043880C460B810146A2
:1034B0001022054631F8043BA0186360FFF765F958
:1034C0002B7D236238BD2DE9F0438DB0149C054659
:1034D0000E46174698466CB91846FFF7A4FFCDE98B
:1034E000004403463A463146284604F07BFD0DB0C1
:1034F000BDE8F0832388022B0FD11021628804934A
:103500006368404606938DF80C10ADF81420FFF761
:103510008AFF03AB01910093E3E70A2B0CD10DF175
:103520000C0949462046FFF7BCFF4046FFF77BFFEA
:103530002423CDE90093D4E700F0D6FF6FF02203F7
:1035400003604FF0FF30D2E770B5044618461546C9
:10355000FFF769FF2A4603462046BDE8704004F0A5
:103560005DBD70B5044618461546FFF75CFF2A4658
:1035700003462046BDE8704004F086BDF0B591B02A
:1035800004460D461646002140226846FFF72AF9F8
:1035900004230022AA420CDB32462946684604F086
:1035A00013FE0022062316460127AA4221DB11B092
:1035B000F0BD54F832104DF83210E15A0132CF0705
:1035C00042BF3DF8030040F001002DF8030048071A
:1035D00042BF3DF8030040F002002DF80300090748
:1035E00042BF3DF8031041F004012DF803100833E9
:1035F000D0E73DF80310E65211F0010F18BFE75273
:10360000890748BFE15A02F1010244BF41F00401B9
:10361000E1520DEB030131F8021C490742BFE15AA8
:1036200041F00801E1520833BFE704F059BD04F04E
:10363000CBBC2DE9F043804687B01846DDE90E4645
:103640009146FFF7F0FE034654B9CDE900444A46DF
:10365000404604F0FDFC0546284607B0BDE8F0836F
:10366000082706AD45F80C7D04AA01950092404656
:103670004A4604F0EDFC059B0546022B07D1BDF838
:1036800018202380079B628063603760E4E70A2B81
:10369000E2D1204606A931F8082B628020F8043BCD
:1036A0001022FFF772F80C9B237518233360D3E7C1
:1036B000B1F58D7F7FB505460C461E460FD103A997
:1036C0001046FFF797FE002809DB089B039A00933A
:1036D00021463346284604F03BFD04B070BD00F09F
:1036E00003FF6FF0290303604FF0FF30F5E738B5B3
:1036F00005461046FFF7A1FE10F12B0F044605D03A
:1037000002462846BDE8384004F04CBC00F0ECFE10
:1037100004604FF0FF3038BD10B50B4609888AB001
:10372000022904460DD110225C885B6802918DF855
:103730000420ADF80C40049301A904F0F7FC0AB092
:1037400010BD0A2907D101A91846FFF7AAFE2422B5
:1037500001A92046F1E700F0C7FE6FF022030360E5
:103760004FF0FF30EBE7F0B5082785B0164604AA06
:103770000C4642F80C7D0DEB070104F0C1FC051E60
:1037800022DB039B022B09D13760BDF81020238078
:10379000059B62806360284605B0F0BD0A2B0ED100
:1037A0001822204604A9326031F8082B628020F8E4
:1037B000043B1022FEF7E9FF0A9B2375EBE700F0BC
:1037C00093FE6FF0220303604FF0FF35E3E72DE92E
:1037D000F04F002514468DB006460F46202229469C
:1037E00004A898460395FEF7FDFF4CB32022294616
:1037F00004A8FEF7F7FF6368E0680593A3680495E3
:103800000693FFF71AFE07902B3000F0948004AA6D
:103810003946304603AB04F0D3FC0027039EC8F8BA
:1038200000704FF0110940F2111A0546002850D0DF
:10383000D8F80000FFF728FE0023C8F800304AE05F
:103840002246E5E7202001F001F8044600286DD06B
:10385000B36872688360F368C0E90655022B05609F
:10386000426041D00EDC002B3CD0012B3FD06FF0EA
:103870002A03E36000236361204600F0E1FF6FF05C
:103880000605D5E7B3F5877F0AD040F201218B42C8
:1038900004D0B3F5827FEAD14FF48173E36001E095
:1038A000C0F80CA0022A24D1082000F0CFFF6061EC
:1038B000002838D00823236173691A8942805A6826
:1038C000DB6802804360002F33D1C8F800402746F0
:1038D000F669002EB6D1039804F074FC28460DB0AA
:1038E000BDE8F08FC560DDE7C0F80C90DAE706238D
:1038F000D4E70A2AC0D1182000F0A8FF83466061EF
:1039000088B11823236173691A89019342805A6828
:1039100020F8042B10229918FEF737FF019B1B6A31
:103920008BF81430CFE7204600F08AFF6FF00905CE
:103930007EE7FC61CBE76FF00605CFE7B1F58D7F41
:103940007FB505460C461E460ED103A91046FFF76B
:1039500051FD002808DB089B21460093284633468A
:1039600004F012FC04B070BD00F0BEFD6FF029033E
:1039700003604FF0FF30F5E710B50B4609888AB0B9
:10398000022904460DD110225C885B6802918DF8F3
:103990000420ADF80C40049301A904F08FFB0AB099
:1039A00010BD0A2907D101A91846FFF77AFD242284
:1039B00001A92046F1E700F097FD6FF022030360B4
:1039C0004FF0FF30EBE743689B6A03B1184770473D
:1039D00038B5436804465B6C03B1984763685B6B1A
:1039E000002B34D020469847002830D063689B696C
:1039F00023B14FF480522049204698471E4B1F4A5E
:103A00001B7811687F2B1E4801D0082B16D1002986
:103A10000ADD00251B4C013911606554222B02BFC1
:103A2000017881F001010170017881B916490978A6
:103A300003290CD8DFE801F0070C0F184C1C1460A8
:103A4000104C6354EAE713B90122104B1A7038BDC9
:103A50000D2BFCD1F8E711680A4A0A4412F8022C2F
:103A6000002AF4D00A2BF4E71168064A0A4412F837
:103A7000022C0D2AEBD1F5E7301002203430022061
:103A8000383002203000022039300220302002205D
:103A9000032910B532D81B4B197048B101282DD11C
:103AA000194800F0FBFC194C206018B9162010BD15
:103AB0001748F6E743689B68ABB92068FFF783FFB8
:103AC000226853689BB9134B40F201221B68002106
:103AD0001B6866209847104B1860431C0CBF6FF0A2
:103AE0000D000020E3E798470028DFD1E5E79B6C55
:103AF000002BE8D0094910469847E4E76FF015001D
:103B0000D5E700BF39300220A81005003C30022064
:103B1000C30B0500304702203C6F0220D13904005E
:103B20002DE9F0411A4D1B4E2A781B4FC2B11B4C98
:103B300020684368DB6A03B1984700232B70184D57
:103B40002A68B2F5805F06DC2AB139683068D1F89E
:103B50002C801449C047002320682B60FFF733FFF7
:103B60003B684FF480525C6A0F4940233068A0479D
:103B7000051E04DD0024094E0B4FAC4201D1BDE807
:103B8000F0813068395D436801345B689847F4E739
:103B9000302002203C6F0220304702203C300220BF
:103BA000343002203000022031200220074B03EB8A
:103BB0008000D0F8003223F44033C0F80032D0F84F
:103BC000003243EA0141C0F80012704700258440EA
:103BD000F8B5036801F01F029B68494D1B790C463C
:103BE00042EA43120023D5F804138668C9B203F5EC
:103BF000A27055F82000C0F30420824265D121FA5A
:103C000003F0C00761D5990001F1804101F544310D
:103C1000D1F8100520F00100C1F81005012101FACA
:103C200003F3C5F8083310460021FFF7BFFFB06863
:103C3000E04010F0010047D0F068E04010F00100D3
:103C400042D07069E04010F001074AD0B369E34008
:103C5000DB073ED43369F169E34021FA04F403F051
:103C6000010304F00104A3420CBF0224012400213B
:103C700001F5A27355F8230010F003002BD18B003F
:103C800003F1804303F54433D3F81065120226F4A0
:103C9000473626F44076C3F81065D3F8106502F471
:103CA000F85242EA0444174A3443C3F8104542F834
:103CB0002100D3F8102542F00102C3F8102501239A
:103CC00003FA01F1C5F80413F8BD0133082B8ED1B6
:103CD000A9E70324CBE701310829C9D16FF012000D
:103CE000F2E7F169336910464B4023FA04F414F00B
:103CF000010F0CBF03210221FFF758FF3846E3E70D
:103D0000001003400011034010B504688068A468E7
:103D100001292468C06903D158406060002010BDAB
:103D200000334FF0010118BF0123D04000F0010023
:103D30009140834214BFA160E160EFE770B5046871
:103D40008068A468C069256801296E692C696D685E
:103D500080EA040084EA050404EA060480EA040018
:103D60001CBFD04000F001001860002070BD8368C7
:103D7000186872B108605A68196002B95960002069
:103D8000704710605868814208BF5A600DE00246D3
:103D900000680028F3D08842F9D10868002AF0D1E1
:103DA0005A681860914200D1586000230B60E6E722
:103DB00001292DE9F04118BFD4B2064612BF2546AD
:103DC0001F2500244FF001088768AC4202D900206B
:103DD000BDE8F081FB6808FA04F223EA0203FB6005
:103DE00021463046FFF7F4FE0028F1D10134E4B259
:103DF000EBE7000008B5094B1A786AB901213120B8
:103E000019700521FEF714FB3120FEF7EDFA4FF093
:103E10000042034BC3F80423002008BD40300220B9
:103E2000001003402DE9F74F8046856803F4704089
:103E3000B0F5804F1E4649D02CDCB0F5805F3DD0F8
:103E4000B0F5405F3ED060BB06F44077B7F5807FA9
:103E50003ED0A7F5007463426341012919BFD4B273
:103E6000A1464FF01F0900244FF0010B06F0010C92
:103E70004FEA4C0747EA0C0747EA0020DFF8C8A0E2
:103E800040EA830706F00203A14523D2002003B0D5
:103E9000BDE8F08FB0F5E04F16D005DCB0F5A04FCF
:103EA0000ED06FF01500F2E7B0F5404F04D0B0F53A
:103EB000504FF6D10720C7E70620C5E70120C3E72A
:103EC0000320C1E70420BFE70520BDE70220BBE7D0
:103ED0000323C2E7D8F800209268117904F01F028A
:103EE00042EA411280324AF82270A9680BFA04F2C1
:103EF000002B25D01143A9606969B0064CBF11435E
:103F000091436961A96970064CBF11439143A9614E
:103F1000296970074CBF114391432961E969300653
:103F20004CBF0A4321EA0202EA612146404601935E
:103F3000FFF74EFE0028AAD10134E4B2019BA3E7AB
:103F400021EA0201D7E700BF002584402DE9F843AC
:103F5000444D2E68012E59D137464FF00009424A90
:103F600093681268DC69D2F80880D3E902120A402B
:103F7000D3E90510014322EA0102D8F800101B69B9
:103F800009695C404C4022EA040472BB2A600023A9
:103F900001279E46354DDFF8D8C0D5F8042307FA2F
:103FA00003F111420FD003EB0C02920011680129BA
:103FB00009D103F5A27055F82000C2F800E0C0F363
:103FC000042081400C430133082BE6D104B3264F73
:103FD000BB681D68E5B1AB681C4204D06B68224623
:103FE0002946384698472D68F4E73A420AD098F8AF
:103FF000043009F01F00002140EA4310FFF7D6FD0E
:1040000022EA070209F101097F00BEE70024BEE7AA
:10401000012E0DD10025144B9C681B689F68D4E9C4
:1040200002321A40D4E905310B4322EA03020AB9ED
:10403000BDE8F883164212D0E169236997F804C0FD
:104040004B40EB4013F0010F05F01F000CBF0321A4
:10405000022140EA4C10FFF7A9FD22EA06020135D1
:104060007600E4E77C110340187002200010034042
:1040700040C4001001292DE9F04118BFD4B2064612
:1040800012BF25461F2500244FF001088768AC4267
:1040900002D90020BDE8F081FB6808FA04F213435E
:1040A000FB6021463046FFF793FD0028F2D1013432
:1040B000E4B2ECE783681A7D72B102689268126814
:1040C000D2F8201141B14FF48071C2F808130121D8
:1040D000D16000221A7570479A680AB1D8681047F3
:1040E0007047000070B54B79012B23D18B79032BDE
:1040F00020D1CC792CB1012C1CD103689B689B7911
:10410000C3B10A7912B1022A14D10E2247F612263F
:1041100003689B681D680B68B3426BD027D8B3F562
:10412000965F61D012D8B3F5167F4DD005D8B3F5A0
:10413000967F74D06FF0220052E0B3F5966F50D0A6
:10414000B3F5166FF6D14FF41D233FE0B3F5615F71
:104150004CD004D8B3F5165FECD1324B36E0B3F552
:10416000964F45D0B3F5E14FE4D12F4B2EE0B3F598
:10417000E13F48D012D84DF6C026B3423DD005D815
:10418000B3F5164FD6D14FF41D031FE0B3F5614FC1
:1041900036D0B3F5963FCDD1244B17E0B3F5E12FE0
:1041A00037D008D8B3F5613F30D0214EB342C1D1EA
:1041B0004FF080630AE0B3F5612F2DD01D4EB3425E
:1041C000B8D14FF0805301E04FF41C33C5F82435CB
:1041D0008368224303C9C5F86C2583E803000020E7
:1041E00070BD4FF49E23F1E7134BEFE7134BEDE760
:1041F000134BEBE74FF40003E8E74FF46503E5E703
:104200004FF46B03E2E74FF0EB73DFE74FF06C73B3
:10421000DCE74FF0E863D9E74FF07063D6E74FF47F
:10422000A033D3E70050270000C0750000903A018A
:1042300090D0030040420F0000B0130000F03A009D
:1042400000A04E000B46826892E8030083E803005A
:1042500000207047036882689B681B68D3F81001D0
:1042600038B1527D00200A700122C3F810011A6093
:1042700070474FF0FF30704782B002AA02F8011D6C
:10428000002103689B681B68C3F82011C3F844250C
:104290000122C3F848259A60D3F820110029FBD0E9
:1042A000DA6002B0704703689B681B68D3F824018A
:1042B00018B1D3F88004C3F8800470470368F0B5E0
:1042C0009E6800243568D5F82031ABB18768B08886
:1042D00023469042A8BF1046C5F8204183423A6960
:1042E00006DB0123C5F84425C5F84805AB60F0BDE1
:1042F000CC5CD4540133F1E71846F8E703689B68B7
:104300001A68D2F8103143B183680020C2F8100156
:1043100001205B7D0B7010607047184670474FF4AA
:10432000807103689B681A688368C2F804130022CE
:104330001A757047012283681A75704703689B6875
:104340001B68D3F8200118B1D3F80403C0F3002090
:10435000704703689B681B68D3F81001003018BFD2
:1043600001207047102203689B681B68C3F8042370
:104370007047102203689B681B68C3F808237047C6
:104380004FF4007203689B681B68C3F804237047EE
:104390004FF4007203689B681B68C3F808237047DA
:1043A000012070478368C3E90212704708B50368AB
:1043B00002469B681968D1F80433DB0505D4D1F8AF
:1043C000040310F0100006D108BDFFF7B7FF002866
:1043D000F5D00120F8E71046FFF7BBFF003018BF0B
:1043E0000120F1E770B50646002201210820FEF702
:1043F0001FF80820FDF7F8FF4FF000523368B5684A
:104400009B6803211C681A4B1D209A600022C3F888
:104410007412C3F87022C4F80C051C20C4F81405EB
:104420004FF000609860C3F86C12C3F868221B2339
:10443000C4F808351A232946C4F810353046FFF76A
:1044400051FE98B90823C4F8003505F11503C4F8E6
:104450001001C4F8343501232A69C4F838352360C3
:10446000C4F84425C4F84805A360E36070BD00BFEC
:104470000025844038B5084B53F82040013053F8EC
:1044800020502046854204F10C0400D838BD54F871
:104490000C3C5B689847F4E730110500104B70B591
:1044A00005461E460F4C9C4204D10E4CB44209D125
:1044B000002412E062681AB122681268AA420CD085
:1044C0000C34F0E763680BB90C34EFE72368284637
:1044D0001968FEF727F90028F6D1204670BD00BF05
:1044E00030700220A06F0220014B98685430704752
:1044F000604B0220FDF7CEBC08B50A4D4FF02002FC
:10450000EFF3118382F3118800F09AFC0121044635
:104510000228D8BF084600F049FD2C62FDF7B8FD1F
:10452000ECE700BF604B02200248034A0021121A48
:10453000FEF758B900000220B04C02200248034A9E
:104540000349121AFEF721B9306F0220D8700220F9
:10455000A039050008B50220FFF78CFF0748FDF7DA
:1045600061FA0320FFF786FF00F0DAFBFCF7A8FEF4
:10457000034A137B23F00103137308BD5811050090
:104580003031022080B586B0314B06AF83F3088806
:104590000024E0222F4B304D83F82220DC771C765C
:1045A0005C769C765A6A2D4E42F4E0225A62FDF700
:1045B00013FFFDF767FD2046FFF75CFF0120FFF7C3
:1045C00059FF00F005FB264B756205930123CDE9E9
:1045D0000144CDE903430094224B4FF48062224909
:1045E000284600F063FB6B7B344623F0040213F093
:1045F0001B0F6A7305D12B6A013302D1284600F0E4
:1046000021FA1A4B012205930F23CDE9033200232F
:10461000174ECDE9013300934FF4A072154B1649A4
:10462000304600F043FB737BE66023F004037373B2
:10463000124BA560C4E906330A4A114B114C83F3AF
:10464000098863B6002181F311881046204700BF16
:10465000306F022000ED00E030310220604B02207C
:104660004811050055450400F06102204D11050078
:1046700084300220F9440400F0650220784B0220C7
:10468000F0650220F512040070B500240A4B0B48B7
:10469000834201D3002070BD00211A699D685C61CE
:1046A000A94201D11C33F3E75E6901311660DE686F
:1046B0005A613244F4E700BF307002206870022073
:1046C00038B5074C074DAC4201D3002038BD04F18A
:1046D00014032046C4E90533FCF753FE1C34F2E70B
:1046E00068700220847002202DE9F04F1D1E85B0F5
:1046F00006460C46174657DD00F06CFC4FF4004CA4
:104700000021804629484FF4A0220023CCFB05015C
:10471000FBF718FD18EB0002254B9046F31A254ACB
:104720009B1002FB03FA06F1140B5FFA8AFA00945D
:1047300003AB02AA39463046FCF76EFE10F10B0FB0
:104740000BD1009403AB02AA39463046FCF764FE55
:1047500010F10B0F08BF6FF00B006379029A84F819
:1047600004A062F3030363716368039A62F31F3367
:104770006360B0B1ADB110F10C0F12D14FF0200356
:10478000EFF3118083F311882A46594600F002FAAC
:104790006B1CCCD000F01EFCB8EB0005C7D56FF049
:1047A0000A0005B0BDE8F08F0022B5E7FFFF040066
:1047B00068700220B76DDBB670B504780268417886
:1047C000134EC4EBC404A400120B01F00F01301906
:1047D000FCF7F1FE4FF02003EFF3118583F311880E
:1047E00004F11400304400F0E3F968B1EFF30583FD
:1047F0000D2B09D81BB1074B5B681B0504D5284658
:10480000BDE8704000F0CCB885F3118870BD00BFE2
:104810006870022000ED00E013B504240A1904D2E8
:1048200000236946FFF760FF10B1002002B010BD01
:10483000224601A90098FDF7A8FF00980430F5E78B
:1048400010B10438FFF7B8BF7047000001460148B7
:10485000FFF7E2BF68700220D0E900231A60026807
:104860005360704708B5FDF7B3FB054B054A1B685D
:104870000021184410611846BDE8084000F096BBBE
:10488000E0310220604B02204FF02003EFF3118053
:1048900083F311887047000038B5104C234653F855
:1048A000285F9D4200D005B9E568A36878B973B167
:1048B0005A7BD2060BD11A6A013208D1DA897F2AD3
:1048C00005D9074A1268934201D0636238BDAB42F2
:1048D00001D0FFF7C7FF6562F8E700BF604B022019
:1048E00054110500F8B50D460746FFF7CDFF4FF40C
:1048F0000046002200210446094B0A481A61C6FB03
:1049000007014FF4A0220023FBF71CFC064B1860A4
:10491000064B1D60FFF7A6FF84F31188F8BD00BFAA
:10492000604B0220FFFF0400E0310220DC31022056
:1049300010B50146FFF7A8FF4B7B04465A060DD57C
:104940000846FFF789FF4B7B23F040034B73054B71
:104950009868431A58425841FFF79EFF84F3118824
:1049600010BD00BF604B022010B50146FFF78CFF61
:1049700004460846FFF770FF4B7B23F002034B739E
:1049800084F3118800238B6010BD10B50446FFF737
:10499000EBFF04F11800BDE8104000F041BA000040
:1049A000EFF305830D2B0BD81BB1074B5B681B0581
:1049B00006D5064B9A685B6A9A4201D0FDF7AEBBFA
:1049C00080F31188704700BF00ED00E0604B0220CB
:1049D00010B5FFF759FF0A4B04469A680120D37BB4
:1049E0000133D373FFF758FF84F311884FF020038E
:1049F000EFF3118083F31188BDE81040FFF7D0BFBB
:104A0000604B0220036810B5984213D093B191F91E
:104A10000E2093F90E40944206DD5A68C1E9003237
:104A20005A681160596010BD4468A34202D01B68E7
:104A3000002BEED1436808604B6043681960416009
:104A4000F1E7000038B50446FFF71EFF2146054692
:104A50000648FFF7D7FF637B002043F040036373F2
:104A6000FFF71AFF85F3118838BD00BF884B02207D
:104A7000427BD20604D1036A013301D1FFF7E2BFC2
:104A8000704738B550F8103C0446A0F1180513B132
:104A90002846FFF769FF14F80B3C284623F004036F
:104AA00004F80B3CBDE83840FFF7E2BF70B50446A0
:104AB000FFF7EAFE0B4D06462046FFF7CDFE2146E6
:104AC0002846FFF79FFF637B55F8200C43F0400317
:104AD0006373031B58425841FFF7DEFE86F31188CB
:104AE00070BD00BF884B0220114B10B51B68EBB1A5
:104AF00010498B68DA897F2A18D80F4A93F90E403B
:104B00001268944212DB0D4A126893420ED01A6A60
:104B100001320BD10A69824206DC1846FFF7C6FF54
:104B2000BDE81040FFF79EBE121A0A6110BD00BF1B
:104B3000E0310220604B0220DC31022054110500DC
:104B400070B504460D461646FFF7F2FE637B43F050
:104B50000203637325B1A56021462846FFF752FF83
:104B6000731C12D04FF40045002108484FF4A022D6
:104B7000C5FB06010023FBF7E5FA0549421C04F1D9
:104B80001800BDE8704000F089B970BDFFFF040057
:104B9000834A040010B50446044B9868FFF7D0FF21
:104BA0002046BDE81040FDF7B9BA00BF604B0220B7
:104BB00038B5054600202C68A54200D004B938BDA0
:104BC0002046FFF7E2FE2046FFF752FF0120F2E702
:104BD0000021044B084603F12802C3E90A22FFF72B
:104BE00081BE00BF604B0220014B9868704700BF38
:104BF000604B0220F8B505460F464FF02003EFF357
:104C0000118483F311884FF40046002108480023E3
:104C10004FF4A022C6FB0701FBF794FA0549421C9A
:104C200005F1180000F03AF984F31188F8BD00BFCF
:104C3000FFFF0400834A0400427BD20604D1036ACA
:104C4000013301D1FFF7FEBE70470000EFF305808E
:104C50000D2807D838B1044B586880F40060C0F3C1
:104C6000C02070470120704700ED00E0024B9B68B8
:104C7000187B00F001007047604B022010B54FF028
:104C80002003EFF3118483F31188437B590702D487
:104C900084F3118810BD23F004034373FFF7CCFFA6
:104CA0002046BDE81040FFF77BBE000030B587B05E
:104CB0000E9D044604950D9D03950C9D02950B9D3C
:104CC00001950A9D0095FDF7DDFB044B9B6813B928
:104CD000236607B030BD1B6EFAE700BF604B0220B1
:104CE000036D10B5044603B19847637BDA060AD119
:104CF000226A013207D12046FFF71AFE637B43F098
:104D00000803637310BD9B0702D52046FFF72CFEF6
:104D1000236A0133F2D004F1180000F081F8EDE7C6
:104D2000F0B5234F234D3E4687B0BD4205F1300418
:104D300014D3214B9A68D37B013BD3734FF02003EC
:104D4000EFF3118583F311881A4CB44223D385F312
:104D5000118807B0BDE8F040FFF73ABE54F8043CB4
:104D6000059354F8103C049354F8143C039354F8FE
:104D7000183C029354F81C3C019354F8203C0093D7
:104D800054E90A2354E90C01FFF790FF54F8303C32
:104D9000DD642546C9E7616A4B1C03D0206819B958
:104DA000FFF76CFF3034D0E7FFF724FFFAE700BFCE
:104DB0003070022030700220604B02200373002309
:104DC000C3734FF0FF334273817303627047000077
:104DD000034B1B680BB9FDF7FBB80020704700BF01
:104DE000E43102204FF02003EFF3118083F31188A8
:104DF00070470000036840B1084A5268904204D0EE
:104E00001BB19A6881680A449A604268136003681B
:104E10005A604FF0FF338360704700BF586F022025
:104E200010B50246FFF7DEFF04469068431C03D02E
:104E30001046FFF7DFFF002084F3118810BD00004B
:104E4000134B70B51B78002B14BF4FF0FF326FF07F
:104E50000042FFF7C7FF0F4B06461C689C420AD072
:104E60004CB1A568FFF7B4FF281A00280DDBA46831
:104E7000FFF7AEFF221A86F31188074B1B6913B1A7
:104E80009A42A8BF1A46104670BD0022F3E700BF41
:104E9000E8310220586F0220604B022070B5C160DB
:104EA00016460446FFF79EFF0546FFF791FF012EC9
:104EB000ACBF80190130164BA0601A689A4201D02D
:104EC0005E6832B95A68236062605A6814605C6038
:104ED0000BE09068A168884214DD411A9160516826
:104EE000C4E9002151680C6054601A689A4206D0E7
:104EF000944204D1FFF7A4FF0021FDF735F885F3B4
:104F0000118870BD091A9642A160DBD01268D8E7FB
:104F1000586F02202DE9F04B04464FF00008204D59
:104F2000204E214FFFF7E0FD2C60FFF75BFF346858
:104F30008146B4421CD094B1A1682B68994215DC1B
:104F40005B1A2B60D7E9002312EB010B43EBE17CEA
:104F5000C4F808802046C7E900BCFFF74BFF89F37F
:104F600011883CB1E36820469847DEE7C91AA16082
:104F70000024F4E7FFF736FF0B490646D1E900238A
:104F800028682C60171843EBE078C1E90078FFF738
:104F900057FF2146FCF7E8FF86F31188BDE8F08B48
:104FA000E4310220586F0220F031022070B50E4625
:104FB0000446FFF717FF0546FFF742FF431C01D0E9
:104FC000A04203DD31462046FCF7CEFF85F3118871
:104FD00070BD00002DE91848FFF704FF0446FCF7F8
:104FE000F7FF064BD3E9002312EB000B43F1000C53
:104FF0005846614684F31188BDE81888F0310220D4
:1050000070470000704700BF03F0DEBC08B5074BD7
:105010001A6842F000421A601B68DB0702D4FFF7EF
:10502000F1FF08BDFFF7F0FF08BD00BFF831022017
:1050300010B5084C23684BB90123236000F01AF81F
:105040002368002B01DB0223236010BD0F20FFF734
:10505000D9FF10BDF83102200FB408B52D20FEF79E
:10506000DAF8BDE808404FF0FF3004B0704700BFE9
:10507000FFF7CCBFF0B593B003F0D8FA20B92649BA
:1050800001A803F047FB18B1FFF7C0FF13B0F0BD54
:10509000FEF78CF902F0AEFB02460028F4D1202383
:1050A0004FF4804008214FF4405C1C4FCDE91022A2
:1050B0001B4E0393059307931A4D1B4C1B4A1C4B25
:1050C00009900D900DEB0100CDF82CC0CDE90E112B
:1050D00002970496069508940A920C9300F046FBFA
:1050E0000028D1D102F0F2F90028CDD103F0A2FFBF
:1050F0000028C9D101F026F90028C5D104F088F9AB
:105100000028C1D101F03CF80028BDD100F06EF8B4
:105110000028BBD0B8E700BF18120500000001202E
:10512000400001202000012060700120600001206B
:10513000603001200A2808B508D0662816D0022859
:1051400004D01620FEF767F8002008BDA2F5827291
:105150000A2A11D8012340F20341084803FA02F257
:105160000A4200F1280318BF184608BD40F2012387
:105170009A42E6D1024808BD004808BDB0110500BA
:105180008811050010B502F0AFFA044620B3836819
:1051900002690A2B0ED0662B06D0022B0AD01620ED
:1051A000FEF739F8002010BD40F201239A42F6D1F3
:1051B0000C4810BDA2F582720A2A0BD8012340F2D6
:1051C0000341094803FA02F20A4200F1280418BF19
:1051D000204610BD044810BD0920FEF71CF82046EB
:1051E00010BD00BF88110500B011050070B586B074
:1051F0001D4902A803F08EFA00BB0146044640F2A6
:105200000122662003F018FF184E00280546306082
:1052100010DB1748FDF77EFA23460246144928465C
:105220000194009403F0B8FE05461148FDF772FAA8
:10523000A84207D00524204606B070BD6924204648
:1052400006B070BD3068CDE9004403A923460A22A8
:1052500003F080FF0128EDDD03A802220549FDF7D8
:105260006EFA0028E7D0E5E7646F0220606F022045
:10527000301205003C120500014B1860704700BF5A
:1052800008420220F0B56C4B83B01B78002B00F075
:10529000AD806A4B1C68A26863689A422DD04BF6B9
:1052A000EF63ADF8003023786E468DF80430636804
:1052B00005219A422ABF27699F1ABF1A9A4294BFB2
:1052C0000025E568BFB288BF5B1B304688BF9DB232
:1052D000ADF80270FEF774F8BDF80210A068FEF792
:1052E0006FF8A36822691F44974208BFE368A7606C
:1052F00008BFA360002D40F08D80514B1C68A26850
:1053000063689A422CD04BF6EF63ADF800302378F7
:105310006E468DF80430636805219A422ABF2769DA
:105320009F1ABF1A9A4294BF0025E568BFB288BF92
:105330005B1B304688BF9DB2ADF80270FEF740F8A7
:10534000BDF80210A068FEF73BF8A36822691F446D
:10535000974208BFE368A76008BFA360002D48D14B
:10536000384B1C68A26863689A422BD04BF6EF63F7
:10537000ADF8003023786E468DF80430636805215F
:105380009A422ABF27699F1ABF1A9A4294BF0025E2
:10539000E568BFB288BF5B1B304688BF9DB2ADF8E1
:1053A0000270FEF70DF8BDF80210A068FEF708F8CD
:1053B000A36822691F44974208BFE368A76008BF3B
:1053C000A3600DB903B0F0BD30460521ADF8025021
:1053D000FDF7F6FFBDF80210E068FDF7F1FFBDF83C
:1053E0000220E3681344A36003B0F0BDFDF7AAFFF9
:1053F0004FE705213046ADF80250FDF7E1FFBDF85B
:105400000210E068FDF7DCFFBDF80220E3681344FA
:10541000A360A5E705213046ADF80250FDF7D0FFA7
:10542000BDF80210E068FDF7CBFFBDF80220E3688D
:105430001344A36061E700BF0C4202200442022033
:10544000FC4102200042022000222DE9F04FB04B27
:1054500083B01B6819695C69187C1A74587C5A748B
:10546000987C9A74D87CDA74187D1A75587D5A75B0
:10547000987D9A75D87DDA75B9B10139032914D8A8
:10548000DFE811F0D6000301040016000125032017
:1054900000226FF05F019F4C25701C7A1872587AB9
:1054A0005A72987A9A72DA7AD97203B0BDE8F08F9C
:1054B000042100226FF05F001C7A1972597A5A7227
:1054C00094499C7A9A72DC7AD8720A700B78002B15
:1054D00000F01781904B1C68A26863689A422DD037
:1054E0004BF6EF63ADF8003023786E468DF804304C
:1054F000636805219A422ABF27699F1ABF1A9A42F8
:1055000094BF0025E568BFB288BF5B1B304688BFEB
:105510009DB2ADF80270FDF753FFBDF80210A06810
:10552000FDF74EFFA36822691F44974208BFE36856
:10553000A76008BFA360002D40F0D280774B1C68A5
:10554000A26863689A422DD04BF6EF63ADF8003045
:1055500023786E468DF80430636805219A422ABF8D
:1055600027699F1ABF1A9A4294BF0025E568BFB207
:1055700088BF5B1B304688BF9DB2ADF80270FDF757
:105580001FFFBDF80210A068FDF71AFFA36822698B
:105590001F44974208BFE368A76008BFA360002DBF
:1055A00040F08D805E4B1C68A26863689A423FF4AD
:1055B0007CAF4BF6EF63ADF8003023786E468DF884
:1055C0000430636805219A422ABF27699F1ABF1ACF
:1055D0009A4294BF0025E568BFB288BF5B1B304686
:1055E00088BF9DB2ADF80270FDF7EAFEBDF802106B
:1055F000A068FDF7E5FEA36822691F44974208BF33
:10560000E368A76008BFA360002D3FF44EAF0521FB
:105610003046ADF80250FDF7D3FEBDF80210E06849
:10562000FDF7CEFEBDF80220E3681344A3603CE71B
:10563000384A117809B100211170A568002D39D0C0
:105640004FF0000CDFF8D4A0DFF8CCB03449E146CD
:1056500066466246D1F800E0DAF80080DBF80070B8
:1056600008E0632916D0612904BF074601260132EC
:10567000AA4213D0911C04EB810148680178622989
:10568000EFD180464FF00109F1E7FDF753FE03B07B
:10569000BDE8F08F86464FF0010CE8E7A6BBB9F1F4
:1056A000000F01D0CAF80080BCF1000F02D01C4AE4
:1056B000C2F800E0012000226FF05F01EDE6052155
:1056C0003046ADF80250FDF77BFEBDF80210E068F1
:1056D000FDF776FEBDF80220E3681344A36061E79E
:1056E00005213046ADF80250FDF76AFEBDF8021004
:1056F000E068FDF765FEBDF80220E3681344A3608F
:105700001CE7FDF71FFEE5E6CBF80070C7E700BF1A
:10571000084202200C42022004420220FC410220E6
:1057200000420220014B1878704700BF0C42022053
:10573000002070470B4BD3E90023134498420DD24D
:1057400082420BD810B5044600F0E0FC40B1064A96
:1057500084600260BDE8104000F020BC03F028B96E
:1057600010BD00BF104202200100020000282BD013
:1057700030B589B001AA6946044600F025FB03460E
:1057800040B1134A04F1280003C882E80300184618
:1057900009B030BDDDE90012204600F04BF80346A9
:1057A0000028EED10B4B0C490C480D4A03930D4DCC
:1057B0000D4B049105900D4902A80793069502929E
:1057C00002F0A2F90346DCE70E231846704700BF3B
:1057D000104202209D6004006D6104005D5D0400C4
:1057E0009D5F040035570400315704001842022021
:1057F00060B108B54368DBB2022B0ED003681B0C06
:10580000022B05D0042B0ED0002008BD00207047CD
:10581000806803F0CDF8002008BD0146BDE80840CF
:10582000034802F05BB8024802F0CEF9002008BD40
:1058300018420220002800F0FF802DE9F04F056893
:1058400095B0002D00F0EE808368002B00F0EA8018
:105850000769002F00F0E680846A002C00F0E280E7
:1058600044681B2C40F2E380C4680B2C40F2DF80BC
:10587000D0F814E0BEF1170F40F2D980002604469C
:105880006F48CDE90012DFF8D8A16E490680A06B01
:10589000DFF8D0C1DFF8D081DFF8D0B1DFF8D091E8
:1058A00072460E60CAF8000031463846CCF80060F7
:1058B000CBF80030C8F80060C9F80060FCF792FF30
:1058C000E36938463B60A3697B60FFF7D5FC0122A2
:1058D0004FF0040C5C4B5D49C3F8105609688020FA
:1058E00004915B49DDF810E0C3F8146609682E7076
:1058F00003916E70EE70AA700399A16ADBF800E064
:105900006960E16A019CA960EC60009C5149AF614B
:10591000C5F814E02C61C3F890250C68A1F59261DC
:105920000594059CC3F898C5D1F898444FF4806756
:105930000694069C1024C3F8A045D1F8A044464D17
:105940000794079C4024C3F8A845D1F8A8440894BC
:10595000089CC3F8AC05D1F8AC0409900998C3F8C9
:10596000006108680A900A98C3F8086188680B907B
:105970000B98C3F8106108690C900C98C3F8186173
:1059800088690D900D98C3F81C61C86901F5017113
:105990000E900E98D3F804031043C3F804030C6868
:1059A0002E480F940F9CD3F8044344EA0C04C3F828
:1059B00004430C681094109CD3F8044344F0100482
:1059C000C3F804430C681194119CD3F8044344F0C9
:1059D0004004C3F804430C681294129CD3F80443A7
:1059E00044F08004C3F80443DAF8003009685B012E
:1059F0001391DBB21399C8F8002080F82A33C0F85D
:105A0000847147600296C5F81066D5F81036029387
:105A1000029BD8F80030012BFBD0D9F8000015B05C
:105A2000BDE8F08F4CF20E0015B0BDE8F08F4CF2DF
:105A3000090015B0BDE8F08F4CF20E00704700BFB2
:105A40001C4202202C42022000A0024010A602406C
:105A500014A6024090A502400050004000E100E082
:105A600024420220304202202842022034420220F6
:105A7000204202202DE9F0474FF48065A94C86B002
:105A8000C4F88450BFF34F8FBFF36F8FA64EC4F896
:105A90008451D6F80C331F0669D4A34BD3F80C23DA
:105AA000D00775D4D3F80C2312F0400259D1D3F8A3
:105AB0000C13490741D59D4F3968012900F0C98071
:105AC0009B4BDFF894821F683A6872B300210C4642
:105AD00002E00134944226D207EBC405AB68002BE8
:105AE000F7D06E68F6B2012EF3D16868B8F80030CE
:105AF000B3EB104FEDD16A68013322F0FF0242F0A0
:105B000002026A60A868A8F80030FFF771FE31460B
:105B100028B96B6823F0FF0343F003036B603A6816
:105B200001349442D8D30029CFD100217E4A814B41
:105B3000C2F808111B680393039B7B4BD3F80C330B
:105B4000DB0643D44FF480617B4B764A1B685B01D4
:105B5000DBB282F82A33C2F88411516006B0BDE886
:105B6000F0870622714B1A6006B0BDE8F087FFF798
:105B70006BFCFFF7D7FD002866D1704BC6F81C01FF
:105B80001B680193019B684BD3F80C23D00789D580
:105B900000216B4AC3F80011126803240292029A92
:105BA000D3F814366149A3F50043013B022B8CBFA7
:105BB0000323644A0C6098BF52F82330624A1846A7
:105BC000136006B0BDE8F047FFF752BA5F4BDFF84D
:105BD00088811F683A6872B300210C4602E00134E4
:105BE000944226D207EBC405AB68002BF7D06E6851
:105BF000F6B2012EF3D16868B8F80030B3EB104F5D
:105C0000EDD16A68013322F0FF0242F002026A60BD
:105C1000A868A8F80030FFF7EBFD314628B96B689B
:105C200023F0FF0343F003036B603A6801349442AE
:105C3000D8D30029CFD100213B4A454BC2F81011DF
:105C40001B680493049B7DE7E02384F82A33656096
:105C50008AE73849C3F808213E4A0B681268059361
:105C600093683A4832490360D2F80480059AC1F833
:105C700000808BB1B8F1000F0ED01B68102B03D839
:105C8000D8F80010102909D94CF2060303222E4936
:105C900018460B603A6094E71023F7E7DFF8B890F6
:105CA00059B3002008F1040A044602E001348C4292
:105CB00021D2E50008EB05039A68002AF6D05E6859
:105CC000F6B2012EF2D1D3F804C0B9F80020B2EB3D
:105CD0001C4FEBD15968013221F0FF0141F0020164
:105CE00059609868A9F80020FFF782FD68B1304636
:105CF000D8F80010DAE70028D2D102200E4B4FF47A
:105D00008061084A1B68386021E75AF80530304640
:105D100023F0FF0343F003034AF80530D8F80010DE
:105D2000C4E700BF00E100E000A0024028420220DA
:105D30002C42022008A10240244202201CA1024061
:105D400000A1024040120500204202203042022001
:105D500010A10240344202201C42022030B4184BF1
:105D60001C6825686DB1A368834227D0002302E038
:105D70008968814219D00133DA00AB4204EB020199
:105D8000F6D1104B1C6825686DB1A368834215D00D
:105D9000002302E08968814207D00133DA009D4286
:105DA00004EB0201F6D130BC70470432A35823F053
:105DB000FF0343F00303A35030BC70470422F5E710
:105DC000304202202C420220002800F0B880002936
:105DD00000F0B580002A00F0B2802DE9F04F046A8F
:105DE00085B0002C00F0A680406A002800F0A28058
:105DF00042F687454FF0000A554EA84286F800A0AB
:105E000040F2A0800827DFF88091204616460D4614
:105E100044225146C9F80040FCF7E4FCD9F80020C0
:105E200004F14403DFF8648182F801A082F802A043
:105E300082F803A01770184644225146C8F8003073
:105E4000FCF7D0FCD8F8002004F18803DFF840B15B
:105E5000177082F801A082F802A082F803A0184609
:105E60004FF400725146CBF80030FCF7BBFC394BC5
:105E700004F5227CC3F800C0514660464FF400721E
:105E8000FCF7B0FC4FF4205C06214FF0010E4FF4FC
:105E900001304FF48832304B04F591645C602F4C34
:105EA000C3F808C09981A3F800E019461C612C4B87
:105EB000DFF8E0C020612B48636003F5C073A06089
:105EC000C4F800C02848E360626102F023FC0028A7
:105ED00032D14FF0020C2024D9F80010DBF800205A
:105EE00029601C4BD8F80010DFF8ACE01F4D316082
:105EF000CEF800201B681E4902F500722A601D4E74
:105F00001D4A1E4D0B6003F500731D493360288048
:105F1000C2F814C509681B4B03910399C2F81C759C
:105F200019683B4402910299C2F824451B68019309
:105F3000019B01E04CF2070005B0BDE8F08F4CF288
:105F40000E0070474CF2040005B0BDE8F08F00BFB2
:105F50004E4202206442022050420220744202203B
:105F60008000040000010400384202204442022064
:105F7000404202203C42022000A002404C4202204B
:105F800014A502401CA50240704202206842022073
:105F90006C420220400008004842022000285ED0E7
:105FA00070B4334B83B01A68324B82421ED81B68E0
:105FB00031498342096803D8304C2468844246D86A
:105FC00081420ED92E4B1B78002B4BD1831A2D49C1
:105FD0009E099B060A682C4C4FF003014FF0020506
:105FE00014D04CF2100003B070BC70471B6898428C
:105FF000F7D3224A12689042F3D20121C31A234AEE
:106000009E099B060D461268214CEAD14368DBB21B
:106010009D421FD1202002EBC60253681D4D03F4A0
:106020007F432E8843F0010343EA0643536000BFD9
:106030000138FCD10122184B43F8212022682B881B
:106040000192019A01332B8003B070BC70478142EA
:10605000D3D9B7E74CF2070003B070BC70474CF2DD
:106060000E0070474CF20F0003B070BC704700BFC9
:106070004842022040420220444202203C42022088
:106080004E420220704202200CA0024068420220D0
:1060900004A002404C42022000A00240184B1B7892
:1060A00063BBF0B4174A03F0FF001468164B256871
:1060B0001E68A5B10746C10063185A68D2B2032A08
:1060C00004D19F605A6822F0FF025A605A6812F0A9
:1060D000FF0F01D19B682BB10130A842EBD100200A
:1060E000F0BC704706EB801021448860436823F0C1
:1060F000FF0343F002034360F0BC70470020704789
:106100004E420220704202206C420220F0B4154A36
:10611000154B14681E682568ADB100200746C10004
:1061200063185A68D2B2032A04D19F605A6822F0D9
:10613000FF025A605A6812F0FF0F01D19B682BB121
:1061400001308542EBD10020F0BC704706EB801097
:1061500021448860436823F0FF0343F00103436058
:10616000F0BC70476842022064420220034B1B7857
:106170000BB902F013BC0020704700BF4E42022052
:10618000F0B53B4CC7B0266816BB012739482760DD
:10619000FCF7C0FA0546C0F5807331464FF48072B3
:1061A00006A80293FCF71EFB2A46324906A8FCF714
:1061B000ECFA06AA009702AB2A4420212E4802F0EE
:1061C0001FFC064638B100232320236047B0F0BDF2
:1061D0000E2047B0F0BD2220029B27601D4406AF71
:1061E00006AB78552B4440F20122022166205E70F6
:1061F00002F022FF071EE6DB2048FCF78BFA33464D
:1062000002461E49CDE90066384602F0C5FE023559
:1062100003A933460A22CDE90066384602F09AFF08
:10622000CDE9006606A92A463346384602F0B4FE98
:10623000A84203D0384602F047FFC4E7CDE9006624
:1062400033460A2203A9384602F084FF0128F1DD13
:1062500003A802220A49FCF772FA05460028E9D190
:1062600002233846236002F02FFF2846AEE700BF26
:106270008C4202204C120500904B02205C1205005B
:106280003C12050010B50446006803F06BF8A068E6
:1062900018B1BDE8104002F075BB10BD70B5002507
:1062A00082B002AC44F8045D06460D46204619460D
:1062B000144603F025F860B9019B082258729872C1
:1062C000D872184644EA0644DC601D611A7202B0B6
:1062D00070BD019B184602B070BD00BF70B50C4682
:1062E0000546114620461E4603F01EF800B970BD53
:1062F000206808B103F036F8204603F02BF82E6032
:10630000232070BD38B50023054601F081F904460D
:1063100030B10E2C10D80A4B53F82440204638BD1B
:10632000284601F0E1F90028F8D04468002CF5D0A7
:1063300000230E2C4360EED92D24204638BD00BF2B
:106340006C12050038B50023074D084C1946202271
:1063500007482B602360FCF745FA02F0CBFF0030C2
:1063600018BF0120404238BD9842022094420220CA
:10637000A042022000232DE9F04120F0080682B05F
:10638000022E009340F095804B1E012B0C4655D8F1
:106390000746002A4ED1012908BF0126484A214656
:1063A000684601F09FF8009B8046002B4FD00021EB
:1063B00002A840F8041DC3E902741E6102F0A0FFA8
:1063C000002841D147F201024FF0FF330821019D1F
:1063D00042EA0842EA606872A872E87229722B7475
:1063E0006B74AB74EB740A2F0CBF02220122AB68F2
:1063F000EE610C33AC616A61AB6047F20101284683
:10640000009E02F091FF38B3286808B102F0AAFF9D
:10641000284602F09FFF012323253360404601F008
:10642000B5F82846FCF7F7FE4FF0FF38404602B0BB
:10643000BDE8F08101290CD0022AAFD01620FCF76C
:10644000EAFE4FF0FF38F1E7019D002DCBD10C257E
:10645000E4E7012AA2D0F1E703464FF6FF720221DA
:10646000404601F0D5F80546A0B10E2D10D8154BC9
:1064700053F82550002DD1D1022CD7D1009B1A689A
:1064800042F400321A601A6842F400221A60CDE722
:106490002D25C3E7404601F027F90028ECD04368DA
:1064A000002BE9D00E2B4560F2D8064A52F8235053
:1064B000E0E72F20FCF7AFFE4FF0FF38B6E700BF54
:1064C000856204006C1205002DE9F04182B0064699
:1064D00001F00AF9002862D00446002102A82768CA
:1064E00040F8041DD4F8148002F00AFF002839D1C6
:1064F00047F209030822019D43EA0643EB60C5F811
:1065000010806872A872E8722A72236847F2090143
:106510001B0C1B0443F00E0323602368284623F45E
:1065200000332360236823F40023236002F0FCFE81
:1065300038BB03464FF6FF720F21304601F068F872
:106540000446A0B1174C54F8260020B102F002FF17
:10655000002344F82630304601F018F8002002B03D
:10656000BDE8F081019D0C20002DCED112E0304617
:1065700001F0BAF80028E5D04368002BE2D044606F
:10658000E0E7286808B102F0EDFE284602F0E2FEDE
:1065900023202760FCF73FFE4FF0FF30DFE70920A4
:1065A000F8E700BFA04202202DE9F043002483B0A9
:1065B000884617469946019405460A9E01F094F8CC
:1065C000002800F0C480C3680446012B5CD0236817
:1065D0009B0340F1B880394601A802F091FE0028E3
:1065E00040F0B3800C22019B1A7258729872D872D4
:1065F000F6B1A26871688A4209D1022A03F11C002F
:10660000317845D00A2A02D1242900F08480186804
:1066100010B102F0A7FE019B184602F09BFE162067
:106620004FF0FF36FCF7F7FD304603B0BDE8F083CE
:1066300047F206021646C3F81490616942EA054221
:10664000DA6019615F60B8F1000F04D03A46414644
:106650001868FCF79AF827682368314623F400335A
:106660002360236843F480132360019E304602F0C8
:106670005BFEC0B1306808B102F074FE304602F033
:1066800069FE27602320CBE7002EA0D01620C7E7A5
:106690001029BCD1042231895A83198306F10C01D7
:1066A000FCF773F83EE04FF40032034611462846EB
:1066B00000F0AEFF064608B30E2E15D8254B53F852
:1066C0002600236890B923F480132360224C54F8E9
:1066D00025309E69184602F03DFE0023304644F8FE
:1066E000253003B0BDE8F0832D20236843F4003348
:1066F0002360236823F48013236091E7284600F089
:10670000F3FFD8B14368CBB10E2B4660ECD8114AE9
:1067100052F82300D5E7102231895A831983B11822
:10672000FCF733F847F20702019B16469968588B2D
:1067300004310144C3F8149099607EE7236823F480
:1067400080132360C2E723206AE70C2068E7092052
:1067500066E700BF6C120500A04202202DE9F04F51
:1067600087B00191119E002A00F0C18083F00207DA
:106770009A468346904600F0B7FFC7F340070446A9
:10678000002800F0B7800368D90340F1AD801AF00B
:10679000100F27D000254FF023092368A06923F4A8
:1067A000803323600368DB689847421C49D08045EA
:1067B00025DDE568012D22D14FF4803200231146FA
:1067C000584600F025FF0746002862D00E2841D821
:1067D0004A4B53F82090B9F1000F3DD14FF000091A
:1067E0000127DAE74FF02309444D2368A06923F419
:1067F000803323600368DB689847013016D0236834
:1068000043F48033236006B13668019BA069CDE96B
:106810000238109B5246CDE90436036802A99B68F2
:106820009847431C53D007B0BDE8F08F236843F46A
:1068300080332360D7B94FF0FF30B9F1000FF2D0A9
:106840000EE0236843F480332360002FB4D1002D81
:10685000F1D0D4E74FF02D09236843F4803323604F
:106860004846FCF7D8FC4FF0FF30DCE74FF48032AD
:1068700000231146584600F0CBFE8146C0B10E28D9
:10688000E8D855F82090B9F1000FE5D14FF0000994
:10689000ABE7584600F028FF00289FD04368002B44
:1068A0009CD00E2B4760D5D8144A52F8239092E71B
:1068B000584600F019FF0028E8D04368002BE5D0C7
:1068C0000E2BC0F80490C5D855F82390DBE7A069DB
:1068D0000368DB689847013006D023684FF023092E
:1068E00043F480332360BBE74FF02309B8E74FF050
:1068F0001609B5E74FF00909B2E700BF6C120500B1
:106900002DE9F04182B0002940D0002A3ED0064651
:106910000F4600F0E9FE0546002800F08F8003686E
:106920009BB2022B04D003689BB2042B40F08680FC
:10693000002102A840F8041DD5F8148002F0E0FC04
:1069400060BB08213304019C43F4E04242F00202A0
:10695000E260C4F810806072A072E072217243F4A9
:10696000E04343F00203E360A3686A6904332261F1
:10697000A360AB687A68934208D1022B04F1180037
:106980003A7832D00A2B01D1242A0CD01620FCF7F9
:1069900042FC4FF0FF3002B0BDE8F081019C002CBA
:1069A0005DD03304DBE710223B89B918E282A38271
:1069B000FBF7EBFEA368E28A47F202011344A360EF
:1069C0002F682B6820461B0C1B0443F005032B602B
:1069D00002F0AAFCA0B1206808B102F0C3FC204676
:1069E00002F0B8FC2F602320D1E7102ACED1042278
:1069F0003B8907F10C01E282A382FBF7C6FED9E7CF
:106A000003464FF6FF720621304600F001FE0446B1
:106A1000B0B10E2C05D8134B53F8240020B12F60D1
:106A2000B5E72F602D20B2E72B68002043F4003338
:106A30002B602B6843F400232B60ACE70920A6E70A
:106A4000304600F051FE0028EED04368002BEBD01A
:106A50000E2B4460E5D8034A52F82300DEE70C20F1
:106A600095E700BF6C1205002DE9F04182B091B3AB
:106A70008AB307460E4600F037FE0546002800F0B0
:106A8000818003689BB2022B7CD1002102A840F8D0
:106A9000041DD5F8148002F033FC20BB47F2050337
:106AA0000822019C43EA0743E360C4F81080607247
:106AB000A072E0722272A3680433A360AB687268AC
:106AC000934208D1022B04F1180032783FD00A2BF0
:106AD00001D1242A0CD01620FCF79DFB4FF0FF308B
:106AE00002B0BDE8F081019C0C20002CE3D1F3E75B
:106AF00010223389B118E282A382FBF746FEA36815
:106B0000E28A314E1344A3602B6847F205013340FB
:106B100043F003032B602046D5F8008002F004FC0C
:106B200000BB03464FF6FF720421384600F070FDAB
:106B3000044690B30E2827D8244B53F8200050B3B6
:106B40002B681B0C1B0443F002032B60C4E7102AC4
:106B5000C1D10422338906F10C01E282A382FBF742
:106B600014FECCE7206808B102F0FCFB4FEA18489D
:106B700020464FEA084802F0EDFB48F002032B6084
:106B80002320A9E70920A7E72B682D201E4046F007
:106B900002062E60A0E70020A2E7384600F0A4FD20
:106BA0000028F8D04368002BF5D00E2B446003D8A2
:106BB000064A52F82300C2E72B682D20334043F0E9
:106BC00002032B6088E700BF0000FFFF6C12050086
:106BD0002DE9F04182B0064600F086FD002877D00E
:106BE000036805469BB2042B72D10021414A30460E
:106BF00000F0E0FC0146002873D102A840F8041D13
:106C00006F6902F07DFB002838D147F208030822A3
:106C1000019C43EA0643E36027616072A072E07260
:106C20002272A368344F0433A3602B6847F2080133
:106C30003B4043F007032B602046D5F8008002F06C
:106C400073FB00BB03464FF6FF720821304600F08D
:106C5000DFFC044690B30E2829D8284B53F82000B7
:106C600090B32B681B0C1B0443F004032B60FCF750
:106C7000D2FA4FF0FF3002B0BDE8F081019C0C2049
:106C8000002CCED10EE0206808B102F06BFB20464C
:106C900002F060FB23204FEA18484FEA084848F00A
:106CA00004032B60FCF7B7FA4FF0FF30E3E72B68E3
:106CB0002D201F4047F004072F60F3E7304600F017
:106CC00013FD08B143682BB9002002B0BDE8F08184
:106CD0000920E7E70E2B446005D8084A52F8230044
:106CE000BEE72320DEE72B682D203B4043F0040362
:106CF0002B60D7E7856204000000FFFF6C120500DF
:106D00002DE9F04F4FF0000B85B08846CDE9012BFF
:106D1000064600F0E9FC0446002800F0F980076808
:106D2000BFB2082F40F0E780056815F4803500F009
:106D3000E080794AC16802A800F0D4FB029A0546B7
:106D40008146002A00F0DA80236904A81361A36851
:106D500040F804BD9360E3685946D360D4F814B09A
:106D600002F0CEFA002838D147F20C03DDF80CA06F
:106D700043EA0643CAF80C30CAF810B08AF8087023
:106D80008AF809008AF80A008AF80B002368DFF8FD
:106D900094B147F20C0103EA0B0343F009032360AB
:106DA0005046276802F0C0FAF0B903464FF6FF726A
:106DB0000A21304600F02CFC0746002838D00E2867
:106DC0002ED8564B53F82070002F38D023681B0C58
:106DD0001B0443F00803236014E0DDF80CA00C272B
:106DE000BAF1000FD2D10DE0DAF8000008B102F0DC
:106DF000B9FA3F0C3F0447F00807504602F0AAFAE0
:106E000027602327029B13B1284600F0BFFB4FF0F9
:106E1000FF393846FCF7FFF9484605B0BDE8F08F6A
:106E200023682D2703EA0B0B4BF008032360E9E7E7
:106E3000304600F059FC10B14368002B47D1384D63
:106E4000029955F826309B694B61B8F1000F08D0C4
:106E50008B680A2B24D0022B03D1019A1268102AC6
:106E60003CD00A682F48024042F006020A60029AAB
:106E7000116841F400311160116841F40021116082
:106E80002368034043F00803236055F8260002F00E
:106E900061FA0023484645F8263005B0BDE8F08F7A
:106EA000019A1268242ADCD188F800201022C8F840
:106EB000043055F8263008F110009B8BA8F80830F4
:106EC00055F826102031FBF760FC0299C9E70E2B1C
:106ED000476015D8114A52F8237075E788F80020EA
:106EE000C8F8043055F8263008F10C009B8B0422BA
:106EF000E4E7092786E75D46092783E70C2786E74D
:106F000023682D2703EA0B0343F00803236079E786
:106F10000546092776E700BF856204006C1205006C
:106F2000A04202200000FFFF012901D02A20704763
:106F300038B51D46144600F0D7FB034668B1142C43
:106F400007D165B1049A042A05D12A680020DA61C4
:106F500038BD2A2038BD162038BD092038BD0E2086
:106F600038BD00BF4FF0FF30704700BF2DE9F04F34
:106F7000474F83B0396800296CD1DFF818A1DFF8DA
:106F80001891064698461546CAF80010C9F8001030
:106F900090B1FBF7BFFB8346002302A840F8043DF5
:106FA000594602F0ADF948B1019CDCB90C20002330
:106FB0003B6003B0BDE8F08F8346EDE74FF0FF3351
:106FC0004FF00D0C70210822019C84F80CC06072F7
:106FD000A072E07261732272A373E373237463740B
:106FE000A374E374002D39D06B6823F00802022AE1
:106FF0003BD10A2B14BF01230223A361EB68236258
:10700000AB68E3612B686361A3681033A3602EB1A2
:10701000206818B15A463146FBF7B7FB012347F207
:107020000D0120463B6002F07FF908B12320BEE746
:1070300000212046FCF7EDF83B68012BF8D0D9F889
:1070400000000028B3D1DAF80030C8F8003003B0EF
:10705000BDE8F08F732003B0BDE8F08F2946102201
:1070600004F11400FBF7BEFBCEE72F20FCF7D3F8AA
:10707000A3681033A36016B94FF0FF3097E720687C
:107080000028F9D05A463146FBF77FFBF4E700BFF2
:1070900094420220984202209042022038B50B4CC4
:1070A0002368022B00D038BD30B10546406901F09D
:1070B00069FC284601F066FC0023054A0549136077
:1070C00023600868BDE8384002F04CB994420220C1
:1070D000904202209C4202202DE9F04F01F410431F
:1070E000B3F5104F064687B00D46C06858D0040C63
:1070F000204600F0F9FA0746002843D02A463146D8
:1071000002F0CAFC002839D048F207039D4263D937
:1071100048F20C039D4200F0288176D848F208031B
:107120009D4200F0938048F209039D4267D13B687D
:107130009BB20E2B22D17069002840F056813B682B
:107140001B0C1B0443F00F033B6018E0738A002BF9
:1071500000F09480242001F0F7FB0446002800F0A2
:107160008881728A102A00F06881042A00F09681D2
:10717000306802F0F7F8204601F004FC002007B068
:10718000BDE8F08F48F20D039D4234680CD0002C0E
:10719000F4D0204602F0E6F8002007B0BDE8F08FFA
:1071A00000F05AFA0446A3E7DFF81CB3DBF800202E
:1071B000012AECD17269002A74D00E2A88BF2D21D1
:1071C0004FF0020098BFBB49CBF8000098BF51F8C0
:1071D0002210B94A1160DAE748F206039D4280F0B6
:1071E000D78048F202039D4200F0ED8048F205038B
:1071F0009D421CD048F201039D4200F0D9803068C6
:107200000028BBD002F0AEF8B8E749F201039D4276
:107210002BD049F202039D42F1D13B689BB2082B6F
:10722000ACD13B68002043F480333B60A7E73B6868
:107230009BB2032BA2D17069002840F0D6803B6836
:107240001B0C1B0443F004033B6098E73B689BB2B4
:10725000072B93D17069002840F0C7803B681B0C56
:107260001B0443F008033B6089E73C6814F40024E6
:1072700000F0DE80B368042B3FF668AF002331686E
:107280007268CDE90433CDE90212B86902A9036836
:107290005B689847013000F0EC803B6843F4803332
:1072A0003B606BE7854A1460B5696B011846019332
:1072B00001F04AFB8246002800F0DF80EE007019E2
:1072C000800001F041FB002800F0E480002D44D054
:1072D0000425103600EB060900F110080AF120071A
:1072E0006259631947F8202C5A681435022A14BFD2
:1072F00002220A2247F81C2C9968A8F1100247F8CC
:10730000181CD868611947F8140C188A47F8100C33
:1073100004285E8A47F80C2C6AD00A2348F80C3CF3
:107320004FF0240308F8103C57F8102C4046FBF7A8
:107330002CFA57F8103C08F108081D446319C145A0
:1073400047F8047C47F8083C354407F12007C7D1CB
:107350000021019B534443F8041C0221584ACBF8F6
:107360000010C2F800A0002009E73B689BB2092B7F
:107370007FF404AF7369002B57D1524B012043F8BF
:1073800024603B681B0C1B0443F00A033B60F6E6D9
:107390003B68DB027FF5F2AE7369002B45D1494BA8
:1073A000012043F824603B6843F400333B60E6E689
:1073B0003B68012B7FF4E2AE7069B0B902233B60F9
:1073C000B3697B61DBE63B689BB2052B7FF4D6AEED
:1073D000706950B93B681B0C1B0443F006033B600B
:1073E0003B6843F400333B60C9E678600020C6E6A2
:1073F0001023022208F8103C48F80C2C57F8102CE7
:10740000A8F10400FBF7C1F957F8103C08F108088F
:107410001D446319C84547F8047C47F8083C3544C7
:1074200007F120077FF45CAF92E77B600020A6E6BF
:10743000306801F097FF2046A1E60A232425436027
:107440000570338A06F1140103811030FBF79DF9B2
:1074500073683268CDE90445CDE90223B86902A911
:1074600003685B68984701307FF417AF204601F04E
:1074700089FA306801F076FF80E601F083FA0C208B
:1074800002210D4A346810600D4ACBF80010C2F892
:1074900000A07CE60C21084A11605EE7022310255B
:1074A00043600570338A06F1140103810C30FBF749
:1074B0006CF9CDE76C120500904202209C4202203C
:1074C00098420220A04202209442022008B54FF4C4
:1074D000807200210248FBF785F9002008BD00BF3B
:1074E000B04B0220F8B5284B06461D680846E5B1AA
:1074F0001C6A002C3BD01C6C002C3AD01C6E002C5B
:1075000039D0D3F8801079B1D3F8A010A9B3D3F84B
:10751000C010A1B3D3F8E01099B34FF0FF350C20A1
:10752000FBF779FE2846F8BD04254FF0010C4FF01B
:10753000FF376C0143F804C01C44114667612246C2
:1075400001F0EAFB0346A06158B11B681B6898472D
:1075500010B934602846F8BDA06901F0FBFB002398
:10756000A361204620220021FBF73CF9D5E7012545
:10757000DBE70225D9E70325D7E70525D5E706256B
:10758000D3E70725D1E700BFB04B0220072800D979
:10759000704710B5064C04EB4014A06908B101F027
:1075A000D9FB2046BDE8104020220021FBF71AB984
:1075B000B04B022007282DE9F04118D8134D4401A3
:1075C0002B592F199BB1084611463A46D7F8188017
:1075D00001F0A2FBB861B8B103681B689847064682
:1075E00048B9404601F0B6FB3046BDE8F0810526BB
:1075F0003046BDE8F081B86901F0ACFB2819C0F84D
:1076000018803046BDE8F0810426F7E7B04B022031
:107610002DE9F0410F4C40012558044415408D429E
:1076200011D0606878B998460F461646254606E0A0
:107630006B6843B941462046FBF7EBFD30B928683B
:107640003040B842F4D10020BDE8F0813C20BDE8D4
:10765000F08100BFB04B0220224B1A6812B15A6968
:10766000824231D01A6A12B15A6B82422ED01A6C01
:1076700012B15A6D82422BD01A6E12B15A6F8242E9
:1076800028D0D3F880201AB1D3F89420824223D096
:10769000D3F8A0201AB1D3F8B42082421ED0D3F878
:1076A000C0201AB1D3F8D420824219D0D3F8E020F8
:1076B0003AB1D3F8F430834214BF4FF0FF300720C3
:1076C00070474FF0FF30704700207047012070472F
:1076D0000220704703207047042070470520704740
:1076E00006207047B04B0220072807D8044B400102
:1076F0001A581844002A08BF00207047002070471D
:10770000B04B022019B1072802D908230B6070473B
:10771000044B40011A58002AF7D01B58C3F3024308
:107720000B607047B04B02202DE9F0412E4CFBF767
:10773000F9FD03272D4D2E4E04F1800802E0083498
:1077400044453BD014F8043C022BF8D1206829882A
:10775000026892B2914233D0298A914232D0298C68
:1077600091421CD02B8E93422ED0B5F840309342DC
:107770002FD0B5F8503093422DD0B5F860309342F9
:107780002BD0B5F87030934229D0B5F880309342B1
:1077900027D0B5F89030934208BF0923CFD105EB2D
:1077A00003135A68D968904780B90122206804F809
:1077B000042CF368083498474445C3D1BDE8F081F0
:1077C0000023ECE70123EAE70323E8E704F8047C5D
:1077D000B5E70423E3E70523E1E70623DFE7072313
:1077E000DDE70823DBE700BFFC430220C0420220A4
:1077F0006043022008B5A02200210248FAF7F2FFF8
:10780000002008BDC04202200388002B45D04268FA
:107810000146002A50D0304A108883423DD02DE9DD
:10782000F047148AA34235D0158CAB4232D0168E65
:10783000B3422FD0B2F84070BB422BD0B2F850C048
:10784000634527D0B2F860E0734523D0B2F870806A
:1078500043451FD0B2F880904B451BD0B2F890A0A2
:10786000534517D0E0B15CB365B36EB377B3BCF1E9
:10787000000F2DD0BEF1000F20D0B8F1000F29D09D
:10788000B9F1000F0BD00920BAF1000F08D0042085
:10789000BDE8F0870720BDE8F08707207047082083
:1078A000000113524B68024453608B6800209360C0
:1078B000CB68D360BDE8F0870E2070470620EFE765
:1078C0000120EDE70220EBE70320E9E70420E7E7EA
:1078D0000520E5E70720E3E7C042022038B5864AE5
:1078E0000B6810889BB2984229D0108A984226D003
:1078F000108C984223D0108E984220D0B2F84000CD
:1079000098421CD0B2F85000984218D0B2F86000EB
:10791000984214D0B2F87000984210D0B2F88000AB
:1079200098420CD0B2F890209A4208D0886800287B
:1079300000F0A980714B1B699847002038BD88680A
:10794000002800F091806E4A1568002D3BD09468A5
:10795000002C00F09A801469002C00F09880946943
:10796000002C00F09680146A002C00F09480946A39
:10797000002C00F08680146B002C00F09080946B3B
:10798000002C00F09080146C002C00F09080946C1F
:10799000002C00F09080146D002C00F09280946D0B
:1079A000002C00F09080146E002C00F09280946EF9
:1079B000002C00F09080146F002C00F08E80946FEB
:1079C000002CB7D10F2502EBC50442F83500A38087
:1079D0004C4B1A78012A60D01A7A012A47D01A7CB7
:1079E000012A5ED01A7E012A5FD093F82020012A56
:1079F0005FD093F82820012A5FD093F83020012A25
:107A00005DD093F83820012A5FD093F84020012AF6
:107A10005DD093F84820012A61D093F85020012AC4
:107A20005FD093F85820012A5DD093F86020012A96
:107A30005BD093F86820012A59D093F87020012A6E
:107A400057D093F87820012A10D0102D1BD0002495
:107A50002B4B2A4A03EBC50043F8354084808868E5
:107A600013699847204638BD1025B1E70F2202243C
:107A700003EBC200416003F83240FBF74BFC0120EE
:107A800038BD05259FE7002038BD01259BE702256D
:107A900099E7032597E7042595E70022E7E7062500
:107AA00091E70222E3E707258DE70322DFE70825B8
:107AB00089E70422DBE7092585E70522D7E70622C7
:107AC000D5E70A257FE70B257DE70722CFE70822C8
:107AD000CDE70C2577E70D2575E70E2573E709221D
:107AE000C5E70A22C3E70B22C1E70C22BFE70D223C
:107AF000BDE70E22BBE700BFC04202206043022068
:107B000078430220F8430220F0B4002952D0002824
:107B100050D08368002B4DD00369002B4AD04368B6
:107B2000002B47D0C368002B44D00368002B41D002
:107B30004369002B3ED00126002504460F461F4A0C
:107B40001F4BDFF880C01674167682F8206082F82A
:107B5000286082F8306082F8386082F8406082F8ED
:107B6000486082F8506082F8586082F8606082F85D
:107B7000686082F8706082F878601D619D611D62A6
:107B80009D621D639D631D649D641D659D651D66ED
:107B90009D661D679D67167016721D609D600FCCF7
:107BA000ACE80F0094E803008CE803003E60284630
:107BB000F0BC70470E252846F0BC7047F843022001
:107BC000784302206043022000283AD02DE9F04794
:107BD00080461D4C04F1A005A368103403B19847FA
:107BE000AC42F9D14FF001090026184C184DDFF8CE
:107BF00064A004F1800714F8043C012B05D0DAF8E6
:107C00000C302068984704F8049C55F8040C08349C
:107C100028B1DAF8103098472E8045F8046CBC4241
:107C200005F10805E7D1D8F800001822013800EB6B
:107C300040000AEBC0000021FAF7D4FD0020BDE8A7
:107C4000F0870E20704700BFC0420220FC43022094
:107C50007C4302206043022068B171B1094A536835
:107C60006BB14B68088023F0FF0343F002031268F6
:107C70004B6008461047072070470E2070470820C9
:107C8000704700BF604302205AB3E8B100232DE9DA
:107C9000F041DFF858801360D8F804301BB3164663
:107CA0000C46054698470746C8B1C46074B12046E3
:107CB000D8F808309847B86060B93846D8F80C3022
:107CC00098470420BDE8F081072070470472447291
:107CD0008472C4723D8037600020BDE8F0810420CA
:107CE000F0E70E2070470820ECE700BF6043022059
:107CF00000283DD0002900F0918038B5524C6368CF
:107D0000002B37D0514A08465368994234D0D36883
:107D100098423DD0536998423FD0D369984241D0B0
:107D2000536A984244D0D36A984247D0536B9842E2
:107D30004AD0D36B98424DD0536C984250D0D36CFC
:107D4000984253D0536D984256D0D36D984259D033
:107D5000536E98425CD0D36E984261D0536F984274
:107D600064D0D36F834267D0E3689847002038BD62
:107D700007207047082038BD11780329C7D100219A
:107D800001251846E46802F83150A047002038BDAC
:107D9000117A0329BED10121F2E7117C0329BCD15C
:107DA0000221EDE7117E0329EAD0536A9842BAD145
:107DB00092F820100329B6D10421E1E792F82810A7
:107DC0000329B3D10521DBE792F830100329B0D1A4
:107DD0000621D5E792F838100329ADD10721CFE766
:107DE00092F840100329AAD10821C9E792F8481057
:107DF0000329A7D10921C3E792F850100329A4D180
:107E00000A21BDE792F858100329A1D10B21B7E749
:107E100092F8601003299ED10C21B1E70E20704723
:107E200092F86810032999D10D21A9E792F87010F2
:107E3000032996D10E21A3E792F87830032B93D132
:107E400003460F219CE700BF60430220F843022055
:107E500000283DD0002900F08B8038B54F4A536888
:107E6000002B37D04E4B1C68A14235D09C68A142F4
:107E70003DD01C69A1423FD09C69A14241D01C6AFF
:107E8000A14243D09C6AA14245D01C6BA14247D07D
:107E90009C6BA14249D01C6CA1424BD09C6CA1426E
:107EA0004ED01C6DA14251D09C6DA14254D01C6E8D
:107EB000A14257D09C6EA1425CD01C6FA1425FD002
:107EC0009C6F8C4262D0084613699847002038BDE9
:107ED00007207047082038BD9C888442C6D1002402
:107EE000002003EBC40543F83400A880EBE79C892D
:107EF0008442BED10124F3E79C8A8442BCD102248F
:107F0000EEE79C8B8442BAD10324E9E79C8C84423F
:107F1000B8D10424E4E79C8D8442B6D10524DFE780
:107F20009C8E8442B4D10624DAE79C8F8442B2D17D
:107F30000724D5E7B3F844408442AFD10824CFE703
:107F4000B3F84C408442ACD10924C9E7B3F854409B
:107F50008442A9D10A24C3E7B3F85C408442A6D185
:107F60000B24BDE7B3F864408442A3D10C24B7E7E7
:107F70000E207047B3F86C4084429ED10D24AFE7C9
:107F8000B3F8744084429BD10E24A9E7B3F87C4037
:107F9000844208BF0F2496D1A2E700BF60430220AD
:107FA0007843022070B504460D461646FDF7C2F828
:107FB00030B10368324629462046BDE87040184774
:107FC0004FF0FF3070BD00BF10B50446FDF7DAF882
:107FD00020B143682046BDE8104018474FF0FF30FD
:107FE00010BD00BF2DE9F0470D46DDE908891646B2
:107FF0001F460446FDF7C6F858B1CDE90889D0F808
:1080000008E03B46324629462046F446BDE8F047A4
:1080100060474FF0FF30BDE8F08700BF2DE9F04129
:1080200082B00E46174698460546FDF7ABF860B19C
:1080300004460020CDE9000043463A463146284632
:10804000A468A04702B0BDE8F0814FF0FF30F9E727
:108050002DE9F0470D46DDE9088916461F4604461E
:10806000FDF790F858B1CDE90889D0F80CE03B460F
:10807000324629462046F446BDE8F04760474FF0B7
:10808000FF30BDE8F08700BF2DE9F04182B00E4619
:10809000174698460546FDF775F860B1044600207E
:1080A000CDE9000043463A4631462846E468A047F9
:1080B00002B0BDE8F0814FF0FF30F9E770B50D4632
:1080C00016460446FDF75EF830B14369324629464C
:1080D0002046BDE8704018474FF0FF3070BD00BF2C
:1080E00070B50D460446FDF74DF828B18369294661
:1080F0002046BDE8704018474FF0FF3070BD00BF0C
:108100002DE9F0410D4616460446FDF73BF840B117
:10811000C769324629462046BC46BDE8F0410023E7
:1081200060474FF0FF30BDE8F08100BF70B50D46ED
:1081300016460446FDF726F830B103693246294653
:108140002046BDE8704018474FF0FF3070BD00BFBB
:108150002DE9F041DDF818800D4616461F4604460D
:10816000FDF710F858B1CDF81880D0F820E03B4664
:10817000324629462046F446BDE8F04160474FF0BC
:10818000FF30BDE8F08100BF2DE9F041DDF8188037
:108190000D4616461F460446FCF7F4FF58B1CDF8CD
:1081A0001880D0F824E03B46324629462046F44663
:1081B000BDE8F04160474FF0FF30BDE8F08100BFFF
:1081C00001F09CBC01F09CBC01F09CBC2DE9F04F7F
:1081D000DFF8CCC083B000900CF13C0BDCF8083029
:1081E0002BB1DCF80020009C1078A04206D00CF1E6
:1081F0000C0CE345F2D103B0BDE8F08FDCF804A02D
:1082000003EB0A08C245F2D25368CDF804C0D64643
:108210009C46D2F810909789AEEB0A00DFB3B9F80C
:10822000022090421CD36546002409F1040303E0B8
:108230005A880433824215D833F8046C0134A742BB
:1082400002FB0655A0EB02001E46F1D10020814240
:108250000DD00EF1010EF045DED1DDF804C0C6E709
:1082600065464E46338800FB03508142F1D1BEF58E
:10827000007FDDF804C0BAD00123084A4FEA5E113E
:1082800052F821000EF01F0E03FA0EFE4EEA000017
:1082900042F82100AFE73846D9E700BF7844022012
:1082A000BC440220002850D06D4BD3F88820904267
:1082B0004BD82DE9F04FD3F88CB083B0BBF1000F51
:1082C00054D00BF1FF32914600264FF01208654F53
:1082D00001920BF1110E06EB090253F838400132FE
:1082E000520804EB440C02F1120153F8315057F8D4
:1082F0002CA053F83E4003EBC80CDCF804C005EB9F
:10830000450504EB4404DAF810A057F8255057F857
:1083100024403AF82CA003EBC10103EBCE0C4968D2
:108320002D692469DCF804C0504535F8215034F833
:108330002C1015D9884211D2A84208D9561CB14533
:10834000C0F0878002F11308C5E70020704702F1F2
:10835000FF394E457DD802F1110EBCE709F1010647
:10836000B34507D0102E01D0B34508D8002003B084
:10837000BDE8F08F019A102A18BF1646F6D0DFF834
:10838000E8C003EBC608D8E9242402EB420257F800
:10839000223007EB8202D2F804E01D69002C56D08F
:1083A0002A467046A40005EB040951880432914521
:1083B0000844FAD12919B1F802A08244824518D99B
:1083C00041095CF8212000F01F0422FA04F919F099
:1083D000010F07D013E05CF8212022FA04F919F00C
:1083E000010F0CD1013082454FEA501100F01F04FB
:1083F000F1D101365E4508F10808C4D3B6E701267D
:1084000006FA04F49E8922EA0402A0EB0E004CF85E
:1084100021205C68002EA9D06A88824211D80021F0
:108420002B1D03E05A88043382420AD833F8045CD7
:1084300001318E4202FB0544A0EB02001D46F1D142
:1084400094E72B8800FB034003B0BDE8F08F704633
:10845000B0E7BBF1100F08BF0F2690D086E700BF32
:10846000FC440220BC4402207844022000284CD066
:108470006B4B1A68904248D82DE9F04F5F6883B083
:108480000097002F51D07A1E964600214FF0010C24
:10849000644C019201EB0E02013253F83C50520839
:1084A00002F1010805EB450553F8379054F825A073
:1084B00053F8386009EB490503EBCC09D9F804906F
:1084C00006EB4606DAF810A054F8266054F825505A
:1084D0003AF829A003EBC80B03EBC7093669DBF8B0
:1084E00004B02D69D9F80490504536F82B6035F862
:1084F000295013D9A84210D2B04208D9C6454146E6
:10850000C0F0878008F1010CC4E70020704702F139
:10851000FF3E71457DD81746BCE73946009A8A422E
:1085200007D0102901D08A4208D8002003B0BDE846
:10853000F08F019A102A18BF1146F6D0DFF8E8C074
:10854000DDF8009003EBC108D8E9022602EB4202F5
:1085500054F8223004EB8202D2F804E01F69002EA6
:1085600055D03A467046B60007EB060A55880432E5
:1085700092452844FAD1BD19B5F802B08344834529
:1085800018D945095CF8252000F01F0622FA06FAE2
:108590001AF0010F07D013E05CF8252022FA06FA42
:1085A0001AF0010F0CD1013083454FEA501500F04D
:1085B0001F06F1D10131494508F10808C4D3B4E7D9
:1085C0000121B1409E8922EA0102A0EB0E004CF885
:1085D00025205C68002EA8D07A88824211D800211C
:1085E0003B1D03E05A88043382420AD833F8045C06
:1085F00001318E42A0EB020002FB05441F46F1D17F
:1086000093E73B8800FB034003B0BDE8F08F704662
:10861000B1E7009A102A08BF0F218FD085E700BF6D
:10862000FC440220BC4402207844022070B50022A1
:1086300001253348510950F8214002F01F0305FA83
:1086400003F301322343B2F5007F40F82130F1D12A
:1086500000242C4B21463C222B481C60FAF7C2F820
:1086600010210522294B2A4EC3E90044D9605961E3
:10867000D9615962D9625963D9635964D96459651A
:10868000D9655966D9665967D9679A601A619A613E
:108690001A629A621A639A631A649A641A659A65EE
:1086A0001A669A661A679A67C3E92021C3E92244C9
:1086B000C3E92421C3E92621C3E92821C3E92A21EA
:1086C000C3E92C21C3E92E21C3E93021C3E93221BA
:1086D000C3E93421C3E93621C3E93821C3E93A218A
:1086E000C3E93C21C3E93E21C3F80411C3F80021CA
:1086F000C3F80C11C3F808212046357070BD00BFC7
:1087000078440220B8440220BC440220FC440220E9
:10871000F84402202DE9F04F874B87B01B78002BDF
:1087200000F08C8028B321B30B78DFF8188203EBBC
:10873000031308EBC3035B68B1F80CC06344102B50
:1087400011D84FF0000A89467C4B7D4F1B684FEAD9
:108750008C0E0093B96891B10AF1010ABAF1050FC4
:1087600007F10C07F6D148F2071B584607B0BDE8E1
:10877000F08F48F20E1B584607B0BDE8F08FBCF1F1
:10878000000F61D00D460C46D9F810300EEB030BEC
:108790005A8833F8046B15449B4502FB0644F7D115
:1087A000D9F80830A342D7D3009B2B44B3F5007F00
:1087B000D2D2634C0AEB4A029200C0F800A0A01883
:1087C00044F80290009A8B46C0E9012599F80120EF
:1087D0005A48012A0360C8D0B9F80C30002BC4D025
:1087E0000025CDF80490CDF80CA0CDF814B0019B75
:1087F0001F781A693B0103EB0709009308EBC903D3
:10880000596832F82540029139BB039ADD609A60BD
:10881000009B3B441F4608EBC3014B6858F83720C8
:10882000013394424B6012D9019B48F837409B8931
:1088300001359D42DBD3DDF814B096E748F2081B02
:10884000584607B0BDE8F08F009B6546AEE7019B38
:1088500001359B89AB42CAD8EDE7002601F1FF3A0A
:10886000049506EB0A0009EB06020132013058F8C4
:1088700032C04008324D09EB000109EB0A03013117
:1088800001330CEB4C0C58F831E055F82CB058F88B
:1088900033C008EBC2020EEB4E0E0CEB4C0CDBF8B7
:1088A00010B0526855F82EE055F82CC008EBC10105
:1088B00008EBC3033BF82220DEF810E04968DCF83F
:1088C00010C05B6894423EF821103CF823302DD94B
:1088D0009C422DD28C4224D9461CB245C1D21026CE
:1088E000049D029AB24211D9009B3B441A4433447E
:1088F00008EBC20A08EBC309082251460AEB020042
:10890000AAF1080AF9F741FFD145F5D1009B039977
:108910003B443344013308EBC30248F8331055603D
:1089200076E700F1FF3A56459BD9D8E7049DD8E792
:10893000049D0AF10106D4E7F8440220B84402205D
:10894000BC440220FC440220034B1B780BB1FFF710
:108950008DBD1846704700BFF844022038B5084B5B
:108960001D7855B101FB00F42046FFF77FFD054659
:1089700018B122460021F9F735FF284638BD00BF5F
:10898000F8440220044B1B7823B118B101460020A3
:10899000FFF71CBC704700BFF8440220034B1B7854
:1089A0000BB1FFF77FBC1846704700BFF8440220A8
:1089B000044B1B7823B118B101460120FFF706BC18
:1089C000704700BFF84402200023184738B50A4C0E
:1089D0000A4B2578072A28BF0722084603EB4511D2
:1089E000F9F7D3FE237800200133DBB2072B08BF51
:1089F0000023237038BD00BF0C460220A8120500DA
:108A0000F0B5E5B09DF8A87158B152B14BB11F292E
:108A100007D919683F2904D93FB1552905D80C2435
:108A200000E01624204665B0F0BD1D460423002159
:108A30000446164614A84FF4A0728DF80C30F9F7CE
:108A4000D1FE14A804F03AFA002329491A4614A8C2
:108A5000009304F035FB14A82022214604F058FBB3
:108A6000B8B914A804F030FA21460DF10D0007F052
:108A700001FC0446B8B9C7B114A800F03FF80220C1
:108A800000F042F8014614A800F04CF8A8B10E24FA
:108A9000C8E7184A184B11782046072203EB41110A
:108AA000F9F773FEDDE72324BCE703A9701C40221D
:108AB000F9F76BFE41232B60B4E70321159806F00C
:108AC0002BFA0028E3D1159803AA00F1880141236D
:108AD00006F026F80028DAD1314614A82A6800F0FA
:108AE0006FF8B22304462B6000289BD0CFE700BF6D
:108AF000CD8904000C460220A812050010B1002305
:108B0000C0E90033704700BF022805D0034B03289B
:108B10000CBF18460020704701487047C01305007D
:108B20009013050060B159B170B5066866B94B6A1B
:108B300004460D469847606020B12560304670BD00
:108B400002487047024870BD004870BD80C1FFFFF9
:108B500080C0FFFF10B1006800B10078704700BF0F
:108B6000023802288CBF002001207047806D7047BA
:108B70000222034B883088600A704B60704700BF48
:108B800088130500023801288CBF0020012070479F
:108B900010B5044605F06AF92046BDE81040FFF71D
:108BA000F1BE00BF10B5AC210120FFF7D7FE04468F
:108BB00008B105F0F5F8204610BD00BF06F0CEB8AC
:108BC0002DE9F04F0024D7B00DF5AB7388469146E0
:108BD000CDE906430746FFF7BDFF022859D185239B
:108BE00078680BAE0193224600F1880100960AAB2B
:108BF0000A9405F043FF2DAD044668B90798A842D2
:108C00007FD30A9A431B93427BD3831A184631467B
:108C10000793F9F7BAFD0A9C002C31DB079B5A1B1E
:108C2000002A6EDD00215A1E04F1010A079207A8EE
:108C300003F8011C5246294601F088F8041E1FDB88
:108C40000322294607A801F0FBF8B0F1000B1BDB5B
:108C50003846FFF77FFF08AA09A906F09FF90346E7
:108C6000C8B1002B50DBC3F1A20206A9CDE90191E6
:108C7000CDF800802A442549254806F0C7F9044666
:108C8000204657B0BDE8F08F5C46204657B0BDE89F
:108C9000F08F204CF4E705903846FFF75BFF022881
:108CA000059B1DD01846DDE908320090294607A82B
:108CB00001F01CF9002822DB5444A34483445A46A3
:108CC000294607A801F042F8041ED9DB07A8302284
:108CD000294601F0B5F8031E16DBA3445B44C0E748
:108CE0007B68324618780AA906F074F928B9336807
:108CF0000A9A294607A801F0B1F80028D3DA0446F9
:108D0000BEE76FF06B04BBE71C46B9E7FC13050038
:108D10001814050080C6FFFF012838B50D4614461B
:108D200011D002280AD11020FFF70EFE182220B120
:108D3000074B456013448460036038BD0C20FFF787
:108D400003FE0022F3E71420FFF7FEFD3022EEE7DA
:108D50003414050010B5044603681B69984723685E
:108D600020465B6998472046BDE81040FFF70ABEE1
:108D700010B504460C20FFF7E7FDE06028B10023A2
:108D80002361BDE8104000F04DBF042010BD00BFBE
:108D900070B5064614200D46FFF7D6FD78B12B6856
:108DA000044643606B6801468360EB68C360AB6850
:108DB0000361F06800F040FF20B9686870BD4FF0B3
:108DC000FF3070BD2046FFF7DDFD4FF0FF3070BD76
:108DD0002DE9F04F824687B0C0688946934600F07F
:108DE0004BFF002872D00546D9F8080020B12B6946
:108DF00013B1EA68002A5CD10023C9F80C30D9F815
:108E00000020D9F80480DAF810100192B8F1000FB0
:108E10005AD00BF008030024009310E0DAF8103069
:108E20003B44CAF81030284600F02EFF3C4405466B
:108E3000002838D0A04536D90021D9F80020AE68E6
:108E4000A8EB040B761A5E45374628BF5F4632B161
:108E50006868019B01443A461819F9F796FC009B93
:108E6000002BE0D15E45D9D8DAF80C0000F0FAFE0C
:108E7000064670B1D0E90123D0E90301CDE9022310
:108E8000CDE90410DAE9013102A898473046FFF72E
:108E900079FD00232846CAF8103000F0F5FE3C4466
:108EA00005460028C6D12046C9F8044007B0BDE8F1
:108EB000F08FD9F80C309A4228BF1A46C9F80C2016
:108EC0002969F9F762FC9AE74446ECE74FF0FF3076
:108ED000ECE700BF10B50446C06800F0CDFE50B10D
:108EE0002469644283681C4400F0CEFE0028F9D156
:108EF00024EAE47010BD4FF0FF3010BD30B50546D8
:108F0000C06885B0A8B91AE0E86800F0ABFE044676
:108F100070B1D0E90101D4E90332CDE90001CDE916
:108F20000223D5E90131684698472046FFF72AFD1C
:108F3000E86800F0A7FE0028E6D105B030BD0820A3
:108F400005B030BD30B50546C06885B0A0B91CE09D
:108F500000F088FE044670B1D0E90101D4E9033283
:108F6000CDE90001CDE90223D5E9013168469847F2
:108F70002046FFF707FDE86800F084FE0446E86835
:108F8000002CE5D1FFF7FEFCEC6005B030BD00BF62
:108F9000006800F03FBE00BF70B582B00E461446B8
:108FA0000546FEF7A1FB002841D003689B033ED590
:108FB0000368214623F400330360036843F48013FD
:108FC000036001A800F0FCFD78BB0422019B1A722B
:108FD00058729872D872DD607CB91846012100F091
:108FE00003FEC8B94FF40032284611460023FEF7AD
:108FF0000FFBA8B9204602B070BD31461868224662
:10900000F9F7C3FB0121019800F0EEFD0028E9D03B
:10901000019B186800F0FEFD019800F0F3FD23208D
:10902000FAF7F9F84FF0FF30E5E70C20F8E71620E3
:10903000F6E700BF00F0BEBD2DE9F041002582B08B
:1090400002AB43F8085D80460F46184616460221DB
:109050001C4AFEF747FA009B044603B3C3E90287A4
:109060001E61294601A800F0ABFDE0B90422019B76
:10907000052158729872D8721A72DC60184600F096
:10908000B3FDD0B90222034611462046FEF7C0FACE
:10909000054648B9009A136843F40033136020462C
:1090A00002B0BDE8F0810C252046FEF76FFA284695
:1090B000FAF7B1F84FF0FF34F1E7019800F0A2FDA4
:1090C0002325F1E7918F0400F0B583B00646FEF743
:1090D0000BFB00283CD00E2307680360036804469E
:1090E0009B031ED4002101A800F06AFD18BB0422D6
:1090F000019B062158729872D8721A72DE60184667
:1091000000F072FDC8B90F22034611463046FEF743
:109110007FFA0546A8B93046FEF738FA284603B06C
:10912000F0BD0368002123F40033036001A800F0C0
:1091300047FD0028DBD00C2503E0019800F062FD1C
:10914000232527602846FAF766F84FF0FF35E5E754
:109150001625F7E72DE9F04184B0884615461E46EE
:109160000746FEF7C1FA002844D00023CDE9008568
:1091700016F002050446CDE9023309D019E07DBBA3
:109180004FF48032E36911463846FEF741FA05464E
:109190002368A06923F480332360036832469B6808
:1091A00069469847B0F10008E9DB404604B0BDE8E5
:1091B000F0810368806923F48033236003683246BA
:1091C0009B6869469847B0F10008EEDAB8F1FF3FB6
:1091D000EBD12320FAF71FF8404604B0BDE8F08138
:1091E000B8F1FF3FE1D12846FAF715F8404604B040
:1091F000BDE8F0811620FAF70EF84FF0FF38D4E7FB
:109200004FF0FF30704700BF012901D02A2070477E
:1092100038B51D461446FEF767FA034668B1142CAC
:1092200007D165B1049A042A05D12A680020DA61C1
:1092300038BD2A2038BD162038BD092038BD0E2083
:1092400038BD00BF70B5054684B0C0680E46FEF755
:109250004BFA40B3036804469BB2012B1FD003684E
:109260009BB20E2B27D003689BB2022B2ED0033E5D
:10927000012E11D8002329686A68CDE90233CDE9AF
:109280000012A069694603685B689847013017D0EF
:10929000236843F480332360002004B070BD022EA5
:1092A000E5D10660F8E728680028F5D000F0B2FCA8
:1092B000002004B070BD022ED9D10F230360EBE76C
:1092C000286800F0A7FC002004B070BD0368DB0232
:1092D000CDD5022ECBD1036823F48013036003683D
:1092E00043F400330360D7E750F8081B090CFDF77F
:1092F000F3BE00BF0148FEF787BA00BF7C1405002B
:10930000002310B582B0019358B1044601AA04208D
:10931000FEF7BAFC18B9019B0BB10833236002B009
:1093200010BD072002B010BD01F47043B3F5E04F4B
:109330000BD160B1034630F8082C042042EA014109
:1093400043F8081D1946FEF787BC0F207047072019
:10935000704700BF20B1A0F108010420FEF7C8BC8F
:109360000720704718B101460420FEF771BD0720A1
:10937000704700BFF8B50C460023496947F28102E7
:1093800027680646FCF78AFF00283CD005461F4B9D
:1093900006EBC60103EB810124221430F9F7F5F93D
:1093A000AB6829462433AB6022683B46120C12049A
:1093B00042F00B022260204647F28102FCF78EFF4A
:1093C00040B903464FF6FF720C213046FCF79AFF76
:1093D00008B12760F8BD4FF400020346114630463D
:1093E000FCF790FF0028F4D10D22236823F400033A
:1093F00023602260236843F400332360236843F42E
:1094000000232360F8BD0C20F8BD00BF10460220E9
:109410000020704738B520F00803022B06D02F201B
:10942000F9F7F9FE4FF0FF35284638BD14464A1EBD
:10943000012A28D814BB012906BF01234FF48274E6
:109440004FF487741A46FCF795FF051E26DB154B73
:1094500005EBC50003EB800024221349F9F795F9C9
:109460002846FEF741F90368046123F400230360F2
:10947000036823F400330360284638BD012908D06F
:10948000B4F5877FDED01620F9F7C5FE4FF0FF3523
:10949000CAE7B4F5827FF6D10B46D3E74FF0FF352C
:1094A000C2E700BF104602208C14050010B5044628
:1094B000FEF71AF920B12046BDE81040FDF704B8C8
:1094C0000920F9F7A8FE4FF0FF3010BD2DE9F04755
:1094D0000D46DDE9088916461F460446FEF704F9E5
:1094E00000283BD003689BB20D2B39D003689BB298
:1094F0000C2B11D1204B04EBC40413F82430022BA5
:1095000038D0C368012B14BF39202A20F9F783FE15
:109510004FF0FF30BDE8F087C368012B0BD0022B62
:1095200001D03920F2E703689BB2022B07D0036811
:109530009BB2042B03D003689BB2062BF1D10E4BD8
:1095400004EBC40213F82230022BEAD10146204674
:10955000FFF710FF002803D0D8DCD9E70920D5E7B2
:10956000CDE908893B46324629462046BDE8F0470A
:10957000FDF71AB82320C9E7104602202DE9F04371
:1095800083B00D46DDE90A8916461F460446FEF7FC
:10959000ABF8002839D003689BB20D2B2AD0C368E2
:1095A000012B12D0022B08D04FF0FF342320F9F703
:1095B00032FE204603B0BDE8F08303689BB2022B65
:1095C00007D003689BB2042B03D003689BB2062B21
:1095D000EAD1154B04EBC40213F82230022BE3D17D
:1095E00001462046FFF7C6FE002812D04FF0FF3498
:1095F000DDDCDEE72046CDE900893B4632462946E0
:10960000FDF7ACF804462320D1E74FF0FF340920E2
:10961000CDE73B46324629462046CDE90A8903B0CC
:10962000BDE8F043FDF79AB8104602202DE9F84353
:109630000C4617460646FEF757F8002855D0036833
:1096400005469BB2022B4AD121463A463046FDF7E9
:109650000BFA0446C8BB06EBC607DFF89480BF00D0
:1096600018F80730012B02D02046BDE8F8830346E6
:1096700047F2810269693046FCF710FE814690B3DB
:1096800008EB070124221430F9F77FF8D9F80830E5
:1096900049462433C9F808302A680423120C1204FE
:1096A00042F00B022A60284647F28102FCF716FEC0
:1096B000B8B9304623464FF6FF720C21FCF722FE64
:1096C0000028D1D0042304462B60002CCCDD20469A
:1096D0004FF0FF34F9F79FFD2046BDE8F8832D24B5
:1096E000F5E70446F1E70C24F1E70924EFE700BFB2
:1096F00010460220F8B50E4617460546FDF7F4FF62
:1097000028B3174B05EBC50213F82230022B24D1E6
:10971000036804469BB2022B03D003689BB2042B60
:109720001BD13A4631462846FDF7EAF810B1002829
:109730000EDCF8BD2368284623F400332360236839
:10974000214623F400232360FFF714FEEFE70920EE
:10975000F9F761FD4FF0FF30F8BD2D20F8E700BFAD
:10976000104602202DE9F0470F460646FDF7BCFFE4
:10977000002861D0C3680446012B5BD103689BB20B
:10978000042B47D023689BB20C2B53D1F300DFF896
:10979000AC909A1919F82220012A4BD101223344A6
:1097A0009D0009F805206169002347F281023046D7
:1097B000D4F80080FCF772FD8246A0B309EB0501E6
:1097C00024221430F8F7E1FFDAF808305146243348
:1097D000CAF8083022684346120C120442F00B0209
:1097E0002260204647F28102FCF778FD48B9034623
:1097F0004FF6FF720C213046FCF784FD28B1C4F807
:109800000080002810DCBDE8F08739463046FDF7BF
:10981000DFF9F6E7F300DFF824909A1919F822200F
:10982000022AAFD1BAE70C20F9F7F5FC4FF0FF3070
:10983000BDE8F0872D20F7E70920F5E71046022064
:10984000F8B50C4616461F460546FDF74DFF0028A5
:109850003AD0006880B2072836D121463B463246CE
:109860002846FDF74DFA044618B1002C2DDC2046A1
:10987000F8BD2846FDF738FF0368174F23F400337F
:109880000360036805EBC50523F400230646036067
:1098900007EB850124223846F8F777FF02233B7057
:1098A00032682346120C120442F00C023260204649
:1098B0004FF6FF720D21FCF725FD04460028D6D097
:1098C0000020FCF701FED0E7092420464FF0FF34CA
:1098D000F9F7A1FC2046F8BD104602202DE9F04121
:1098E000B1F58D7F069F1DD11C46C3B1BFB10546A2
:1098F0001646FDF7F9FEC8B103689BB2022B07D0EC
:1099000003689BB2042B03D003689BB2062B0DD1D6
:10991000013E032E51D8DFE806F02532180B0E2049
:10992000BDE8F081BDE8F041FDF7FEBA0920F7E798
:10993000042F39D12368022B36D8214A05EBC505FF
:1099400002EB8505AB700020EAE7012F2CD12378CC
:10995000012B29D81A4A05EBC50502EB8502537085
:109960000020DDE7042F1FD12068F8B101281BD1AA
:10997000134B05EBC50503F825000020D0E75FEA8F
:10998000970C11D017F003060ED105EBC505AD00FD
:109990000B4B281D18442B443A46214683F803C03C
:1099A000F8F7F3FE3046BBE71620B9E70222044B76
:1099B00005EBC50503F82520B2E72A20B0E700BF74
:1099C000104602202DE9F041B1F58D7F069F12D19E
:1099D0001D466BB167B106461446FDF785FE0028AB
:1099E0004FD0013C032C52D8DFE804F0392115098F
:1099F0000E20BDE8F081BDE8F041FDF7B3BA3B6849
:109A0000042B3CD1234B06EBC60603EB8606B3784A
:109A100000202B60EDE73B68042B30D11D4B06EB9B
:109A2000C60603EB8606737800202B60E1E706EBA1
:109A3000C60618493B68B6008A1913F00304D078AB
:109A400021D19B08834228BF03469A00DBB104362C
:109A500031443A602846F8F798FE2046C9E73B684B
:109A6000042B0CD10B4B06EBC60613F82630002056
:109A7000A3F10103B3FA83F35B092B60B9E7162066
:109A8000B7E70920B5E70028F9D13860B1E72A2007
:109A9000AFE700BF1046022010B448F28104A24292
:109AA000034610D049F28200824208D11BB11A68E5
:109AB00092B20C2A16D000205DF8044B70470120AA
:109AC0005DF8044B70470028F5D0026892B20B2A6B
:109AD000F1D1486958B91A68120C120442F00C020C
:109AE0001A60EDE7086920B158600020E8E7586087
:109AF000E1E71A6842F400021A60E1E7FDF736BABE
:109B0000FDF7CCBA2DE9F04F83B0002847D00729E4
:109B100045D8074691468846824600EBC106B8F113
:109B2000000F18D03C460025206801A9B4F804B005
:109B3000FDF7E8FD019B083403F003030BEA030380
:109B400024F8023C03B10135B442EDD11DB12846E1
:109B500003B0BDE8F08F49463846F9F75AFBB9F132
:109B6000000FDCD0B8F1000F17D00025DAF80000A4
:109B700001A9BAF80440FDF7C5FD019B0AF1080AE6
:109B800003F0030323402AF8023C03B10135B24538
:109B9000ECD1284603B0BDE8F08F4546D7E74FF03B
:109BA000FF35D4E720B150F8081B090CFFF74ABB7A
:109BB000704700BF0148FDF727BE00BFB014050085
:109BC00080B1002310B582B002AA044642F8043DD9
:109BD0000320FEF759F818B9019B0BB10833236035
:109BE00002B010BD0E20704750B1034630F8082C6B
:109BF000032042EA014143F8081D1946FEF72CB83C
:109C00000E20704720B1A0F108010320FEF770B8C4
:109C10000E20704718B101460320FEF719B90E2037
:109C2000704700BF28B100230360C0E90133184624
:109C300070470720704700BF0268034601320ED00C
:109C400000220A6002683AB18268116081601A6875
:109C5000002001321A607047C0E90111F7E70420C3
:109C6000704700BF0346006828B158681A68016849
:109C7000013A59601A60704703680BB14068704739
:109C800018467047006870470068704730B4034654
:109C90000068B2F5803FA0EB010114D2022951DD2A
:109CA000411E196000F8012C19688224481E1860B2
:109CB0000320120A01F8012C1A68511E196002F8DB
:109CC000014C30BC7047B2F1807F1AD2032939DDD4
:109CD0008324411E196000F8012C1968100A4D1EDA
:109CE0001D6001F8010C1968120C481E186001F87B
:109CF000012C1A680420511E196002F8014C30BC76
:109D0000704704291EDD8424411E196000F8012CCF
:109D10001968100A4D1E1D6001F8010C1968100C1D
:109D20004D1E1D6001F8010C1968120E481E1860C6
:109D300001F8012C1A680520511E196002F8014C27
:109D400030BC70476FF06B00BBE700BF30B40468F5
:109D50007F2A0346A4EB010108D800296CDD611EAF
:109D60000160012004F8012C30BC7047FF2A0ED896
:109D7000012961DD8121601E186004F8012C1A6838
:109D80000220541E1C6002F8011C30BC7047B2F562
:109D9000803F1CD3B2F1807F2ED203294CDD832576
:109DA000611E016004F8012C0168100A4C1E1C6041
:109DB00001F8010C1968120C481E186001F8012CFA
:109DC0001A680420511E196002F8015CCCE70229D0
:109DD00032DD8225611E016004F8012C0168120A3F
:109DE000481E186001F8012C1A680320511E1960E2
:109DF00002F8015C30BC704704291DDD8425611E1A
:109E0000016004F8012C0168100A4C1E1C6001F866
:109E1000010C1968100C4C1E1C6001F8010C19682B
:109E2000120E481E186001F8012C1A680520511EF8
:109E3000196002F8015C97E76FF06B0094E700BFD0
:109E40000368591A002905DD591E0160012003F835
:109E5000012C70476FF06B00704700BFF8B50568C4
:109E6000A9423FD80F46691A8B423BD806461C468A
:109E7000E81A114630601A46F8F787FC002C204695
:109E800015DB7F2C14D83368DA1B002A2ADD012069
:109E90005A1E326003F8014C33680134DF1B002F77
:109EA00020DD0622591E3160204403F8012CF8BD44
:109EB000FF2C0FD83368DA1B012A13DD8122591ECB
:109EC000316003F8014C33680220591E316003F8F9
:109ED000012CE1E7224639463046FFF7D7FE00283D
:109EE000DADAF8BD6FF06B00F8BD00BF2DE9F04184
:109EF000DDF818800568B8F1000F13D16C1A002C3A
:109F000040F387806C1E046005F8018C0468651AB4
:109F1000002D7EDD05254FF00208661E066004F860
:109F2000015C0568A94274D86C1AA34271D8064630
:109F30001C46E81A0F46306011461A46F8F725FC11
:109F4000002C20462FDB7F2C41D83368DA1B002AF7
:109F50005FDD01205A1E326003F8014C3368013482
:109F6000DA1B002A55DD06220444591E002C3160FC
:109F7000204603F8012C16DB44447F2C15D83368A7
:109F8000DA1B002A45DD01205A1E326003F8014C1D
:109F900033680134DF1B002F3BDD3022591E316056
:109FA000204403F8012CBDE8F081FF2C21D8336850
:109FB000DA1B012A2DDD8122591E316003F8014C84
:109FC00033680220591E316003F8012CE0E7FF2CB2
:109FD00017D83368DA1B012A1BDD8122591E316034
:109FE00003F8014C33680220591E316003F8012C3C
:109FF000B4E7224639463046FFF748FE0028D2DB58
:10A00000C6E7224639463046FFF740FE0028A5DA6B
:10A01000C9E76FF06B00C6E72DE9F04FDDF824C00B
:10A02000BCF1000F65D0424CA4FB0C54640804EB57
:10A030004408C44518BF0134B4F1804F71D2A40064
:10A0400001348C4269D8002867D0B8F1000F61D084
:10A0500086460027374EDC1C002514F8031C14F834
:10A06000023C14F801BC4FEAA109090101F03001DA
:10A0700006EB131A16F809909B001AF801A003F0DA
:10A080003C0106EB9B13595C69F307050BF03F039A
:10A09000F35C6AF30F2561F31745033763F31F651C
:10A0A0000EF10401B845CEF8005023468E4604F167
:10A0B0000304D1D8BC4514D91C781E4D0137A61015
:10A0C00067454FEA041404F0300415F806E015D390
:10A0D0003D262B5D81F800E04B703D238E70CB70E8
:10A0E000043100239C46081A10600B706046BDE8DE
:10A0F000F08FC2F800C06046BDE8F08F5B7881F851
:10A1000000E005EB1316345D9B0003F03C034C703C
:10A11000EE5CE2E747460146CCE714606FF0290C9D
:10A12000E4E74FF0FF336FF0290C1360DEE700BF68
:10A13000ABAAAAAAC01405000F282DE9F04F864645
:10A1400040F2E0824FF00008844601F1400402F141
:10A15000400054F8406C50F8405CA3FB066718EBD5
:10A1600006082CBF4FF001094FF0000915EB080558
:10A170004F444FF0000928BF4FF0010940F8405C00
:10A1800054F83C6CB944A3FB06AB19EB0A092CBF8D
:10A190004FF001084FF0000850F83C6C08EB0B053D
:10A1A00016EB09064FF0000828BF4FF0010840F8F1
:10A1B0003C6C54F8386CA844A3FB066718EB0608FF
:10A1C0002CBF4FF001094FF0000950F8385C4F44A4
:10A1D00015EB08054FF0000928BF4FF0010940F8C2
:10A1E000385C54F8346CB944A3FB06AB19EB0A098C
:10A1F0002CBF4FF001084FF0000850F8346C08EB0A
:10A200000B0516EB09064FF0000828BF4FF00108B8
:10A2100040F8346C54F8306CA844A3FB066718EB84
:10A2200006082CBF4FF001094FF0000950F8305CD0
:10A230004F4415EB08054FF0000928BF4FF0010906
:10A2400040F8305C54F82C6CB944A3FB06AB19EB16
:10A250000A092CBF4FF001084FF0000850F82C6C91
:10A2600008EB0B0516EB09064FF0000828BF4FF06E
:10A27000010840F82C6C54F8286CA844A3FB06672E
:10A2800018EB06082CBF4FF001094FF0000950F8F9
:10A29000285C4F4415EB08054FF0000928BF4FF02C
:10A2A000010940F8285C54F8246CB944A3FB06ABC0
:10A2B00019EB0A092CBF4FF001084FF0000850F8C5
:10A2C000246C08EB0B0516EB09064FF0000828BFBD
:10A2D0004FF0010840F8246C54F8206CA844A3FB0C
:10A2E000066718EB06082CBF4FF001094FF0000974
:10A2F00050F8205C4F4415EB08054FF0000928BFCB
:10A300004FF0010940F8205C54F81C6CB944A3FBE1
:10A3100006AB19EB0A092CBF4FF001084FF00008FB
:10A3200050F81C6C08EB0B0516EB09064FF0000803
:10A3300028BF4FF0010840F81C6C54F8186CA84472
:10A34000A3FB066718EB06082CBF4FF001094FF07E
:10A35000000950F8185C4F4415EB08054FF0000950
:10A3600028BF4FF0010940F8185C54F8146CB94448
:10A37000A3FB06AB19EB0A092CBF4FF001084FF005
:10A38000000850F8146C08EB0B0516EB09064FF0AB
:10A39000000828BF4FF0010840F8146C54F8106C06
:10A3A000A844A3FB066718EB06082CBF4FF0010971
:10A3B0004FF0000950F8105C4F4415EB08054FF0C2
:10A3C000000928BF4FF0010940F8105C54F80C6CEC
:10A3D000B944A3FB06AB19EB0A092CBF4FF00108E7
:10A3E0004FF0000850F80C6C08EB0B0516EB090653
:10A3F0004FF0000828BF4FF0010840F80C6C54F8EB
:10A40000086CA844A3FB066718EB06082CBF4FF0A6
:10A4100001094FF0000950F8085C4F4415EB08059E
:10A420004FF0000928BF4FF0010940F8085C54F8CC
:10A43000046CB944A3FB06AB19EB0A092CBF4FF01F
:10A4400001084FF0000850F8046C08EB0B0516EB00
:10A4500009064FF0000828BF4FF00108ACF1100CBE
:10A46000BCF10F0F40F8046CA84404F1400400F163
:10A4700040003FF66EAEAEF11000000901308001E1
:10A48000014402440EF00F000728176840F2928042
:10A490000C685668A3FB049A18EB09082CBF4FF010
:10A4A000010C4FF0000C17EB08072CBF012400240F
:10A4B00017604F680AEB0C05A3FB07892C4414EBCB
:10A4C00008042CBF01250025A61905EB09074FF04C
:10A4D000000528BF012556608E683D44A3FB067821
:10A4E000ED192CBF01240024966808EB0407AD1970
:10A4F0004FF0000428BF01249560CE683C44A3FBC4
:10A500000678E4192CBF01250025D66808EB05075D
:10A51000A4194FF0000528BF0125D4600E693D4401
:10A52000A3FB0678ED192CBF01240024166908EB63
:10A530000407AD194FF0000428BF012415614E69CE
:10A540003C44A3FB0678E4192CBF0125002556697D
:10A5500008EB0507A4194FF0000528BF0125546139
:10A560008E693D44A3FB0678ED192CBF012400241D
:10A57000966908EB0407AD194FF0000428BF0124C9
:10A580009561CE693C44A3FB069A14EB09042CBFE9
:10A590004FF001084FF00008D66908EB0A05A4192E
:10A5A0004FF0000828BF4FF00108D4612031A844C3
:10A5B00008382032002800F097800C681668A3FB4A
:10A5C000049A19EB08082CBF0124002416EB080696
:10A5D0004FF0000528BF01255444012805EB04086D
:10A5E00016607FD04C685668A3FB049A19EB0808E4
:10A5F0002CBF0124002416EB08064FF0000528BFED
:10A6000001255444022805EB040856606AD08C6882
:10A610009668A3FB049A19EB08082CBF01240024B8
:10A6200016EB08064FF0000528BF01255444032807
:10A6300005EB0408966055D0CC68D668A3FB049A55
:10A6400019EB08082CBF0124002416EB08064FF074
:10A65000000528BF01255444042805EB0408D660F2
:10A6600040D00C691669A3FB049A19EB08042CBFAF
:10A670004FF001084FF00008A6190AEB08054FF04B
:10A68000000828BF4FF001080528A844166129D00A
:10A690004C695669A3FB049A18EB09042CBF4FF0D0
:10A6A00001084FF00008A6190AEB08054FF0000852
:10A6B00028BF4FF001080628A844566112D08C69C3
:10A6C0009169A3FB044514EB08082CBF0123002368
:10A6D00011EB08014FF0000428BF01242B4404EBC8
:10A6E0000308916102EB80021568002315EB080551
:10A6F00028BF012342F8045B4FF00108002BF3D17F
:10A70000BDE8F08F4FF00008BEE600BF4368002BA5
:10A7100033D030B403F180428568013A55F82240C5
:10A7200005EB82021CB109E052F8044D34B9013B3B
:10A73000FAD18B681868D0B930BC70478A68126843
:10A7400092B1012B10D800680B68002801DD002BA6
:10A7500011DB002B01DD002816DB2B689342EBD8C0
:10A7600006D330BC00207047006830BC70470868D2
:10A77000404230BC70470120DEE78B68186800B9A2
:10A78000704708684042FBE74FF0FF30D4E700BF56
:10A7900020B100230122C0E900238360704700BF7D
:10A7A000B0B110B50446806860B16268531E3AB11A
:10A7B0000022013B591C026000F10400F9D1A0689D
:10A7C000FEF7E0F800230122C4E90023A36010BDD6
:10A7D000704700BF70B5426805468A420C4607D8EC
:10A7E00042F21073994251D88A4235D3002070BD8D
:10A7F000511E10D0836853F82100002849D102F17E
:10A800008042013A03EB820303E053F8040D18B9C8
:10A8100011464A1EF9D101218C4238BF0C46042151
:10A820002046FEF79BF8064680B3A96881B1A200D6
:10A83000F7F7ABFFD5E90120531E3AB10022013BE7
:10A84000591C026000F10400F9D1A868FEF79AF8DB
:10A85000C5E90146002070BD04212046FEF77EF8C0
:10A86000064698B1A9680029F2D06A689200F7F705
:10A870008CFFD5E90120531E002AE7D00022013BBE
:10A88000591C026000F10400F9D1DEE76FF00F00FF
:10A8900070BD1146C0E700BF884252D0F8B58A6843
:10A8A0000E460546002A4ED049684B1E0ED052F87F
:10A8B000230000283BD101F18041013902EB8102E4
:10A8C00002E052F8040D90BB013BFAD10124336839
:10A8D0002B606A68A2420CD3AF6892000021384610
:10A8E000F7F780FFA200B168A868F7F74EFF0020D5
:10A8F000F8BD04212046FEF731F80746F0B1A968FB
:10A9000089B16A689200F7F740FFD5E90120531E2C
:10A910003AB10022013B591C026000F10400F9D158
:10A92000A868FEF72FF82246C5E90147D5E742F2AD
:10A93000107231685C1C94422960CAD96FF00F0014
:10A94000F8BD002070470028D1D0806858B16968F0
:10A950004B1E31B1013B5C1C026000F10400F9D1D7
:10A96000A868FEF70FF800200123C5E90030A860B1
:10A97000F8BD00BFF0B54B680D4685B014460646DD
:10A9800051687BB1A86803F18042013A50F8227007
:10A9900000EB820027B14FE050F8042D002A4BD184
:10A9A000013BF9D189B101F18040A768013857F81E
:10A9B0002020002A40F0998007EB800003E050F847
:10A9C000042D002A42D10139F9D100230122B442D9
:10A9D000CDE9012303937FD0B54205D02946304607
:10A9E000FFF75AFF0746A8B901233360606880B1BA
:10A9F000D4F808C000F18043013B5CF823200CEB45
:10AA0000830322B142E053F8042D002A3ED10138DD
:10AA1000F9D10027039860B1029A531E3AB100227F
:10AA2000013B591C026000F10400F9D10398FDF7C5
:10AA3000A9FF384605B0F0BD0029C6D001F180401D
:10AA4000A768013857F82020002AB5D08B42BCD81F
:10AA50004BD3002BB9D0A86803F18041013950F8DD
:10AA600021C057F821E08900E645084407EB0102C0
:10AA7000ABD33AD8014606E051F8047D52F8040DF4
:10AA80008742A2D831D3013BF6D19EE700252B4661
:10AA9000B16851F8046B0135F21A41F8042C5CF8E6
:10AAA000047B0C46BA422CBF4FF0000E4FF0010E53
:10AAB000D21B9E422CBF73460EF10103854241F822
:10AAC000042CE6D30BB9A4E701232268D11A9A42D9
:10AAD00044F8041BF8D39CE7214601A8FFF7DCFEED
:10AAE0000746002896D101AC76E76FF00907384693
:10AAF00005B0F0BD42F210732DE9F0414F685642A7
:10AB000016439F42C6F3C0164FD842680446974288
:10AB10000D462CD82968236801FB06F1C6F1010710
:10AB200003FB071323606B688BB10023A168AA683D
:10AB300051F8230052F8232000FB07F002FB060225
:10AB400041F823206A6801339A42EFD86268934241
:10AB50000AD29A00A0680133815807FB01F18150A5
:10AB6000616804329942F5D80020BDE8F0810421E3
:10AB70003846FDF7F3FE8046B8B1A16889B1626836
:10AB80009200F7F702FED4E90120531E3AB10022E9
:10AB9000013B591C026000F10400F9D1A068FDF7E7
:10ABA000F1FE3A46C4E90178B4E76FF00F00DCE744
:10ABB000F8B5456804460E469DB18768AA00384638
:10ABC0000021F7F70FFE002EACBF01234FF0FF333B
:10ABD00086EAE671A268A1EBE671116023600020AD
:10ABE000F8BD04210120FDF7B9FE0746B8B1A16800
:10ABF00081B162689200F7F7C8FDD4E90120531EC5
:10AC000032B1013B5A1C056000F10400F9D1A06883
:10AC1000FDF7B8FE01230422C4E90137CFE76FF046
:10AC20000F00F8BD4368B1EB431F09D283684A099E
:10AC300053F8220001F01F01C84000F001007047E6
:10AC400000207047436813B310B48268581E24D0A4
:10AC500052F82010E9B903F18043013B02EB830372
:10AC600002E053F8041DA1B90138FAD1202411687B
:10AC700000224FF0004302E00132202A04D00B42B0
:10AC80004FEA5303F8D0A01A5DF8044B70471846FA
:10AC90007047400100F12004EAE711682024E7E74B
:10ACA000436823B310B48268581E26D052F820108F
:10ACB000F9B903F18043013B02EB830302E053F84F
:10ACC000041DB1B90138FAD12024116800224FF0D7
:10ACD000004302E00132202A04D00B424FEA530322
:10ACE000F8D0A01A0730C0085DF8044B704718462A
:10ACF0007047400100F12004E8E711682024E5E7EF
:10AD00002DE9F84305460F461646002A7ED00C78FA
:10AD10000B4624B17EE013F8012F002A46D10134FE
:10AD2000A642F8D1D5F80480B8F1000F69D104210A
:10AD30000120FDF713FE814600286DD0A96889B176
:10AD40006A689200F7F721FDD5E90120531E3AB158
:10AD50004246013B591C026000F10400F9D1A86889
:10AD6000FDF710FE01230422C5E901390021484600
:10AD7000F7F738FD00230122A968A6420B602A607C
:10AD800011D907EB060C341BAE6823F00301DF007A
:10AD90001CF8010D725807F01807B8400133024340
:10ADA000A3427250F0D10020BDE8F883321B12F0AC
:10ADB000030818BF4FF0010842F2107308EB920825
:10ADC000984529D86B68984529D904214046FDF754
:10ADD000C5FD814600B3A96889B16A689200F7F79A
:10ADE000D4FCD5E90120531E3AB10022013B591C85
:10ADF000026000F10400F9D1A868FDF7C3FDC5E9C0
:10AE000001894FEA8802D5F80890AFE7D0F80480AE
:10AE1000144689E70024CAE76FF00F00C4E798469C
:10AE200082E700BF2DE9F04144688846002C3ED0FF
:10AE30001546621E0746806840D050F8221099BB24
:10AE400004F18043013B00EB830302E053F8041D4F
:10AE500051BB013AFAD12726016800224FF0004386
:10AE600002E00132202A03D00B424FEA5303F8D00C
:10AE7000B61AF608B54224D32A4600214046F7F711
:10AE8000B1FC76B10023A844B96823F003028C58C2
:10AE9000DD0005F018050133EC40B34208F8014D20
:10AEA000F2D10020BDE8F08156012736D5E70846EB
:10AEB0002146F7F797FC2046BDE8F0810168272678
:10AEC000CBE76FF00700EDE72DE9F041436804465A
:10AED0004D0901F01F0643B35A1ED0F808E000F0F8
:10AEE00099805EF822C0BCF1000F40F09C8003F115
:10AEF000804001380EEB800003E050F8047D002F05
:10AF00005ED1013AF9D14FF02008DEF80070002040
:10AF10004FF0004202E00130202805D03A424FEACB
:10AF20005202F8D0A8EB000C6144B1EB431F0BD9DF
:10AF300011F01F0218BF012242F2107002EB5117EC
:10AF400087426DD89F4240D8F5B19D425DD26FF0E7
:10AF500040477F1BDA19C7EB87779200BF00A068D4
:10AF6000013BC119805811449D4241F8040CA2F1E3
:10AF70000402F4D1002103F18043013B9B00A2684D
:10AF8000D150043B1A1DFAD1BEB163689D4214D260
:10AF90000027C6F1200CAB00A0680135C15801FAAA
:10AFA00006F2C250A068C2583A43C250626821FA01
:10AFB0000CF7AA4203F10403EED80020BDE8F081AB
:10AFC0004FEA421C0CF12008A1E704213846FDF7A6
:10AFD000C5FC804620B3A16889B162689200F7F78A
:10AFE000D4FBD4E90120531E3AB10022013B591C85
:10AFF000026000F10400F9D1A068FDF7C3FC3B46F4
:10B00000C4E90178002DBFD09FE7002BB2D1002EFC
:10B01000BBD1D2E7DEF8007094464FF0200876E707
:10B020006FF00F00CAE75201674602F1200894460C
:10B030006DE700BFF8B544684D09AC423AD301F062
:10B040001F0132D0B5B10023AA008468A65804328B
:10B0500044F8236044680133661B9E42F5D89C4245
:10B0600008D900259A0084680133A5504468043249
:10B070009C42F8D8B9B1B4B1002704F18043013B38
:10B080009B00C1F1200C8668013CF55825FA01F2BD
:10B09000F2508668F25842EA0702F25005FA0CF7BD
:10B0A000A3F10403EFD10020F8BD19B9002CFAD0A8
:10B0B0000B46D6E7054664B18668A20030460021FB
:10B0C000F7F790FB00230122A96818460B602A605D
:10B0D000F8BD04210120FDF741FC0646B8B1A9687E
:10B0E00081B16A689200F7F750FBD5E90120531E41
:10B0F00032B1013B5A1C046000F10400F9D1A86888
:10B10000FDF740FC01230422C5E90136D6E76FF0C4
:10B110000F00F8BD70B443684A6873B1846803F1E6
:10B120008045013D54F8256004EB85041EB11AE00A
:10B1300054F8045DBDB9013BFAD18AB102F18044F3
:10B140008E68013C56F82450CDB906EB840402E029
:10B1500054F8045D8DB9013AFAD1002B37D002685A
:10B16000104670BC7047002AF9D002F180448E6806
:10B17000013C56F82450002DE7D09342EFD893427B
:10B18000096803D270BC4A42104670470268002A20
:10B1900001DD002924DB002901DD002A1DDBB3B11C
:10B1A000846803F18041013954F8215056F8210098
:10B1B000890085420C443144D2D80CD3013B06D0DF
:10B1C00054F8045D51F8040D8542F6D9C8E71A46D3
:10B1D00070BC104670475242C2E74FF0FF32BFE7E3
:10B1E0000122BDE7F0B400290546436832DB002B9D
:10B1F00042D0866803F18042013A56F8220006EBFD
:10B20000820268B94FF0FF30012702E052F8044D86
:10B210003CB9013BFAD1002908BF0020F0BC7047BF
:10B220000127A1B1012B12D82868002801DD7B1C61
:10B230001ED0012F01D1002824DB00293368B8BFBC
:10B2400049429942EAD315D8F0BC002070472868DB
:10B25000F0BC704763B1866803F18042013A56F84A
:10B26000220006EB820250B901204FF0FF37D0E7F1
:10B270000120D3E74042D1E74FF0FF30CBE74FF05A
:10B28000FF37CFE74FF0FF30C8E700BF90422DE90E
:10B29000F04707460C4606D08842154602D0FFF715
:10B2A000FBFAA0B92C4601233B60656875B1A36821
:10B2B00005F18042013A53F8221003EB820219B1E2
:10B2C00007E052F8041D21B9013DFAD10020BDE884
:10B2D000F08742F21072954275D87A68AA4276D207
:10B2E00004212846FDF73AFB064600286BD0B968D2
:10B2F00089B17A689200F7F748FAD7E90120531E1E
:10B300003AB10022013B591C026000F10400F9D15E
:10B31000B868FDF737FBC7E90156A36800244FEA78
:10B32000850AA3F1040C06EB0A00002233680CF135
:10B33000040CDCF800101B19144628BF01225B180E
:10B3400028BF012446F8043B86421444EDD1002C6A
:10B35000BCD042F210784FF000090FE0BD6805EB59
:10B360000A00036800221C1928BF012240F8044B80
:10B370000AF1040A35460124002AA7D07B686E1C16
:10B38000AB42EED846451ED8B342E7D20421304640
:10B39000FDF7E4FA0546B0B1B96889B17A68920060
:10B3A000F7F7F3F9D7E90120531E3AB1013B5A1CD4
:10B3B000C0F8009000F10400F8D1B868FDF7E2FA97
:10B3C000C7E90165CBE76FF00F00BDE8F087BE6805
:10B3D000A4E700BFF0B54B680D4685B0144606469D
:10B3E00051687BB1A86803F18042013A50F822709D
:10B3F00000EB820027B14FE050F8042D002A4BD11A
:10B40000013BF9D189B101F18040A768013857F8B3
:10B410002020002A40F0998007EB800003E050F8DC
:10B42000042D002A42D10139F9D100230122B4426E
:10B43000CDE9012303937FD0B54205D0294630469C
:10B44000FFF72AFA0746A8B901233360606880B184
:10B45000D4F808C000F18043013B5CF823200CEBDA
:10B46000830322B142E053F8042D002A3ED1013873
:10B47000F9D10027039860B1029A531E3AB1002215
:10B48000013B591C026000F10400F9D10398FDF75B
:10B4900079FA384605B0F0BD0029C6D001F18040E8
:10B4A000A768013857F82020002AB5D08B42BCD8B5
:10B4B0004BD3002BB9D0A86803F18041013950F873
:10B4C00021C057F821E08900E645084407EB010256
:10B4D000ABD33AD8014606E051F8047D52F8040D8A
:10B4E0008742A2D831D3013BF6D19EE700252B46F7
:10B4F000B16851F8046B0135F21A41F8042C5CF87C
:10B50000047B0C46BA422CBF4FF0000E4FF0010EE8
:10B51000D21B9E422CBF73460EF10103854241F8B7
:10B52000042CE6D30BB9A4E701232268D11A9A426E
:10B5300044F8041BF8D39CE7214601A8FFF7ACF9B7
:10B540000746002896D101AC76E76FF00907384628
:10B5500005B0F0BD2DE9F0410C681368054603FB0A
:10B5600004F3002B39DA4B6817460E46526883B154
:10B57000896803F18040013851F820C001EB800157
:10B58000BCF1000F03D02EE051F8040D58BB013B75
:10B59000FAD17AB102F18041D7F808C001395CF8DC
:10B5A000210078B90CEB810102E051F8040D28BBB1
:10B5B000013AFAD13A4631462846FFF70BFF48B127
:10B5C000BDE8F081324639462846FFF703FF0028E0
:10B5D000F6D164422C60BDE8F081FFF757FE0028E9
:10B5E000EED12C60F7E7002AE4D002F18041D7F8D1
:10B5F00008C001395CF821000028D3D09342D9D883
:10B60000E0D3002BD6D0B06803F18041013950F867
:10B6100021805CF821E08900F04508440CEB010230
:10B62000C8D8CFD3014606E051F804CD52F8040D36
:10B630008445BFD8C6D3013BF6D1BBE72DE9F04125
:10B640000C681368054603FB04F3002B64DD4B68AC
:10B6500017460E46526883B1896803F1804001386D
:10B6600051F820C001EB8001BCF1000F03D01FE0B6
:10B6700051F8040DE0B9013BFAD182B102F18041E9
:10B68000D7F808C001395CF8210000283BD10CEB49
:10B69000810102E051F8040DA8B9013AFAD13A4605
:10B6A00031462846FFF796FE00B92C60BDE8F081D0
:10B6B000002AF4D002F18041D7F808C001395CF8C3
:10B6C00021000028E3D09342E9D81CD3002BE6D018
:10B6D000B06803F18041013950F821805CF821E025
:10B6E0008900F04508440CEB0102D8D80BD3014681
:10B6F00006E051F804CD52F8040D8445CFD802D3AA
:10B70000013BF6D1CBE7324639462846FFF762FEC9
:10B710000028CBD16442C8E7FFF7B8FD0028C4D0A9
:10B72000BDE8F081002AACBF01234FF0FF33F0B534
:10B7300001260D6882EAE27C05FB03F785B0ACEBDD
:10B74000E27C002F0296CDE900C3CDF80CD006466E
:10B750002CDD4B680C4673B1A76803F180410139B9
:10B7600057F8210007EB810118B10EE051F8040DE4
:10B7700058B9013BFAD182B9214601AA3046FFF7F8
:10B78000F9F800B9356005B0F0BD002AF4D0012BFE
:10B79000F2D83B689C45EFD3EED9224601A930464A
:10B7A000FFF718FE0028EED16D42EBE701AAFFF784
:10B7B0006DFD0028E6D005B0F0BD00BF2DE9F047D3
:10B7C00006460023012086B08E42904600900390EA
:10B7D000CDE90133CDE9043300F0D1800F46464571
:10B7E00000F0D5807D6885B1BB6805F18042013AE3
:10B7F00053F8221003EB820329B1BAE053F8042D69
:10B80000002A40F0B680013DF8D1D8F80440002568
:10B81000002C3DD0D8F8083004F18042013A53F8AA
:10B82000221003EB820319B104E053F8042D0AB986
:10B83000013CFAD142F2107304EB0509994500F27C
:10B84000B080D6F804A0D14525D904214846FDF79B
:10B8500085F88246002800F0A480B16889B172683A
:10B860009200F6F792FFD6E90120531E3AB100226A
:10B87000013B591C026000F10400F9D1B068FDF7EA
:10B8800081F8C6E9019A4FEA8902D6F8089025E0C6
:10B890002546D6F804A0BAF1000F40F085800421B7
:10B8A0000120FDF75BF8814600287AD0B16889B1A4
:10B8B00072689200F6F769FFD6E90120531E3AB18B
:10B8C0005246013B591C026000F10400F9D1B068F6
:10B8D000FDF758F801230422C6E901390021484642
:10B8E000F6F780FF00210123B268116033609CB13C
:10B8F00004F1804909F1FF394FEA8909D8F8083085
:10B90000B26853F809304A44B9682846FEF714FC77
:10B91000013CA9F10409F1D100243A68D8F80030BB
:10B9200003FB02F33360059860B1049A531E3AB1E9
:10B930000022013B5D1C026000F10400F9D1059872
:10B94000FDF720F8002201230298CDE90332059289
:10B9500058B101994B1E31B1013B591C026000F1F5
:10B960000400F9D10298FDF70DF8204606B0BDE8B5
:10B97000F087D8F80440002C7FF44CAF5AE76846B3
:10B98000FEF78AFF04460028CDD16F4627E703A8BB
:10B990003146FEF781FF04460028C4D10DF10C08A2
:10B9A00020E76FF00F04BEE7D1466CE7012300B536
:10B9B00085B0009201AACDE90133CDF80CD0FFF794
:10B9C000FDFE05B05DF804FB2DE9F04F5E68A3B005
:10B9D00096B1D3F8088006F1804909F1FF3958F88B
:10B9E000295008EB890E6DB9F446374602E05CF841
:10B9F000044D3CB9013FFAD16FF00B06304623B03D
:10BA0000BDE8F08F1D68002DF6D014468A4600224E
:10BA100001219B4663680546109113911691199177
:10BA20001C91CDE91122CDE91422CDE91722CDE9EF
:10BA30001A22CDE91D22002B00F01A82A26803F120
:10BA40008041013952F8210002EB810220B17BE0F4
:10BA500052F8041D002977D1013BF9D158F829206B
:10BA6000002A77D1724603E052F8041D00296FD1F5
:10BA7000013EF9D110A82146FEF70EFF0646002828
:10BA800000F092800027129860B1119A531E3AB1CB
:10BA90000022013B5C1C026000F10400F9D1129805
:10BAA000FCF770FF002201231598CDE910321292A5
:10BAB00058B114994B1E31B1013B591C026000F181
:10BAC0000400F9D11598FCF75DFF002201231898B6
:10BAD000CDE91332159258B117994B1E31B1013B84
:10BAE0005D1C026000F10400F9D11898FCF74AFFD0
:10BAF000002201231B98CDE91632189258B11A99E9
:10BB00004B1E31B1013B5C1C026000F10400F9D115
:10BB10001B98FCF737FF002101231B91CDE9193158
:10BB2000002F3FF46BAF1D9A531E32B13A46013BD2
:10BB3000581C116002F10402F9D13846FCF722FFCB
:10BB4000304623B0BDE8F08F58F82920002A89D06C
:10BB50009E428FD39E4200F29081002B8AD0A16832
:10BB600003F18042013A51F8220058F82260920015
:10BB7000864211449044FFF47DAF00F27E810A4674
:10BB800008E052F8040D58F8041D88423FF672AFE1
:10BB9000C0F07381013BF4D110A82146FEF77CFE72
:10BBA000064600287FF46EAF13A85946FEF774FED0
:10BBB000064600287FF466AF42F2107201236768E0
:10BBC000139302379742109300F29381DDF85C8063
:10BBD00047451DD904213846FCF7C0FE81460028A0
:10BBE00000F08781189981B1179A9200F6F7CDFD80
:10BBF000DDE91720531E32B1013B5A1C066000F1EB
:10BC00000400F9D11898FCF7BDFEB846CDE91779C4
:10BC1000B8F1000F00F07181189E4FEA88020027EA
:10BC200030463946F6F7DEFD0122189B1F601A9B4D
:10BC30001692934240F2B28104210320FCF78EFE5B
:10BC40000746002800F055810323149ACDE91D30E2
:10BC50000392002A00F07181B2F10109159900F0F8
:10BC6000CF8151F82900002840F0C58102F18042BF
:10BC7000013A4B4601EB820204E052F8040D002821
:10BC800040F0AE81013BF8D12026086800224FF039
:10BC9000004102E00132202A04D001424FEA510162
:10BCA000F8D0B31A03F01F031F2B40F09F8100232D
:10BCB0000293119B13A80493013BA3EB0908019382
:10BCC0004FEA481319460593FFF7FEF80646002889
:10BCD0007FF4D9AE4FEA88080DE0189810A950F803
:10BCE000083013AA013340F808300846FFF7A6FCD5
:10BCF000002840F0798113A910A8FFF70BFA00285B
:10BD0000EBDA059913A8FFF795F9064600287FF4AA
:10BD1000BAAE6FF00303039ACDE908B502F180478C
:10BD2000049A03FB09F302F18042023A920015469D
:10BD300005934FEA89030393C9EBC963023FCDE939
:10BD40000630CDE90AA4B9000491019B4B4540F2AD
:10BD5000738103981299159A05F1040A125851F843
:10BD60000A300598934200EB0504189EC0F04C8100
:10BD70004FF0FF3333510126189A1E9F1359A5F136
:10BD8000040B334413514BE0DDF86C8092004046C5
:10BD90000021F6F727FD00221B9B1A601996B9F1C6
:10BDA000000F00F0F980159B049A9B581B9A039989
:10BDB0001360159A1B9B525819A95A60189B0DF1D4
:10BDC0003C081B591FAA08460F93CDE91F66CDF802
:10BDD0008480FFF7F3FC002840F006811D9A002ABA
:10BDE00000F0C280920000213846F6F7FBFC0023E9
:10BDF0003B60019B1C96012B1CA9129B00F0ED805F
:10BE000053F80B3019A83B60129B5B597B60129B67
:10BE100053F80A30BB60FFF77DF9002840F31C811E
:10BE2000189A1359013B13511A9A002AACD10421D4
:10BE30000120FCF793FD8046002800F040811B990B
:10BE400091B11A9A9200F6F7A0FCDDE91A100246A9
:10BE50004B1E39B10021013B1160591C02F1040253
:10BE6000F8D11B98FCF78EFD0422CDE91A688EE705
:10BE700058F82920002A3FF4F5AD55B36E68EEB9A5
:10BE800004210120FCF76AFD074690B3A96881B13F
:10BE90006A689200F6F779FCD5E90120531E32B1A9
:10BEA000013B591C066000F10400F9D1A868FCF7B9
:10BEB00069FD01230422C5E9013701E0AF68B20042
:10BEC00000213846F6F78EFC00210123AA68116094
:10BED0002B60BAF1000F07D021465046FEF7DCFC7C
:10BEE000064600287FF4CEAD0026304623B0BDE8DC
:10BEF000F08F00276FF00F06C5E504210120FCF745
:10BF00002DFD06460028F4D0189989B1179A9200A1
:10BF1000F6F73BFCDDE917305A1E3BB14346013AC8
:10BF2000571C036000F10400F9D11898FCF72AFDB2
:10BF300001230422CDE9173671E61F231946029327
:10BF400010A8FEF7C1FF064600287FF49CAD0299B9
:10BF500013A8FEF7B9FF064600287FF494AD149BA2
:10BF6000039303F1FF39A4E6042101200D92FCF7AD
:10BF7000F5FC0346002800F0A28047B10D9A39462F
:10BF80000C90F6F702FC3846FCF7FCFC0C9B1F46B5
:10BF90000422CDE91D6326E74B4607E70421022072
:10BFA000FCF7DCFC06460028A3D01B9989B11A9A3D
:10BFB0009200F6F7EAFBDDE91A1318464A1E31B182
:10BFC000013A501C1F6003F10403F9D11B98FCF7E0
:10BFD000D9FC0223CDE91A362EE65B5919A815E7DC
:10BFE0005B0103F1200651E606464CE5C3F11F0351
:10BFF00002931946A4E74FEA491303F1200645E6E8
:10C00000086820264B4641E64F5992B19C464FF0B6
:10C01000000B61465B464BEA0700F4F7E3F80023A8
:10C020004FF0FF328B4208BF824200D2104630519F
:10C03000A1E64FF0FF30FAE7DDE9076BDDE9095AC9
:10C040000B9C002D5FD016A92846FEF725FC002882
:10C0500053D006461E9F16E50125189B1FAA1B59A3
:10C0600013A919A80F93CDF88480CDE91F55FFF7C8
:10C07000A5FB0028B8D1069B019A03F10063013BA0
:10C0800013445E01314619A8FEF71EFF0028ABD10C
:10C0900010A919AA0846FFF7D1FA034658BB1FA9F1
:10C0A00010A80F93CDE91F55CDF88480FEF72EFB25
:10C0B000002807DB019B5D46013B019345E66FF0DD
:10C0C0000F06E0E413A919A8FEF7E6FB00288BD1C0
:10C0D000314619A8FEF7F8FE002885D110A919AA43
:10C0E0000846FFF737FA00287FF47EAF189A1359F5
:10C0F000013B1351DEE70646C5E4DBF80030226859
:10C1000003FB02F32B60BAF1000F05D0029910A8CF
:10C11000FEF790FF064608B11E9FB4E4236810A9FD
:10C1200050461093FEF7B8FB06460028F4D10124D0
:10C130000FAB1FA950460F96CDE91F442193FEF780
:10C14000E5FA0028E8D1CAF80040E5E72DE9F0411A
:10C150005368174683B1946803F18045013D54F854
:10C16000252004EB85042AB11AE154F8045D002D62
:10C1700040F01681013BF8D10A46064601463B468F
:10C180000020FFF721FC002851D16FF04048716872
:10C1900091B1B06801EB080350F823C000EB8302B3
:10C1A000BCF1000F56D114460B4603E054F8045D71
:10C1B000002D4FD1013BF9D16FF040443946304654
:10C1C000FEF7A8FF002842DB35683B6803FB05F358
:10C1D000002B2EDD73687A6883B1B168181951F8A5
:10C1E00020C001EB8001BCF1000F05D090E051F8B8
:10C1F000040D002840F08C80013BF8D18AB1D7F8BB
:10C2000008C011195CF82100002840F0BE800CEB3A
:10C21000810104E051F8040D002840F08380013AC8
:10C22000F8D13A4631463046FFF7D4F840B1BDE880
:10C23000F0813A4631463046FFF728F80028F6D11B
:10C24000356039463046FEF765FF0028BCDA00202D
:10C25000BDE8F0813468002CAEDA3B6803FB04F3E0
:10C26000002B23DABCF1000F29D1134602E053F86A
:10C27000042D22BB0139FAD17B6873B1D7F808C00D
:10C2800003EB08025CF822500CEB82021DB171E056
:10C2900052F8045D05BB013BFAD13A4631463046BF
:10C2A000FFF798F80028C2D1346070E73A4631466B
:10C2B0003046FEF7EBFF0028F6D0BDE8F0817B6842
:10C2C000002BEAD0D7F808C003EB08025CF8225034
:10C2D0000CEB8202002DDED09942DED84AD3002931
:10C2E000DBD001EB080350F823205CF823509B00BF
:10C2F000954218446344D0D307D93BE050F8045D1D
:10C3000053F8042D9542C8D834D30139F6D1C4E787
:10C31000002A86D0D7F808C011195CF8210000283F
:10C320003FF475AF93423FF67CAF2ED3002B3FF422
:10C3300078AFB1681A1951F822005CF822E0920037
:10C34000864511446244FFF46CAF08D91DE051F8F2
:10C3500004CD52F8040D84453FF663AF15D3013B7D
:10C36000F5D13A4631463046FFF734F800287FF4DD
:10C370005EAF65E7324639463046FFF72BF80028B6
:10C380007FF455AF6442346001E7324639463046A7
:10C39000FFF720F800287FF44AAF6D4235600DE7C3
:10C3A0003B68002BBFF6E8AE6FF009003FE700BF27
:10C3B0002DE9F0410F4601250021BB6886B00446F7
:10C3C000164600950395CDE90111CDE90411002B26
:10C3D00040D079684A1E11D053F82200002840F05E
:10C3E000C48001F18041013903EB810304E053F87B
:10C3F000041D002940F0B980013AF8D101253B68BD
:10C40000009304212846FCF7A9FA8046002800F092
:10C410003C81029989B1019A9200F6F7B6F9DDE9FB
:10C420000120531E3AB10022013B591C026000F169
:10C430000400F9D10298FCF7A5FACDE90158AD0046
:10C440002A4600214046F6F7CDF92A46B9680298F7
:10C45000F6F79BF9314603A8FEF71EFA07460028B7
:10C460005DD1019E002E00F00E810146029D043D2B
:10C47000002255F8040F04E0202A01F1010100F028
:10C48000818020FA02F313F0010302F10102F3D0DC
:10C49000049DB5B100208446059F043F002257F853
:10C4A000046F03E0202A00F1010071D026FA02F3A4
:10C4B00013F0010302F10102F4D0814228BF0146CA
:10C4C0000D4668462946FEF7B5FD074638BB2946A6
:10C4D00003A8FEF7AFFD074608BB01236FF04046F7
:10C4E00003930093019F7FB10298BA1950F822304C
:10C4F00000EB8202002B51D13B4603E052F8041DB1
:10C5000000294BD1013BF9D1294603A8FEF7DCFCF9
:10C51000074620B903A92046FEF7BEF90746029850
:10C5200060B1019A531E3AB10022013B5C1C0260CB
:10C5300000F10400F9D10298FCF724FA002201234B
:10C540000598CDE90032029258B104994B1E31B1E1
:10C55000013B591C026000F10400F9D10598FCF779
:10C5600011FA384606B0BDE8F08142F2107339681E
:10C57000551C9D42009100F28380002D7FF441AF55
:10C58000A8465DE70137BE427FF472AF19467FE7E8
:10C590000CF1010CAC4581D11D4692E7009B002BAC
:10C5A000B2D000218E46A0F1040C00225CF8040FEA
:10C5B00003E0202A01F1010142D020FA02F313F036
:10C5C000010302F10102F4D06846FEF733FD07468D
:10C5D0000028A4D1DDF810C0BCF1000F4ED00146F8
:10C5E0008646059F043F002257F8040F03E0202AE7
:10C5F00001F101012AD020FA02F313F0010302F144
:10C600000102F4D003A8FEF715FD0746002886D1E5
:10C6100003A96846FEF77EFD00281DDB03AA6946D4
:10C620006846FEF7D7FE074600287FF478AF012161
:10C630006846FEF7FFFC074600283FF453AF6EE75D
:10C640000EF1010EBE45B0D11946BDE70EF1010E47
:10C65000E645C8D11946D5E703A96A460846FEF75C
:10C66000B9FE074600287FF45AAF012103A8FEF760
:10C67000E1FC074600283FF435AF50E76146C1E7CB
:10C680006FF00F075AE7314602E702986FF00F0785
:10C6900046E700BF2DE9F043B1F5806FADF2044DE0
:10C6A00000F2A5800D4617460646694618462A46FA
:10C6B000B847074620B138460DF2044DBDE8F08377
:10C6C000002D00F08A809DF80030002B40F089801A
:10C6D0006B46044603E013F8012F002A4DD10134C4
:10C6E000A542F8D1D6F80480B8F1000F70D104212A
:10C6F0000120FCF733F98146002875D0B16889B173
:10C7000072689200F6F741F8D6E90120531E3AB15B
:10C710004246013B591C026000F10400F9D1B068A7
:10C72000FCF730F901230422C6E90139002148460B
:10C73000F6F758F800230122B168A5420B60326079
:10C74000B9D90DEB05022C1BB16823F003084FEAA1
:10C75000C30E12F801CD51F808000EF0180E0CFAB5
:10C760000EFC013340EA0C00A34241F80800EBD173
:10C7700038460DF2044DBDE8F0832A1B12F0030881
:10C7800018BF4FF0010842F2107308EB9208984569
:10C790002AD8736898452DD904214046FCF7DEF865
:10C7A000814608B3B16889B172689200F5F7EDFF70
:10C7B000D6E90120531E3AB10022013B591C026008
:10C7C00000F10400F9D1B068FCF7DCF8C6E9018992
:10C7D0004FEA8802D6F80890A8E7D6F804802C46DD
:10C7E00082E72A460446C9E76FF00F0763E76FF058
:10C7F000030760E7984677E72DE9F0435368A1B057
:10C800007BB1946803F1804C0CF1FF3C54F82C5040
:10C8100004EB8C041DB10AE054F8045D3DB9013B02
:10C82000FAD16FF00304204621B0BDE8F08313680D
:10C83000002BF6DD01240023064602A80594089487
:10C840000B940E9402941194149417941A940F4616
:10C850001546CDE90633CDE90933CDE90C33CDE9F1
:10C860000F33CDE90333CDE91233CDE91533CDE9EB
:10C870001833CDE91B33FFF79BFD0446A0B9039B9A
:10C8800083B1049903F18044013C51F8242001EB69
:10C8900084042AB1B5E054F8042D002A40F0B18098
:10C8A000013BF8D16FF00D04079860B1069A531E52
:10C8B0003AB10022013B591C026000F10400F9D199
:10C8C0000798FCF75FF8002201230A98CDE90532AA
:10C8D000079258B109994B1E31B1013B5F1C0260B0
:10C8E00000F10400F9D10A98FCF74CF8002201236A
:10C8F0000D98CDE908320A9258B10C994B1E31B10E
:10C90000013B5E1C026000F10400F9D10D98FCF7B8
:10C9100039F8002201231098CDE90B320D9258B15D
:10C920000F994B1E31B1013B5D1C026000F1040008
:10C93000F9D11098FCF726F8002201230498CDE9DC
:10C940000E32109258B103994B1E31B1013B591C64
:10C95000026000F10400F9D10498FCF713F80022FA
:10C9600001231398CDE90232049258B112994B1E5B
:10C9700031B1013B5F1C026000F10400F9D1139852
:10C98000FCF700F8002201231698CDE9113213922A
:10C9900058B115994B1E31B1013B5E1C026000F18C
:10C9A0000400F9D11698FBF7EDFF00220123199836
:10C9B000CDE91432169258B118994B1E31B1013B92
:10C9C0005D1C026000F10400F9D11998FBF7DAFF51
:10C9D000002201231C98CDE91732199200283FF458
:10C9E00022AF1B994B1E31B1013B591C026000F173
:10C9F0000400F9D11C98FBF7C5FF204621B0BDE823
:10CA0000F083012B029A6BD9002A7FF44BAF394691
:10CA100005A82A46FFF79AFB044600287FF444AF96
:10CA200008A805A9FDF738FF044600287FF43CAFAD
:10CA300011A82946FDF730FF044600287FF434AFE3
:10CA400014A82946FDF728FF044600287FF42CAFE0
:10CA50000BA80121FEF7ACF8044600287FF424AFB0
:10CA600001460EA8FEF7A4F8044600287FF41CAF88
:10CA7000014617A8FEF79CF8044600287FF414AF7F
:10CA80001AA80121FEF794F8044600287FF40CAFA1
:10CA900081464FF0010801AF0A9B1B68DA072CD4CE
:10CAA000012108A8FEF7C6FA044600287FF4FCAE70
:10CAB0000D9B1B68D80744D4109B1B68D90740D432
:10CAC00001210BA8FEF7B6FA044600287FF4ECAE6D
:10CAD00001210EA8FEF7AEFA04460028DCD0E3E6FA
:10CAE000002AFFF6DFAE0B68012B8DD8002B8ED10C
:10CAF0005242002A7FF4D6AE89E7169B1B68D807FE
:10CB000043D4012114A8FEF795FA044600287FF4C7
:10CB1000CBAE199B1B68DB0725D41C9B1B68DC076D
:10CB200021D4012117A8FEF785FA044600287FF4D6
:10CB3000BBAE01211AA8FEF77DFA04460028DCD01E
:10CB4000B2E60BA911AA0846FEF704FD0446002828
:10CB50007FF4AAAE0EA905AA0846FEF76FFD0446AB
:10CB60000028ADD0A0E617A911AA0846FEF7F2FCEE
:10CB7000044600287FF498AE1AA905AA0846FEF7D5
:10CB80005DFD04460028CCD08EE614A908A8FEF767
:10CB9000C1FA00283DDB08A914AA0846FEF74EFD9D
:10CBA000044600287FF480AE0BA917AA0846FEF7BA
:10CBB00045FD044600287FF477AE0EA91AAA084660
:10CBC000FEF73CFD044600287FF46EAE1DA908A8C0
:10CBD000CDF80490CDE91D881F97FDF797FD00283B
:10CBE0007FF45AAF80464FF001091DA917A8CDF870
:10CBF0000480CDE91D991F97FDF788FD002823DAF1
:10CC000017A92A460846FEF7A5FC04460028ECD0E2
:10CC10004AE614A908AA0846FEF710FD04460028B3
:10CC20007FF442AE17A90BAA0846FEF707FD04469B
:10CC300000287FF439AE1AA90EAA0846FEF7FEFCBA
:10CC400004460028C2D02FE6294617A8FEF762FA4C
:10CC5000002808DB17A92A460846FEF7EFFC044621
:10CC60000028F1D020E617A93046FDF715FE04464E
:10CC70001AE600BF2DE9F04FB2F5C07FADF5497D52
:10CC800000F2198192460C464FF4D0720021814681
:10CC900060A8F5F7A7FD1AA802F01CFB00203023BE
:10CCA00066AD4FEA1A22ADF890018DF89221214627
:10CCB000524628468DF897318DF893A106AEF5F7C8
:10CCC00064FD8022334605F80A200EAF991B03F855
:10CCD000011B9F42FAD14FF4807231461AA802F02C
:10CCE00005FB8346002840F0C88001900AF1190A2C
:10CCF00002AC102200212046F5F774FDD04664AD49
:10CD0000227815F8103C94F801C015F80F1CA07893
:10CD1000534015F80E2C8CEA010C5040E17815F8C0
:10CD20000D2C94F804E0514015F80C2C23708EEA79
:10CD3000020215F80B3C94F805E084F801C08EEA75
:10CD4000030315F80ACC94F806E0A0708EEA0C0CE8
:10CD500015F8090C94F807E0E1708EEA000015F868
:10CD6000081C94F808E022718EEA010115F8072CDE
:10CD700094F809E063718EEA0202A37A15F806ECD2
:10CD800084F806C083EA0E03E07121726272A37216
:10CD9000E17A15F8053C94F80CC0607B4B4015F81F
:10CDA000042C15F8031C8CEA0202414094F80EC0D2
:10CDB00015F8020C94F80FE08CEA000015F801CC8D
:10CDC000E3728EEA0C0C22736173A0732346224631
:10CDD00001211AA884F80FC003F03EFAB8F1100F31
:10CDE000834694BFA8EB0808A8F11008002845D195
:10CDF0001035B8F1000F83D1019D1022214678191A
:10CE0000F5F7C3FC9DF8833105F110020133302A98
:10CE100001928DF883317FF46CAF4FF48072394604
:10CE20001AA802F063FA834640BB4D4609F1300868
:10CE300016AB1A4601211AA803F00EFA8346E8B988
:10CE40001022284616A91544F5F79FFC4545EFD159
:10CE50001AA802F045FA60A84FF4D07102F054F914
:10CE60003846302102F050F93046202102F04CF9CA
:10CE70002046102102F048F918E002AC1AA802F08E
:10CE80002FFA60A84FF4D07102F03EF938463021F5
:10CE900002F03AF93046202102F036F920461021FE
:10CEA00002F032F94846302102F02EF958460DF5CD
:10CEB000497DBDE8F08F6FF0370BF7E74FF4A072B4
:10CEC0000021F5F78FBC00BF58B110B504462030E3
:10CED00002F006FA2046BDE810404FF4A07102F0BF
:10CEE00013B97047F0B58369EDB0B3F5C07F00F2B8
:10CEF000E180C3F5C0739342C0F0DC800446154660
:10CF00000E464FF4C07200210CA8F5F76BFC0CA97B
:10CF1000D4F83831A269D4F83C019847002840F091
:10CF2000CC80A76906B14DB90CA93A460846FFF76F
:10CF3000A1FE054688B128466DB0F0BD0CAB2A466F
:10CF4000D8193146F5F721FC2F440CA93A4608467A
:10CF5000FFF790FE05460028EDD1684630222946AD
:10CF6000F5F740FC2E4604F12007E27B0DEB0603AB
:10CF70000132D2B2E273002A4DD1A27B0132D2B289
:10CF8000A273002A47D1627B0132D2B26273002AB7
:10CF900041D1227B0132D2B22273002A3BD1E27A04
:10CFA0000132D2B2E272002A35D1A27A0132D2B273
:10CFB000A272002A2FD1627A0132D2B2627252BBBF
:10CFC000227A0132D2B222722ABBE2790132D2B283
:10CFD000E27102BBA2790132D2B2A271DAB96279EE
:10CFE0000132D2B26271B2B922790132D2B2227167
:10CFF0008AB9E2780132D2B2E27062B9A278013223
:10D00000D2B2A2703AB962780132D2B2627012B969
:10D0100022780132227022460121384603F01CF9A1
:10D020000546002887D11036302E9ED101990C9BE1
:10D0300000980D9A58404A400E9B02990090594022
:10D0400003980F9B01924340109A0498029150401C
:10D050000599119A03935140129B069A04905A40E5
:10D060000798139B059158400899149B06925940C4
:10D07000099A159B07905A400A98169B08914340BD
:10D08000CDE909230B9A179B3846534069464FF464
:10D0900080720B9302F02AF9054600287FF44BAF0B
:10D0A000102208A92046F5F770FB012328462361CA
:10D0B0006DB0F0BD6FF037053DE76FF033053AE72F
:10D0C0002DE9F04104461646202288B0A5180F46E7
:10D0D000684600219846F5F785FB284602F0FAF8E5
:10D0E000202242F21073C4F83871C4E9062328469E
:10D0F000C4F83C6169464FF4807202F0F7F820B939
:10D10000414620460E9AFFF7EDFE08B0BDE8F081DB
:10D110002DE9F04FB2F5806FF9B000F22682044697
:10D1200015460F46302268460021F5F75BFB226961
:10D13000E3699A4201DC636913B3A369B3F5C07F65
:10D1400000F216820DF1600A4FF4C07200215046C1
:10D15000F5F748FB5146D4F83831A269D4F83C01C0
:10D1600098476FF0330938B9A26951465046FFF726
:10D1700081FD8146002877D0484679B0BDE8F08F20
:10D1800004F12008002D00F02B810CAE0EE0102DD4
:10D19000A94628BF4FF01009384631464A46F5F7F0
:10D1A000F4FAB5EB09054F4400F01A81E37B013333
:10D1B000DBB2E373002B4DD1A37B0133DBB2A3734E
:10D1C000002B47D1637B0133DBB26373002B41D16A
:10D1D000237B0133DBB22373002B3BD1E37A013392
:10D1E000DBB2E372002B35D1A37A0133DBB2A37239
:10D1F000002B2FD1637A0133DBB2637253BB237AE6
:10D200000133DBB223722BBBE3790133DBB2E37171
:10D2100003BBA3790133DBB2A371DBB963790133BB
:10D22000DBB26371B3B923790133DBB223718BB9FC
:10D23000E3780133DBB2E37063B9A3780133DBB287
:10D24000A3703BB963780133DBB2637013B9237801
:10D2500001332370334622460121404602F0FCFF91
:10D260008146002893D087E70CAE304630224946ED
:10D27000F5F7B8FACB4604F12008E27B06EB0B0386
:10D280000132D2B2E273002A4DD1A27B0132D2B276
:10D29000A273002A47D1627B0132D2B26273002AA4
:10D2A00041D1227B0132D2B22273002A3BD1E27AF1
:10D2B0000132D2B2E272002A35D1A27A0132D2B260
:10D2C000A272002A2FD1627A0132D2B2627252BBAC
:10D2D000227A0132D2B222722ABBE2790132D2B270
:10D2E000E27102BBA2790132D2B2A271DAB96279DB
:10D2F0000132D2B26271B2B922790132D2B2227154
:10D300008AB9E2780132D2B2E27062B9A27801320F
:10D31000D2B2A2703AB962780132D2B2627012B956
:10D3200022780132227022460121404602F094FF09
:10D33000814600287FF420AF0BF1100BBBF1300FBA
:10D340009BD17068DAF800303168DAF8042059406F
:10D350004240DAF80830B068316083EA0001DAF858
:10D360000C30F068726058403269DAF81030B16001
:10D370005340DAF814107269F0604A40B069DAF884
:10D38000181033614840DAF81C30F16972614B4083
:10D39000326ADAF82010B0615140706ADAF824205D
:10D3A000F3615040DAF82830B26A31625340C6E97E
:10D3B0000903F26ADAF82C303146534040464FF404
:10D3C0008072F36201F092FF814600287FF4D4AEB0
:10D3D000102214A92046F5F7D8F901232361D1E6DC
:10D3E0000DF1600A504630220021F5F7FBF90025C7
:10D3F000E27B0AEB05030132D2B2E273002A4DD17F
:10D40000A27B0132D2B2A273002A47D1627B0132E1
:10D41000D2B26273002A41D1227B0132D2B222738E
:10D42000002A3BD1E27A0132D2B2E272002A35D12F
:10D43000A27A0132D2B2A272002A2FD1627A0132CC
:10D44000D2B2627252BB227A0132D2B222722ABBAB
:10D45000E2790132D2B2E27102BBA2790132D2B2D8
:10D46000A271DAB962790132D2B26271B2B92279AB
:10D470000132D2B222718AB9E2780132D2B2E270BC
:10D4800062B9A2780132D2B2A2703AB9627801329E
:10D49000D2B2627012B92278013222702246012182
:10D4A000404602F0D9FE814600287FF465AE103573
:10D4B000302D9DD1DAE90012009B0198594042407D
:10D4C000DAF808300298CAF8001083EA0001DAF8A6
:10D4D0000C300398CAF804205840049ADAF8103047
:10D4E000CAF8081053400599DAF81420CAF80C005D
:10D4F0004A400698DAF81810CAF810304840079BDE
:10D50000DAF81C10CAF814204B40DAF820200899E9
:10D51000CAF818005140DAF82400099ACAF81C30F9
:10D520005040DAF828300A9ACAF820105340CAE965
:10D5300009030B9ADAF82C304046534051464FF419
:10D540008072CAF82C3001F0D1FE814600287FF4A9
:10D5500013AE102220A92046F5F717F94846236993
:10D560000133236179B0BDE8F08F6FF0350903E630
:10D570006FF0370900E600BF70B54B6E0446002B14
:10D580003DD003680D46002B2FDB2046FDF75AFBEC
:10D59000AB6DB0EB430F2DD86B6E20469847064617
:10D5A00008BB04350AE000212046FDF71BFEA0B1B0
:10D5B0002A4621462046FDF7CDFFE8B92368002B17
:10D5C000F1DB29462046FDF7A5FD00280BDB2A46A6
:10D5D00021462046FDF7FEFE70B929462046FDF79C
:10D5E00099FD0028F3DA304670BD0021FDF7FAFD01
:10D5F0000028CAD0054EF6E70646304670BD0A1D23
:10D60000BDE870400146FEF7A1BD00BF80B0FFFF3E
:10D610002DE9F04306468DB0684688461546FDF76D
:10D62000B7F803A8FDF7B4F806A8FDF7B1F809A804
:10D63000FDF7AEF8B369002B00F0B2802A46294608
:10D6400003A8FEF7BBF8044678B16846FDF7A8F8D2
:10D6500003A8FDF7A5F806A8FDF7A2F809A8FDF7AD
:10D660009FF820460DB0BDE8F083314603A8FFF7D0
:10D6700083FF04460028E8D1032203A96846FEF789
:10D6800095F904460028E0D1371D07E03A4669467F
:10D690006846FDF79FFE04460028D6D13946684605
:10D6A000FDF738FD0028F1DA06F11009484600219F
:10D6B000FDF798FD002840F0E28005F10C094A468C
:10D6C000494606A8FEF77AF804460028BDD131463F
:10D6D00006A8FFF751FF04460028B6D1012106A88D
:10D6E000FDF7F2FB044640B1AFE706A93A4608460B
:10D6F000FDF770FE04460028A7D1394606A8FDF7BD
:10D7000009FD0028F1DA06AA294603A8FEF756F813
:10D710000446002899D1314603A8FFF72DFF04469F
:10D72000002892D1012103A8FDF7CEFB044640B1A9
:10D730008BE703A93A460846FDF74CFE044600284D
:10D7400083D1394603A8FDF7E5FC0028F1DA06AAE3
:10D75000114609A8FEF732F8044600287FF475AF99
:10D76000314609A8FFF708FF044600287FF46DAF93
:10D77000012109A8FDF7A8FB044600287FF465AF46
:10D78000394609A8FDF7C6FC0028C0F2C58009A9E2
:10D790003A460846FDF71EFE04460028F0D054E73E
:10D7A00005F11802114603A8FEF708F80446002800
:10D7B0007FF44BAF314603A8FFF7DEFE0446002896
:10D7C0007FF443AF03AA294606A8FDF7C3FE04462B
:10D7D00000287FF43AAF371D08E006A93A4608460C
:10D7E000FDF7F8FD044600287FF42FAF394606A860
:10D7F000FDF790FC0028F0DA03AA294609A8FDF7F6
:10D800001DFF044670B120E7002109A8FDF7EAFCDE
:10D8100058B109A93A460846FDF79CFE044600287F
:10D820007FF413AF099B002BEEDB09AA06A903A81E
:10D83000FDF7C4FF044600287FF407AF314603A874
:10D84000FFF79AFE044600287FF4FFAE032203A9E7
:10D850006846FEF7ABF8044600287FF4F6AE39467A
:10D860006846FDF757FC0028FFF627AF3A466946A1
:10D870006846FDF7AFFD04460028F0D0E5E605F167
:10D880001802114603A8FDF799FF044600287FF40B
:10D89000DCAE314603A8FFF76FFE044600287FF494
:10D8A000D4AE03AA114606A8FDF788FF0446002857
:10D8B0007FF4CBAE314606A8FFF75EFE0446002893
:10D8C0007FF4C3AE4A4606A903A8FDF777FF0446D6
:10D8D00000287FF4BAAE314603A8FFF74DFE044698
:10D8E00000287FF4B2AE03AA69466846FDF732FE0F
:10D8F000044600287FF4A9AE39466846FDF70AFCC5
:10D900000028FFF6DAAE3A4669466846FDF762FD42
:10D9100004460028F0D098E66A46694606A8FDF756
:10D920004DFF044600287FF490AE314606A8FFF76D
:10D9300023FE044600287FF488AE06A903AA084601
:10D94000FDF77CFE044600287FF47FAE069B002B8B
:10D950000DDA002106A8FDF745FC40B106A93A46BC
:10D960000846FDF7F7FD04460028EFD06DE606A94E
:10D9700003AA0846FDF762FE044600287FF465AE60
:10D98000069B002B0DDA002106A8FDF72BFC40B109
:10D9900006A93A460846FDF7DDFD04460028EFD00B
:10D9A00053E603A906AA0846FDF748FE04460028E8
:10D9B0007FF44BAE039B002B0DDA002103A8FDF78B
:10D9C00011FC40B103A93A460846FDF7C3FD0446E1
:10D9D0000028EFD039E603A96A460846FDF7EEFEB7
:10D9E000044600287FF431AE314603A8FFF7C4FD9A
:10D9F000044600287FF429AE03A909AA0846FDF7CA
:10DA00001DFE044600287FF420AE039B002B0DDA98
:10DA1000002103A8FDF7E6FB40B103A93A460846FA
:10DA2000FDF798FD04460028EFD00EE605F1180238
:10DA3000494609A8FDF7C2FE044600287FF405AE5A
:10DA4000314609A8FFF798FD044600287FF4FDAD94
:10DA5000012109A8FDF738FA044600287FF4F5AD46
:10DA6000394609A8FDF756FB002808DB09A93A4604
:10DA70000846FDF7AFFC04460028F1D0E5E506A90D
:10DA80004046FCF709FF044600287FF4DEAD03A9F9
:10DA900008F10C00FCF700FF044600287FF4D5AD28
:10DAA00008F1180009A9FCF7F7FE0446CDE500BF10
:10DAB000F0B501F1180587B00E460746002128464B
:10DAC000FDF790FB18B90446204607B0F0BD684644
:10DAD000FCF75EFE03A8FCF75BFE68463A1D29468C
:10DAE000FEF78AFE044640B16846FCF759FE03A8DB
:10DAF000FCF756FE204607B0F0BD6A46694603A80B
:10DB0000FDF75CFE04460028EED1394603A8FFF776
:10DB100033FD04460028E7D103AA31463046FDF71D
:10DB20004DFE04460028DFD139463046FFF724FD7C
:10DB300004460028D8D10C363146304603AAFDF7FA
:10DB40003DFE04460028CFD139463046FFF714FD8C
:10DB500004460028C8D16A4631463046FDF72EFEFD
:10DB600004460028C0D139463046FFF705FD04467B
:10DB70000028B9D128460121FDF71AF80446B3E779
:10DB80002DE9F04F82468BB08B4610460C2116468D
:10DB9000FAF7E4FE002800F0FE80804601A8FCF7BA
:10DBA000F7FD04A8FCF7F4FD07A8FCF7F1FDDBF88E
:10DBB000001040461831FCF76FFE044660BB012E92
:10DBC00046D9D946012708F10C0508E028465146F8
:10DBD000FFF7D2FC0C35044668B9BE4238D059F87C
:10DBE000042FA5F10C0118322846FDF7E7FD013797
:10DBF00004460028EAD001A8FCF7D2FD04A8FCF7EF
:10DC0000CFFD07A8FCF7CCFD10E001A904A8FCF7A4
:10DC100043FE0446002853D001A8FCF7C1FD04A828
:10DC2000FCF7BEFD07A8FCF7BBFD56B1454606EB69
:10DC3000460608EB860628460C35FCF7B1FDB542D2
:10DC4000F9D14046FAF79EFE20460BB0BDE8F08FB2
:10DC500006EB4605AD00A5F10C0141440AF10402B2
:10DC600001A8FEF7C9FD04460028D5D106F180437E
:10DC7000183D013B45440BEB830B771E002FC4D0AE
:10DC80002A4601A904A8FDF799FD04460028C3D13E
:10DC9000514604A8FFF770FC04460028BCD1DBF80D
:10DCA000002001A918320846FDF788FD0446002827
:10DCB000B2D1514601A8FFF75FFC04460028ABD162
:10DCC00004AA114607A8FDF779FD04460028A3D150
:10DCD000514607A8FFF750FC044600289CD1DBF80A
:10DCE000001007AA0846FDF769FD0446002893D1F5
:10DCF0005146DBF80000FFF73FFC044600288BD1BB
:10DD0000DBF8001007AA0C310846FDF757FD044662
:10DD1000002881D1DBF8000051460C30FFF72CFCC5
:10DD2000044600287FF478AFDBF8001004AA0C3119
:10DD30000846FDF743FD044600287FF46DAFDBF88D
:10DD4000000051460C30FFF717FC044600287FF412
:10DD500063AFDAF80810DBF80000FCF73BFD04467F
:10DD600000287FF459AFDBF80000DAF808100C3017
:10DD7000FCF730FD044600287FF44EAFDBF80000CE
:10DD80000C3D1830ABF1040BFCF70AFD002F3FF4FB
:10DD900043AF013F72E7014C56E700BF80B2FFFF7F
:10DDA000B8B110B504467C220021F4F71BFD04F144
:10DDB0007C00FCF7EDFC04F18800FCF7E9FC04F1C1
:10DDC0009400FCF7E5FC04F1A000BDE81040FCF76E
:10DDD000DFBC7047002848D070B5036E0446012BA5
:10DDE00023D1606FC8B1A26FAAB1002606EBC603AB
:10DDF00010EB830535D02846FCF7D2FC05F10C006A
:10DE0000FCF7CEFC05F11800FCF7CAFCA26F013646
:10DE10009642606FEAD3FAF7B5FD002204F17C0365
:10DE2000227001349C42FBD170BD0430FCF7B8FC79
:10DE300004F11000FCF7B4FC04F11C00FCF7B0FC8A
:10DE400004F12800FCF7ACFC04F13400FCF7A8FC5A
:10DE500004F14000FCF7A4FC04F14C00FCF7A0FC2A
:10DE6000BFE701369642C1D3D5E77047A8B110B5D8
:10DE70000446FFF7AFFF04F17C00FCF791FC04F1CE
:10DE80008800FCF78DFC04F19400FCF789FC04F198
:10DE9000A000BDE81040FCF783BC704710B501211D
:10DEA0000446FCF785FE00B110BD012104F10C0011
:10DEB000FCF77EFE0028F7D1014604F11800BDE80A
:10DEC0001040FCF775BE00BF2DE9F04702F11805C0
:10DED00096B0814688462846002117461E46FDF723
:10DEE00081F9002848D0336A8BB106F11804204626
:10DEF0000021FDF777F9002800F0D780336A33B1AD
:10DF000020460121FDF76EF9002840F0E78001A8C6
:10DF1000FCF73EFC04A8FCF73BFC07A8FCF738FC28
:10DF20000AA8FCF735FC0DA8FCF732FC10A8FCF79A
:10DF30002FFC13A8FCF72CFC2A46294601A8FDF764
:10DF40003DFC044680B301A8FCF72AFC04A8FCF7BA
:10DF500027FC07A8FCF724FC0AA8FCF721FC0DA865
:10DF6000FCF71EFC10A8FCF71BFC13A8FCF718FC20
:10DF7000204616B0BDE8F08731464046FCF78CFCE1
:10DF800004460028F4D106F10C0108F10C00FCF75E
:10DF900083FC04460028EBD106F1180108F11800B3
:10DFA000FCF77AFC0446E3E7494601A8FFF7E4FAE8
:10DFB00004460028C7D12A4601A904A8FDF7FEFBA4
:10DFC00004460028BFD1494604A8FFF7D5FA044605
:10DFD0000028B8D101A932460846FDF7EFFB0446F8
:10DFE0000028B0D1494601A8FFF7C6FA0446002828
:10DFF000A9D104A906F10C020846FDF7DFFB04468F
:10E000000028A0D1494604A8FFF7B6FA0446002824
:10E0100099D101A93A460846FDF710FB04460028AD
:10E0200091D109F104060CE0002101A8FDF7DAF80E
:10E0300050B101A932460846FDF78CFA0446002883
:10E0400081D1019B002BEFDB04A907F10C063246BE
:10E050000846FDF7F3FA044600287FF474AF09F18F
:10E06000040A0DE0002104A8FDF7BCF858B104A98A
:10E0700052460846FDF76EFA044600287FF463AF67
:10E08000049B002BEEDB002101A8FDF7ABF8014655
:10E0900030BB04A8FDF7A6F800287FD13A464146D8
:10E0A0004846FFF7B5FA04464DE739464046FCF7C7
:10E0B000F3FB044600287FF45BAF07F10C0108F185
:10E0C0000C00FCF7E9FB044600287FF451AF294619
:10E0D00008F11800FCF7E0FB044649E78B4C47E7E2
:10E0E000294601AA13A8FDF769FB044600287FF41E
:10E0F0002AAF494613A8FFF73FFA044600287FF4E9
:10E1000022AF01AA114607A8FDF758FB04460028D4
:10E110007FF419AF494607A8FFF72EFA04460028F6
:10E120007FF411AF01AA07A90AA8FDF747FB04462F
:10E1300000287FF408AF49460AA8FFF71DFA0446F5
:10E1400000287FF400AF07A93A460846FDF736FBE2
:10E15000044600287FF4F7AE494607A8FFF70CFAFB
:10E16000044600287FF4EFAE022207A901A8FDF7BC
:10E170001DFC044600287FF4E6AE09F1040529469B
:10E1800001A8FCF7C7FF00280DDB01A92A460846B5
:10E19000FDF720F904460028F1D0D4E64046FFF709
:10E1A0007DFE0446CFE604AA11460DA8FDF706FB46
:10E1B000044600287FF4C7AE49460DA8FFF7DCF9F6
:10E1C000044600287FF4BFAE0DA901AA0846FDF75A
:10E1D00035FA044600287FF4B6AE0D9B002B0DDA0D
:10E1E00000210DA8FCF7FEFF40B10DA92A46084604
:10E1F000FDF7B0F904460028EFD0A4E60DA90AAA5D
:10E200000846FDF71BFA044600287FF49CAE0D9BE0
:10E21000002B0DDA00210DA8FCF7E4FF40B10DA999
:10E220002A460846FDF796F904460028EFD08AE60C
:10E2300007A90DAA0846FDF701FA044600287FF455
:10E2400082AE079B002B0DDA002107A8FCF7CAFF5E
:10E2500040B107A92A460846FDF77CF90446002884
:10E26000EFD070E607A904AA0846FDF7A7FA04460E
:10E2700000287FF468AE494607A8FFF77DF90446F9
:10E2800000287FF460AE0AA932460846FDF796FAE8
:10E29000044600287FF457AE49460AA8FFF76CF9F8
:10E2A000044600287FF44FAE0AAA07A910A8FDF77C
:10E2B000C5F9044600287FF446AE109B002B0DDA0A
:10E2C000002110A8FCF78EFF40B110A92A4608468D
:10E2D000FDF740F904460028EFD034E60DA940468A
:10E2E000FCF7DAFA044600287FF42DAE10A908F1F5
:10E2F0000C00FCF7D1FA044600287FF424AE08F1A4
:10E30000180013A9FCF7C8FA04461CE680B0FFFF0A
:10E310002DE9F04F0546984605F14C031C46E5B043
:10E320000DA8049117460893FCF732FA10A8FCF7E1
:10E330002FFA20460021FCF775FC0128079040F0D9
:10E34000C981EB6D08F10C09B3F5C07F2CBF052620
:10E350000426484605F134012CBF4FF0060A4FF061
:10E36000050AB346FCF7D6FE002872D0EC6DA64233
:10E3700045D201230BF1FF32934002933444DBB2C8
:10E38000013C03930023B4FBF6F402980692059334
:10E390002421FAF7E3FA0190002840D04146FCF727
:10E3A0007BFADDF804A08346002800F08680059BF8
:10E3B000002B7BD10025019C039E013554B12046E2
:10E3C000FCF7EEF904F10C00FCF7EAF904F118008F
:10E3D000FCF7E6F9EBB29E4204F12404EDD8019873
:10E3E000FAF7D0FA0DA8FCF7DBF910A8FCF7D8F97A
:10E3F000BBF1000F1BD1584665B0BDE8F08F022677
:10E400000023012230462421CDE90266CDE9053200
:10E41000FAF7A4FA0134640801900028BED10DA8CF
:10E42000FCF7BEF910A8FCF7BBF9DFF844B6049C72
:10E43000002CE0D02046FCF7B3F904F10C00FCF707
:10E44000AFF904F11800FCF7ABF9584665B0BDE828
:10E45000F08F05F128014046FCF75CFE002885D1CD
:10E46000EB6D9A45C0F0F48202265C1C0123CDE9D5
:10E470000266640806936B6F0193002B00F0EA803C
:10E4800000213846FCF7CEFB394680460DA8FCF744
:10E4900003FA834650B93A46089910A8FDF7CEF81A
:10E4A0008346002836D0079B002B83D00DA8FCF7AD
:10E4B00077F910A8FCF774F9B9E749460AF10C009E
:10E4C000FCF7EAF9834600287FF471AF019B08F15D
:10E4D000180103F11800FCF7DFF9834600287FF4E8
:10E4E00066AF2A464FF001095146254682464C4602
:10E4F000904609960A97069E019F04EBC40407EB19
:10E5000084042046FCF7C8F9002800F0A780834661
:10E51000059B4DE718F1FF3318BF012310A91A46D8
:10E520000DA80293FCF7E6FA83460028BBD122A887
:10E53000621C5946F4F756F9D4B30DF18809D84650
:10E54000CB46C246002751460DA8FCF76BFB9BF853
:10E550000030B84001370343B742A2448BF8003083
:10E56000F1D108F10108A0450BF1010BE9D100231D
:10E570004FF0010C9DF8881019F8016F0CF1010C97
:10E5800086EA0302D04300F0010000FB01F752B21B
:10E590007FB2334002EA07067A4041EAC0103343B3
:10E5A000D1B2E04509F8010CDBB289F80010E3D2E2
:10E5B000002619A8FCF7ECF81CA8FCF7E9F81FA83E
:10E5C000FCF7E6F822AB13F8049023440693049B6F
:10E5D00032469B46019F05953D46039FC9F345087A
:10E5E00003F10C0AA2EB0804B4FA84F46409294686
:10E5F00022465846FCF77EFA013605F10C01243517
:10E6000000286AD122465046FCF774FAF2B200287C
:10E6100063D1BA42E6D3059D16A82B1D1C4608936C
:10E62000FCF7B6F816A821465246FDF707F88346D0
:10E63000002800F0C38016A8FCF7B2F819A8FCF770
:10E64000AFF81CA8FCF7ACF81FA8FCF7A9F8079BCB
:10E650000593ACE601230298059399E64FEA590B1E
:10E660000BEBCB0B07EB8B0B0BF10C0104F10C004C
:10E67000FCF712F900287FF44AAF0BF1180104F1FE
:10E680001800FCF709F900287FF441AF65B1834613
:10E69000224621464046FEF7BBFF0BF1010B002846
:10E6A0007FF435AFAB45F3D14FEA49095FFA89F9F9
:10E6B0000AF1010322AA42F82A405FFA83FA39FAE2
:10E6C00006F34C460BD14FEA590101EBC10107EBB0
:10E6D000810112E7DFF89CB38DE68346AEE7524630
:10E6E000012A2C46099E45460A9F61D922A9404627
:10E6F000FFF746FA8346BBF1000F7FF458AE0123C3
:10E70000019ADA46243A0B9793461F46CDE909460B
:10E7100003B303EBC3034FEA8308019BA8F124046E
:10E720001C4403EB080905E022AAA34542F82A602D
:10E730009A460FD008EB04064B462246314628463F
:10E74000FFF7C2FB0AF10103243CDBB20028EBD047
:10E750008346DDE67B00069ADFB237FA02F23B46DB
:10E76000D6D0BAF1010FDDE909460B9F40F267816F
:10E77000524622A92846FFF703FA8346059BBBF1C0
:10E78000000F7FF415AE23B1019B6B67029BAB6753
:10E7900076E619463846FCF745FA394680460DA814
:10E7A000FCF77AF8834600287FF404AE079072E6FF
:10E7B00022992846FFF77CF983469CE7014650469C
:10E7C000FCF710FD021C18BF012216A902EAD9129B
:10E7D0005046FCF78FF9834616A8FBF7E1FFBBF123
:10E7E000000F7FF42BAF049B012103F11804204696
:10E7F000FCF7DEF9834600287FF420AF6E9B002BE8
:10E8000000F082800C26AB6D13A80733DF08FBF7FE
:10E81000BFFF16A8FBF7BCFFDDF820806F9B6E9A48
:10E82000394613A8FDF736FF06E0012113A8FCF7CF
:10E8300001FC002840F0C880414613A8FCF76AFCA0
:10E840000028F2DA013E00F00081012113A8FCF754
:10E85000C9FC0028E2DD13AA21462046FCF7AEFFE2
:10E86000834630B113A8FBF79BFF16A8FBF798FF70
:10E87000E4E620462946FEF77FFE83460028F1D1D4
:10E8800013AA114616A8FCF799FF83460028E9D180
:10E89000294616A8FEF770FE83460028E2D10498A8
:10E8A00016AA0146FCF78AFF83460028DAD12946DA
:10E8B0000498FEF761FE83460028D3D116A913AA57
:10E8C0000846FCF77BFF83460028CBD1294616A8D3
:10E8D000FEF752FE83460028C4D116AA5146504680
:10E8E000FCF76CFF83460028BCD129465046FEF752
:10E8F00043FE834613A8FBF753FF16A8FBF750FF10
:10E90000BBF1000F7FF49AAEAB46DDF81880DDF85E
:10E910000C90CDF818A0DDF810A022AB434555D0DF
:10E92000524651465846FEF773FE0246002849D12A
:10E930000646044618F8013D019D0593C3F34507BB
:10E94000E41BB4FA84F464092946224619A8FCF7AA
:10E95000D1F8013605F10C01243500287FF4BDAE55
:10E9600022461CA8FCF7C6F8F4B200287FF4B5AE26
:10E97000A145E5D816A8FBF70BFF1CAA089916A815
:10E98000FCF75CFE08B1834655E601461CA8FCF77F
:10E9900029FC021C18BF0122059B16A902EAD3120A
:10E9A0001CA8FCF7A7F8059016A8FBF7F9FE059A36
:10E9B00042B9524619AB51465846FFF785FA02460E
:10E9C0000028AAD0934639E683464BE719A8DDF81C
:10E9D00018A0FBF7E5FE1CA8FBF7E2FE1FA8FBF75B
:10E9E000DFFE19A8FBF7D4FE5246089919A8FCF7D8
:10E9F00025FE5D46834618B119A8FBF7D1FE52E506
:10EA000059465046FCF7EEFB029B19A9002808BFA7
:10EA1000002350461A46FCF76DF8834619A8FBF709
:10EA2000BFFEBBF1000F7FF43EAD28460499FFF70F
:10EA30003FF8079B8346002B7FF4D4ACBAE42299BD
:10EA40002846FFF735F8834698E6DFF82CB0F5E561
:10EA500001220AF1FF310AEB030402FA01F3013C3F
:10EA60000293DBB20691B4FBFAF45646039302E537
:10EA700080B2FFFF80B0FFFF00B3FFFF2DE9F84336
:10EA8000012ADDE9087843D80D468146002105F1C9
:10EA900018001E461446FCF7A5FB38B9B8F1000F64
:10EAA00038D0012338703360BDE8F88309F10400E1
:10EAB000FCF7F6F88146C4B943000133984533604A
:10EAC00028D304233946024601F8013B2846FCF7C7
:10EAD000A9F90028E8D109F1010105F10C00394438
:10EAE0004A46BDE8F843FCF79DB9431C984533609E
:10EAF00010D3002105F10C00FCF794F839460230E0
:10EB000001F8010B4A462846BDE8F843FCF78AB9EC
:10EB10000148C9E70148C7E780B0FFFF00B1FFFF28
:10EB2000002B41D0F8B51E46137814460D46ABB9FC
:10EB3000012E35D131462846FCF73AF800B1F8BD30
:10EB4000314605F10C00FCF733F80028F7D10146F7
:10EB500005F11800BDE8F840FCF72AB80430FCF7CE
:10EB60009FF823780746042B1CD1430001339E42B3
:10EB700016D10246611C2846FCF7C2F80028DED1F7
:10EB8000791C21443A4605F10C00FCF7B9F800283D
:10EB9000D5D105F118000121BDE8F840FCF708B80F
:10EBA0000248F8BD0248F8BD0048704780B0FFFF3A
:10EBB00080B1FFFF2DE9F0410C4686B005460121EA
:10EBC00004F11800FCF70EFB002840F09F802B6B2F
:10EBD000002B00F0A080EB6B002B00F09C80014626
:10EBE00006462046FCF7FEFA0028C0F28F8004F1AA
:10EBF0000C0731463846FCF7F5FA0028C0F286804B
:10EC000005F1040841462046FCF784FA00287DDA25
:10EC100041463846FCF77EFA002877DA6846FBF76B
:10EC2000B7FD03A8FBF7B4FD3A4639466846FCF742
:10EC3000C5FD064648B16846FBF7B2FD03A8FBF7E1
:10EC4000AFFD304606B0BDE8F08129466846FEF7C4
:10EC500093FC06460028EED12246214603A8FCF785
:10EC6000ADFD06460028E6D1294603A8FEF784FC40
:10EC700006460028DFD1AB69002B4ED003A905F171
:10EC800010020846FCF766FC06460028D3D107E0D0
:10EC900003A942460846FCF79DFB06460028CAD158
:10ECA000414603A8FCF736FA0028F1DA03A9224608
:10ECB0000846FCF783FD06460028BCD1294603A878
:10ECC000FEF75AFC06460028B5D103A905F11C023F
:10ECD0000846FCF73FFC06460028ACD107E003A934
:10ECE00042460846FCF776FB06460028A3D141467B
:10ECF00003A8FCF70FFA0028F1DA03A96846FCF72D
:10ED000009FA144E002808BF002694E7114E304639
:10ED100006B0BDE8F081104E93E703A90322084630
:10ED2000FCF700FD0646002885D10EE0002103A86F
:10ED3000FCF758FA0028B9D003A942460846FCF768
:10ED400009FC064600287FF476AF039B002BEDDB21
:10ED5000ACE700BF80B3FFFF80B0FFFF2DE9F043B9
:10ED60000378ABB0002B00F0C4800A789A4240F0E0
:10ED7000C08001F188070C46054639468830FCF70B
:10ED8000C9F9002840F0B58004F19409494605F11D
:10ED90009400FCF7BFF9002840F0AB8004F1A00814
:10EDA00005F1A0004146FCF7B5F90646002840F001
:10EDB000A080254602A8FBF7EBFC05A8FBF7E8FCC2
:10EDC00008A8FBF7E5FC31467C220BA8F3F70AFD07
:10EDD00015F87C1B0BA800F09FF804F140000121FE
:10EDE0002834FCF7FFF9002840F08180179B002BA6
:10EDF0007DD01A9B002B7AD001212846FCF7F2F92E
:10EE00000028C0F283801EA92846FCF783F9002859
:10EE10007CDA21460BA8FFF7CDFE064680B9179B8A
:10EE2000002B64D01A9B002B61D0CDE90000234653
:10EE30002A4602A90BA8FFF76BFA064600284CD019
:10EE400002A8FBF7ADFC05A8FBF7AAFC08A8FBF796
:10EE5000A7FC239B012B26D12898C8B1299AAAB1D7
:10EE6000002505EBC50310EB830432D02046FBF7E9
:10EE700097FC04F10C00FBF793FC04F11800FBF77E
:10EE80008FFC299A013595422898EAD3F9F77AFD43
:10EE900000220BAB1A702AA901338B42FAD13046FB
:10EEA0002BB0BDE8F0830CA8FBF77AFC0FA8FBF7AA
:10EEB00077FC12A8FBF774FC15A8FBF771FC18A8E7
:10EEC000FBF76EFC1BA8FBF76BFC1EA8FBF768FCAE
:10EED000C2E701359542C4D3D8E7394602A8FCF70A
:10EEE00019F920B9494605A8FCF714F930B1084EC4
:10EEF000A6E7074E30462BB0BDE8F083414608A890
:10EF0000FCF708F9064600289AD0F0E7014E97E78B
:10EF100080B0FFFF80B3FFFF70B50D460446FEF7DB
:10EF200059FF032D257025D108230125144A1549C1
:10EF3000A36023622365E362A363E260124B134A7A
:10EF4000134E144821636065E263A3646560E56164
:10EF5000E564A5626563C4E910556662201DFBF790
:10EF600071FEA06504F14C00FBF76CFEC4E91705C7
:10EF7000002070BD2046FEF72DFF074870BD00BF82
:10EF80008015050020150500786F0220401505004A
:10EF9000001505006015050080B1FFFF012830B4A1
:10EFA0000A4B03D10AE01D7C854208D053F8144F68
:10EFB000002CF8D16FF02D0030BC7047044C0C6071
:10EFC0005B68002030BC1360704700BFE01505008F
:10EFD000AC150500032830B40A4B03D10AE01D7CB0
:10EFE000854208D053F8144F002CF8D16FF02D0053
:10EFF00030BC7047044C0C605B68002030BC136070
:10F00000704700BFB8150500A01505002DE9F04FA9
:10F010000E460021054685B00846009317461C465B
:10F02000134603AADDF83890FAF7F6FF2846F3F7FF
:10F0300071FB82463046F3F76DFB03994B1C03EBE3
:10F040009113534418440F9B984253D80120F9F769
:10F0500085FC8246002852D0039900943B4603AABF
:10F06000FAF7DAFF804600283DD12846F3F752FB35
:10F07000294602464846F3F788FB2846F3F74AFB41
:10F08000039B09EB00049BB1D3460A27402B28BF02
:10F0900040231D4659461A462046F3F776FB039B4C
:10F0A0002C445B1B2770AB4401340393002BEDD140
:10F0B0003046F3F72FFB314602462046F3F765FB57
:10F0C0003046F3F727FB002102462318A1540133F1
:10F0D000109AA3EB090350461360F9F753FC40461E
:10F0E00005B0BDE8F08F5046F9F74CFC404605B03E
:10F0F000BDE8F08F109B6FF029081860EFE7DFF88C
:10F100000480ECE780EEFFFF024B0A461B680021FB
:10F11000184700BF7C6F022010B504460C20F9F799
:10F1200013FCE06018B1BDE81040FAF77BBD042085
:10F1300010BD00BF70B5064614200D46F9F704FC5B
:10F1400078B12B68044643606B6801468360EB68C6
:10F15000C360AB680361F068FAF76EFD20B96868B8
:10F1600070BD4FF0FF3070BD2046F9F70BFC4FF03B
:10F17000FF3070BDF0B5064685B0C0680C46174636
:10F18000FAF77AFD002837D082680546D4E90003F3
:10F190009A4228BF1A46626010B16968F3F7F5FA1F
:10F1A000A06818B12B690BB1EA68E2B90023E360EB
:10F1B0003B0702D5606805B0F0BDF068FAF752FD74
:10F1C00005460028F6D0D0E9013102690093C368F2
:10F1D000CDE9011203936846D6E9013198472846E4
:10F1E000F9F7D0FBE6E7E3689A4228BF1A46E260E7
:10F1F0002969F3F7CAFADBE74FF0FF30DBE700BF1E
:10F2000008B5C068FAF738FD08B1806808BD4FF04E
:10F21000FF3008BD30B50546C06885B0A8B91AE012
:10F22000E868FAF71FFD044670B1D0E90101D4E99E
:10F230000332CDE90001CDE90223D5E90131684669
:10F2400098472046F9F79EFBE868FAF71BFD00286F
:10F25000E6D105B030BD082005B030BD30B505465B
:10F26000C06885B0A0B91CE0FAF7FCFC044670B198
:10F27000D0E90101D4E90332CDE90001CDE902234F
:10F28000D5E90131684698472046F9F77BFBE868E5
:10F29000FAF7F8FC0446E868002CE5D1F9F772FBB0
:10F2A000EC6005B030BD00BF0020704710B50C46C3
:10F2B000D0E9013120469847606810BD4FF0FF301B
:10F2C000704700BF4FF0FF30704700BF002070470D
:10F2D000704700BF4FF48C720021F3F783BA00BF70
:10F2E00018B14FF48C71FFF70FBF7047C02A00F0C0
:10F2F0008481B2F5807F00F07D81802A02D06FF09A
:10F300001F0070470A2303602DE9F04F07464FF0B6
:10F31000000C00F1080485B0520947F8044F8B78BF
:10F320004D780E781B0443EA0523CD7833430CF166
:10F33000010C43EA0563944547F8043F01F10401D9
:10F34000EDD303680C2B00F0BF810E2B00F0588129
:10F350000A2B40F04B814469D84BC4F307228168E3
:10F360009A5C250E5E5D81F00101E5B25D5D4A406B
:10F37000C4F3074182EA06425E5C82EA0565C16821
:10F3800085EA06220769514081EA070989EA0404EF
:10F39000C4F307255D5D260E9E5D82F0020C85EAB2
:10F3A0000C0585EA0645E6B213F806C0C4F3074625
:10F3B0009E5D85EA0C6585EA06256F4087EA040CA8
:10F3C000CCF307269E5D4FEA1C6E13F80EE085F025
:10F3D000040886EA080686EA0E465FFA8CFE13F8F1
:10F3E0000EE08261CCF3074286EA0E6613F802E073
:10F3F00085EA010286EA0E2686EA020888EA040EF9
:10F40000C161CEF30721595C4FEA1E6A13F80AA0C6
:10F4100086F0080B81EA0B0181EA0A415FFA8EFA55
:10F4200013F80AA04462CEF307441C5D81EA0A6126
:10F4300081EA042181EA070A8AEA0E04C2620763AC
:10F44000C4F3072288EA0707C0E90E68C0F82090D5
:10F450008562C0F834C0C0F844E00764816413F8E2
:10F4600002C0220E9A5C81F010058CEA050C8CEA31
:10F47000024CE2B29D5CC4F307429A5C8CEA056CD4
:10F480008CEA022C81EA080181EA0C098EEA090261
:10F49000C2F307255E5D150E5D5D8CF020077E4092
:10F4A00086EA0546D5B25D5DC164C2F30741595C89
:10F4B00086EA056686EA01268AEA060E82EA0E08D0
:10F4C000C8F307215F5C4FEA1861595C86F040057C
:10F4D0006F4087EA01475FFA88F1595C8AEA0905BB
:10F4E00087EA0167C8F30741595CC0F850A087EA72
:10F4F000012789EA060A05668AEA070582EA050104
:10F500004465C1F307241C5D4FEA116B13F80BB07F
:10F51000426687F080026240CCB282EA0B4213F866
:10F5200004B0C1F307441C5D82EA0B6282EA042244
:10F530008EEA0204C0F858C081EA040C8666C567EA
:10F540008EEA050687675540CCF30727C0E91BAE56
:10F55000C0F88410C0F88820C0F88060C0F85C90C3
:10F56000C0F87480C0F88C50DE5D82F01B024FEA58
:10F570001C6713F807E056405FFA8CF29F5CCCF3EF
:10F5800007429A5C86EA0E4686EA076686EA022603
:10F5900075406940C1F307229A5C0F0EDF5D86F06B
:10F5A000360E82EA0E0282EA0742CFB213F807E073
:10F5B000C1F30747DF5D82EA0E6383EA072383EA2C
:10F5C000040282EA010EC0E92665C0E92C2EC0F8CB
:10F5D000904083EA05076C40C0F894C0C0F8A410BE
:10F5E000C0F8A830C0F8AC70C0F8A040002005B04A
:10F5F000BDE8F08F0E23036086E60C23036083E6EC
:10F60000D0E903CED0E90789D0E90572466A83685C
:10F610007046DFF8B0A0294DCDF800C05AF804BFFD
:10F62000C6F3072C15F80CE04FEA166C83EA0B03BF
:10F6300015F80CB05FFA86FC8EEA030315F80CC0CF
:10F64000C6F3074E83EA0B4315F80EE083EA0C631A
:10F65000009983EA0E235940484047405FFA87FCEF
:10F6600015F80CE04FEA176C15F80CB0C7F3072C2F
:10F670008EEA020215F80CC0C7F3074E82EA0B624D
:10F6800015F80EE082EA0C2282EA0E4288EA0208AD
:10F69000C4E9083100910A4989EA080986EA09069D
:10F6A0008A45C4E90A07C4E90E96C4E90C2804F1A6
:10F6B0002004B3D1002005B0BDE8F08F98160500F6
:10F6C000B027050094270500C269B24BC2F3072496
:10F6D00081681D5D140E1E5D81F00101D4B21C5DB8
:10F6E0004D40C2F30741595C85EA0645C76885EA83
:10F6F000046585EA012501696F40466981EA0709C9
:10F70000846986EA090684EA060882EA0802C2F3E6
:10F71000072413F804E04FEA126C13F80CA085F0EC
:10F7200002045FFA82FC8EEA040413F80CE0C2F3D0
:10F73000074C13F80CC084EA0A4484EA0E6484EA95
:10F740000C24614001940C4681690562614082EAA3
:10F75000010C0391CCF3072E019913F80EE04FEA48
:10F760001C6A13F80AA081F0040B8EEA0B0E8EEAD5
:10F770000A4A5FFA8CFE13F80EE0C0E90A968AEA9C
:10F780000E65CCF3074E13F80EE087EA010A85EA0E
:10F790000E258AEA050E86EA0E010091214686EAC8
:10F7A0000409009CC0E90C8282EA04064762C0F8A2
:10F7B0003CA002910164039FC6F3072481EA0E086E
:10F7C000C0E9127C1C5D4FEA166CC0E9145EC0F8FB
:10F7D000588085F0080513F80C805FFA86FC0199C3
:10F7E00013F80CC06540C6F307441C5D85EA084564
:10F7F000816385EA0C65029985EA042569400191D7
:10F8000039468469C0F8449084EA050886EA080904
:10F81000C9F3072413F804A04FEA19641C5D85F0AE
:10F82000100C8AEA0C0C5FFA89FA13F80AA08CEA29
:10F83000044CC9F307441C5D8CEA0A6C8EEA050E81
:10F840008CEA042C8EEA0C046240C0F86CE0C2F32F
:10F85000072E13F80EE04FEA126A13F80AA08CF094
:10F86000200B8EEA0B0E8EEA0A4A5FFA82FE13F82C
:10F870000EE0009F8AEA0E6AC2F3074E13F80EB03C
:10F8800081EA070E01998AEA0B2B81EA0B0A009F95
:10F89000C0F860E088EA0A0EC7654666C0F87C904A
:10F8A00082EA0E06016787EA04094F4061408566D7
:10F8B000C0F88810C6F3072588EA0901C0F890103F
:10F8C0005D5D310E595CC0F88440C0F898B084EAA0
:10F8D0000B0447678BF0400BF7B2DF5DC0F8AC60FC
:10F8E00085EA0B05C6F3074685EA0145995D85EA79
:10F8F000076585EA0125C0F89C406C4089EA04064A
:10F90000C0F894207240C2F30721C0F880C0595C4F
:10F9100089EA0A0C170EC0F88C90C0F8A4C013F83E
:10F92000079085F0800CD7B281EA0C0113F807C06C
:10F93000C2F30747DF5D81EA094181EA0C6383EA8C
:10F940000723C0F8788083EA0A0C83EA0808C0F825
:10F95000A8E08EEA060788EA020B8CEA060983EA29
:10F96000040E8AEA0401C0F8A0A0C0E93072C0F811
:10F97000BC60C0E92C54C0E9368BC0F8C830C0E97F
:10F9800034C9C0F8CCE0C0F8B810002005B0BDE81C
:10F99000F08F00BF981605002DE9F04FD0E9000365
:10F9A000401005468BB01C68D1F800A0013D0295BF
:10F9B0004F688D6808928AEA040A029ACC68D9686E
:10F9C00009905E68986884EA010C002A03F110012E
:10F9D00086EA070685EA0005069140F30282D24ACC
:10F9E000D24991460091D249DFF84CB30792019178
:10F9F00003F1300E5FFA8AF35FFA8CF059F8237046
:10FA000059F82040EAB25EF8200C59F8222047400D
:10FA10005EF8140C04924FEA1C632A0E5BF8233044
:10FA20005BF822204440300E5BF8208000985F4055
:10FA30005440F1B2C6F30723CAF3072259F8211044
:10FA400050F8233050F822205EF81C0C03974840F1
:10FA50004FEA1A615BF82110049F48405EF8181CB9
:10FA600005947940009F019C81EA0808C5F30721AD
:10FA700057F82110C6F30746039FCAF3074AC5F398
:10FA8000074554F82AA054F8255054F82660009CE5
:10FA90007B40CCF3072754F82770019CCCF3074C2C
:10FAA00054F82CC0059C6B4062405640484080EAA8
:10FAB0000C0088EA07085FFA83FC350E88EA0A081A
:10FAC00059F82CA05BF82550C0F307220395009D40
:10FAD000C8F3074755F82220019DC4B2190E55F806
:10FAE000277059F824405BF82110009DC8F3072CBB
:10FAF00055F82C5084EA010C019CC6F3074154F8D8
:10FB000021100495039D03915FFA88F159F8214073
:10FB10005EF8101C8AEA050A8AEA010A010E5BF8FF
:10FB200021504FEA18686C40F5B259F825508AEA1E
:10FB3000020A5BF828205EF80C1C85EA02085EF8D1
:10FB4000082C019D6240C0F30740C3F30724C3F3B0
:10FB500007438CEA010C55F82000009955F8235012
:10FB6000049BC6F3072651F824408AEA070A51F895
:10FB700026705EF8046C8CEA0301039B88EA060891
:10FB800081EA0306029B7A4088EA0408013B85EA81
:10FB9000020588EA000C0EF1200E02937FF42AAFD2
:10FBA000099B069A03F10063013B02EB43130693A2
:10FBB0004FF0000E079C5FFA8AF05FFA8CF12B0E73
:10FBC00054F820704FEA1C6254F821005BF82310AF
:10FBD0005BF82220069B4140079803911B68F1B215
:10FBE0007A40009FC6F3072450F82100019957F886
:10FBF00024705A40C5F30744330E51F824105BF8C3
:10FC00002340019BC6F3074653F826604FEA1A6368
:10FC10005BF823307A40049682EA0106079A58403E
:10FC2000EBB2069F52F823200099C5F3072582EA1C
:10FC3000040B0296039C51F82560F968009ACAF3F8
:10FC400007236140019C52F82320CAF3074ACDF8EC
:10FC500024E054F82A40049B514081EA03027B6867
:10FC60009DF8081043407340009ECCF3072056F8DF
:10FC70002000BE68019F0391CCF3074157F8211083
:10FC80008BEA06062B4D4B40704003994440D8B296
:10FC90006F5C285C069900904FEA126B0298096924
:10FCA00015F80BB0C3F3072A15F80AA07940C4F37E
:10FCB0000746000E15F800C0AE5DC4F3072081EAC8
:10FCC0000B6B2F5C8BEA0A2BC2F307408BEA064BC7
:10FCD000CDF804C0069E15F800C00397E1B21F0ED0
:10FCE000C3F30743685CCDF810C00593C2F3072C3B
:10FCF0007369D1B2009AF0465340019A240E83EA08
:10FD000002633246B669EF5DD2F81CA0695C7040B0
:10FD100081EA0A0A029980EA0760C1F30726C1F363
:10FD2000074705990AE000BF98170500981B0500D2
:10FD3000981F050098160500982305002C5D15F8FE
:10FD40000C20AE5D695CED5D039F80EA022083EAD2
:10FD50000723049FF14683EA0743474680EA0545A7
:10FD6000280A65F3070860F30F28280C60F317488A
:10FD700000208AEA046A8AEA062A8AEA01411C0A01
:10FD800063F307074FEA1B260A0A6BF3070E61F3BA
:10FD9000070964F30F271C0C66F30F2E62F30F297B
:10FDA0004FEA1B460A0C64F317471B0E63F31F67E9
:10FDB00066F3174E089B4FEA1B6B2D0E62F3174933
:10FDC000090E6BF31F6E65F31F6861F31F69C3F8BB
:10FDD00000E05F60C3F80880C3F80C900BB0BDE88A
:10FDE000F08F044BDFF818B00793034B0093034BDD
:10FDF0000193DDE698170500981B0500981F050084
:10FE0000982305002DE9F04FD0E90034D1F8009097
:10FE100026688BB05B10581E099389EA0603049389
:10FE20008B68D1F80480CD680892D4E90221534050
:10FE300004F110020792D44A67680192D34A00285D
:10FE4000039088EA070885EA0105DFF848B30092C5
:10FE5000DFF8449340F3E980AA46049A04F1300C99
:10FE60000293019B9DF80850D1B25FFA88F65FFAC1
:10FE70008AF453F8210053F8267053F8244053F8BD
:10FE800025505CF8203C5CF81C6C80EA030E029B59
:10FE900077405CF8146C180E5BF820004FEA18618C
:10FEA0006640140E5BF821105BF82440009B05951A
:10FEB00047408EEA010E04974FEA1A65059FCAF380
:10FEC0000721C2F3072066405CF8184C53F8211054
:10FED00053F820005BF82550029B7C40009F654052
:10FEE0008EEA0101C3F30724C8F3072E57F8244014
:10FEF00057F82EE0CAF3074A049FC3F3074359F8A3
:10FF00002AA059F82330C2F30742784059F822203A
:10FF1000594085EA0E0580EA0A036A401D46C8F387
:10FF2000074859F82880029566409DF808500198C6
:10FF300086EA08065FFA81F850F828800098C6F330
:10FF4000072750F827700198140E50F825505BF8D9
:10FF500024400098C1F3072A50F82A0085EA040AD1
:10FF6000C6F3074459F824404FEA136E5BF82EE0BD
:10FF7000C2F30725C2F307430594D4B25CF8102CF2
:10FF800088EA0E0E59F823308EEA02027A40049075
:10FF90005A4001985CF8083C4FEA11684FEA166E27
:10FFA000F6B250F82440069350F826605BF82830EB
:10FFB00000985BF82EE050F825805E40029D069B7D
:10FFC00084EA0E0E8EEA0304C5F3072350F82330AB
:10FFD000C1F3074159F82110C5F3074063405CF8AD
:10FFE000045C5CF80C7C4B4059F820007540049E82
:10FFF000059C0293039B8AEA070785EA0805774078
:020000025000AC
:10000000013B87EA040885EA000A0CF1200C0393FF
:100010007FF427AF55460492099A079902F10062CE
:10002000013A01EB4212029B0792019E9DF810409B
:100030004FEA186156F824705BF821105FFA88F0D7
:100040001A0E7940009F56F820405BF82200C5F355
:10005000072657F82670C3F3074659F82660604014
:10006000019C0590E8B254F820003446079A4FF0FE
:10007000000C1268E24651407940049F2A0E5BF85A
:1000800022603A0E5BF822206140019C0291D9B2B5
:10009000424054F82100009C80EA060B3E46C3F320
:1000A000072354F82310079BC5F307455868059BA1
:1000B00059F825505840C7F3072354F823300695C4
:1000C000C6F307465840069B59F82670079E5840CD
:1000D0000190F368009853405940C8F30742C8F3B1
:1000E00007232B4D9DF8084050F82300B66859F8B7
:1000F00022308BEA0606019A4B40295D079C70402E
:10010000784090464FEA126BD7B22269C3F30726B4
:100110004A40029915F80B40C1F3072115F801B0C8
:10012000AE5DC3F30741C0F3074915F80990EF5DD1
:10013000CDF810B015F801B082EA0461C2B2AC5C2F
:1001400081EA0621079A019781EA094156690091DF
:100150000199070E4E401146EF5DCDF814B092693B
:100160004FEA136BD1F81C9086EA0767029915F8DD
:100170000B60DBB2EB5CC0F30720624015F800B007
:1001800082EA06620AE000BFC0280500C02C050014
:10019000C0270500C0340500C0300500080EC8F3B4
:1001A0000726285CC1F30744AE5D83EA0903C8F360
:1001B000074915F809902D5D82EA062282EA054575
:1001C000009AE646160A62F3070C0022049983EAB5
:1001D000006387EA0127059983EA0B2387EA014731
:1001E000114683EA09431A0A63F30701280A62F3F6
:1001F0000F2165F3070E039160F30F2E280C60F3B7
:10020000174E03981A0C62F317401B0E63F31F601E
:10021000089B66F30F2CD8600020009E3C0A67F311
:10022000070A0099360C64F30F2A3C0C66F3174C4E
:10023000090E64F3174A3F0E2D0E61F31F6C67F32E
:100240001F6A65F31F6EC3F800C0C3F804A0C3F8AB
:1002500008E00BB0BDE8F08F10B4144601291A462F
:10026000214603D05DF8044BFFF7CCBD5DF8044B8D
:10027000FFF792BB30B599B00546684600F0CEFA5C
:10028000694608A800F0D6F9044608A9284600F0F7
:1002900011F9204619B030BD2DE9F04107460D4651
:1002A000904688B002F12001684607F12006F0F779
:1002B000AFF96A4669466846F0F73EF93046694646
:1002C000F0F7A6F932463146304605F12004F0F742
:1002D00033F96A4669466846F0F72EF920464146EA
:1002E000F0F796F96A4641463846F0F792F9224609
:1002F00021466846F0F720F9224669466846F0F73D
:100300001BF969466846114AF0F716F9694628460E
:10031000F0F77EF93A4629462846F0F74CF93A4676
:1003200029462846F0F747F92A4639462046F0F78D
:1003300042F96A4621462046F0F76BF932462146DB
:100340002046F0F738F908B0BDE8F0812039050003
:10035000F0B504460E4699B00A4601466846F0F7E5
:100360002AF969466846F0F753F96A46214608A813
:1003700006F1200504F12007F0F74BF96A463146F3
:100380006846F0F746F939462A4610A8F0F7D4F83F
:100390002A4639462846F0F70EF929463046F0F746
:1003A00037F96A4608A92046F0F7C6F822463146D2
:1003B0003046F0F700F96A4608A96846F0F7FBF8FE
:1003C0006A4639463846F0F724F9324608A96846A5
:1003D000F0F7F1F86A4629462846F0F71AF93A4646
:1003E00029462846F0F7E7F810A96846F0F710F913
:1003F000224669462046F0F7DEF808A9224608465C
:10040000F0F7D9F810A908AA0846F0F702F93A4619
:1004100010A93846F0F7CFF819B0F0BD2DE9F0413A
:100420000C460546904688B0224601466846F0F7DD
:10043000C2F869466846F0F7EBF86A46294628464E
:1004400004F12006F0F7E5F805F120076A46214699
:100450006846F0F7DEF8324630463946F0F7ABF83A
:1004600031462046F0F7D4F82A4621462046F0F7D8
:10047000A2F86A4621462046F0F79DF86A462946CA
:100480004046F0F798F8424639463846F0F7C1F84A
:10049000224629466846F0F78EF86A4631463046CD
:1004A000F0F7B7F83A4631463046F0F784F808B02E
:1004B000BDE8F08138B504460D4600F0E5F805F1D9
:1004C000200104F12000BDE8384000F0DDB800BF95
:1004D0002DE9F047B8B08A468146114610A8514A26
:1004E000F0F7DEFB5049024610A8F0F7F9FB804612
:1004F000179F4C4908EAD777C7F1010210A8F0F717
:10050000EFFB179D5246ED4328A918A8FFF7C4FE3C
:10051000ED0F20A9C5F10102084600F091F8FE2672
:10052000C8F101086A4618A928A8FFF777FF7311D8
:1005300038AA02EB830353F8A04C06F01F03DC40FB
:1005400004F0010465402A4628A918A8F0F733FCF6
:100550002A4630A920A8F0F72EFC013E28A918A8A9
:10056000FFF7F6FE731C2546DCD1C4F1010208A892
:1005700020A900F065F87D406A4618A928A8FFF771
:100580004DFF28A92A4618A8F0F715FC2A4630A9DD
:1005900020A8F0F710FC08A96A460846F0F739F8D9
:1005A00008A9084600F08AF808A909F120040AF110
:1005B00020020846F0F72DF820A908AA2046F0F7F7
:1005C00028F808AA18A96846F0F723F8694668468B
:1005D000F0F71EF818AA694608A8F0F71AF821469D
:1005E0006846F0F715F808AA69461046EFF7E3FFEA
:1005F00008A90E4A6846EFF7DEFF20462021EFF7F4
:100600008EFF08A943420246684643EA0808F0F70D
:10061000D2FB48466946064AEFF7FBFF404638B032
:10062000BDE8F08760390500003905004039050054
:10063000806F02200A460149FFF74ABFC038050013
:100640002DE9F04104460D468C46002607469046AB
:100650000FCD0FC488B095E80F0084E80F00624604
:1006600069466846CDE90066CDE90266CDE90466D3
:10067000CDE90666EFF79FFF424669463846F0F738
:100680009AFB08B0BDE8F081CB691BBA03608B69A7
:100690001BBA43604B691BBA83600B691BBAC3600A
:1006A000CB681BBA03618B681BBA43614B681BBAEA
:1006B00083610B681BBAC361704700BF70B50D46FC
:1006C000052498B0064610A8EFF7A2FF2A4610A905
:1006D0006846EFF79EFF694610A8EFF799FF10A94B
:1006E0000846EFF795FF6A4610A908A8EFF791FFB3
:1006F00008A910A8EFF78CFF10A90846EFF788FFAC
:1007000010A90846EFF784FF10A90846EFF780FF0D
:1007100010A908AA0846EFF77CFF10A90846EFF7D2
:1007200077FF10A90846EFF773FF10A96A4608A8DB
:10073000EFF76FFF08A910A8EFF76AFF10A90846A6
:10074000EFF766FF013C10A9F5D108AA0846EFF7BC
:1007500060FF052410A90846EFF75AFF10A90846C4
:10076000EFF756FF013CF5D110A908AA0846EFF7AC
:1007700050FF10A908A8EFF74BFF08A90846EFF7AC
:1007800047FF08A96A466846EFF743FF1024694609
:1007900010A8EFF73DFF10A90846EFF739FF013C1D
:1007A00010A9F5D12A460846EFF733FF402410A9D7
:1007B0000846EFF72DFF10A90846EFF729FF013C87
:1007C000F5D110A96A460846EFF723FF102410A9B7
:1007D0000846EFF71DFF10A90846EFF719FF013C87
:1007E000F5D110A96A460846EFF713FF102410A9A7
:1007F0000846EFF70DFF10A90846EFF709FF013C87
:10080000F5D110A908AA0846EFF703FF2A4610A958
:100810003046EFF7FEFE18B070BD00BF38B50B468E
:100820000A68124D12BAC2614A68014612BA826160
:100830009A68044612BA4261DA6812BA02611A6909
:1008400012BAC2605A6912BA82609A6912BA4260D8
:10085000DB692A461BBA0360F0F722FA29460246F2
:100860002046BDE83840F0F73BBA00BF80390500AC
:08087000A4F9FE7F0100000065
:10087800000000006124040000000000612404005E
:10088800000000006124040000000000612404004E
:10089800000000006124040000000000651D040041
:1008A800000000006124040000000000612404002E
:1008B800E86F0220B5400400000000006124040035
:1008C800000000006124040000000000612404000E
:1008D80000000000612404000000000061240400FE
:1008E80000000000612404000000000061240400EE
:1008F80000000000612404000000000061240400DE
:1009080000000000612404000000000061240400CD
:10091800000000006124040000000000A51E04007F
:1009280000000000612404000000000061240400AD
:10093800000000006124040000000000612404009D
:10094800000000006124040000000000612404008D
:10095800000000006124040000000000612404007D
:10096800000000006124040000000000612404006D
:10097800000000006124040000000000612404005D
:10098800000000006124040000000000612404004D
:10099800000000006124040000000000612404003D
:1009A800000000006124040000000000612404002D
:1009B800000000006124040000000000612404001D
:1009C800000000006124040000000000612404000D
:1009D80000000000612404000000000061240400FD
:1009E80000000000612404000000000061240400ED
:1009F8000000000061240400000000004D3F0400D6
:100A080000000000612404000000000061240400CC
:100A180000000000612404000000000061240400BC
:100A280000000000612404000000000061240400AC
:100A3800000000006124040000000000612404009C
:100A4800000000006124040000000000612404008C
:100A5800000000006124040000000000612404007C
:100A6800000000006124040000000000612404006C
:080A78000000000061240400ED
:100A80008B0B0500411A0400000000008B0B0500D1
:100A90008D1C040000000000E40B0500C91D0400CB
:100AA00000000000EF0B0500C91D0400000000005D
:100AB000FA0B0500E51E0400000000008B0B05008A
:100AC0008D260400000000008B0B05009931040006
:100AD000000000008B0B05007934040000000000CA
:100AE000D4100500F53D0400CC100500C30B050033
:100AF000E5430400281105008B0B0500894604001E
:100B0000000000008B0B0500C1460400000000003F
:100B100001000000000000000F0000000E000000B7
:100B200000000000000000000000001007000000AE
:100B300054686520415420686F73742073616D7030
:100B40006C6520737461727465640A005468652072
:100B5000415420686F73742073616D706C652073ED
:100B600074617274656420310A004552524F523AE2
:100B700020415420486F7374206E6F7420696E6931
:100B80007469616C697A6564200D0A0002000000D6
:100B9000940B050000000000B40B050006000000E7
:100BA000E0FF0F0000000220BC0B05002100000048
:100BB000E0FF0320464C4153485F30005352414D03
:100BC0005F3000554152545F30000000091D0400A1
:100BD0000000000000000000E11D0400A91C04004A
:100BE00000000000636C6B5F6B33327372630063F1
:100BF0006C6B5F6D3136737263007379735F636C16
:100C00006F636B002A2A2A2A2A2042555320464124
:100C1000554C54202A2A2A2A2A0A0020205072657C
:100C20006369736520646174612062757320657205
:100C3000726F720A00202042464152204164647261
:100C40006573733A20307825780A002020496D704A
:100C500072656369736520646174612062757320D5
:100C60006572726F720A002020496E737472756328
:100C700074696F6E20627573206572726F720A00FC
:100C80005265736572766564204578636570746932
:100C90006F6E20280053707572696F757320696ECE
:100CA00074657272757074202849525120002A2A86
:100CB0002A2A2A2048415244204641554C54202A91
:100CC0002A2A2A2A0A002020427573206661756C40
:100CD00074206F6E20766563746F72207461626C2D
:100CE0006520726561640A0020204661756C74207D
:100CF000657363616C6174696F6E2028736565202C
:100D000062656C6F77290A002A2A2A2A2A204465FC
:100D1000627567206D6F6E69746F722065786365A8
:100D20007074696F6E20286E6F7420696D706C65C9
:100D30006D656E74656429202A2A2A2A2A0A002AE7
:100D40002A2A2A2A20257320256429202A2A2A2AA9
:100D50002A0A002A2A2A2A2A204D5055204641557F
:100D60004C54202A2A2A2A2A0A002020537461631C
:100D70006B696E67206572726F720A002020556E73
:100D8000737461636B696E67206572726F720A00BB
:100D90002020446174612041636365737320566948
:100DA0006F6C6174696F6E0A0020204D4D46415290
:100DB00020416464726573733A20307825780A00A4
:100DC0002020496E737472756374696F6E2041637D
:100DD000636573732056696F6C6174696F6E0A0086
:100DE0002020466C6F6174696E672D706F696E7438
:100DF000206C617A792073746174652070726573F8
:100E00006572766174696F6E206572726F720A0026
:100E10002A2A2A2A2A205553414745204641554C23
:100E200054202A2A2A2A2A0A002020446976697333
:100E3000696F6E206279207A65726F0A00202055F2
:100E40006E616C69676E6564206D656D6F72792087
:100E50006163636573730A002020537461636B20C0
:100E60006F766572666C6F770A0020204E6F206384
:100E70006F70726F636573736F7220696E737472D3
:100E8000756374696F6E730A002020496C6C656726
:100E9000616C206C6F6164206F66204558435F521F
:100EA000455455524E20696E746F2050430A0020FD
:100EB00020496C6C6567616C20757365206F6620D6
:100EC00074686520455053520A00202041747465AF
:100ED0006D707420746F2065786563757465207516
:100EE0006E646566696E656420696E73747275639D
:100EF00074696F6E0A002A2A2A2A2A2048617264BD
:100F00007761726520657863657074696F6E202AF9
:100F10002A2A2A2A0A002A2A2A2A204B65726E6562
:100F20006C20416C6C6F636174696F6E20466169FF
:100F30006C75726521202A2A2A2A0A002A2A2A2A5E
:100F40002A204B65726E656C204F4F505321202A2A
:100F50002A2A2A2A0A002A2A2A2A2A204B65726E5D
:100F6000656C2050616E696321202A2A2A2A2A0A88
:100F7000002A2A2A2A20556E6B6E6F776E204661F2
:100F800074616C204572726F7220256421202A2AB8
:100F90002A2A0A0043757272656E7420746872653D
:100FA0006164204944203D2025700A4661756C74B7
:100FB000696E6720696E737472756374696F6E20F1
:100FC00061646472657373203D20307825780A006F
:100FD00049535200657373656E7469616C2074685F
:100FE0007265616400466174616C206661756C7441
:100FF00020696E20257321205370696E6E696E67BB
:101000002E2E2E0A00466174616C206661756C7428
:1010100020696E207468726561642025702120410A
:10102000626F7274696E672E0A002D2B20233000C8
:10103000686C4C7A000000006D3104000000000074
:101040004D3104003810050054100500381005001B
:101050005C1005008000000070500220800000003D
:10106000F05902200090004000000000EF3604001C
:101070002F36040067370400193704002B360400AC
:10108000793904007D350400B13604003D3904008F
:10109000633504003336040049350400C7340400C6
:1010A000CF37040089340400554152545F310000A9
:1010B000253E0400093D04003D3D04006F3D040051
:1010C00075400400B13D040000000000002584408C
:1010D000000000004750494F5F30000055420400B7
:1010E00079420400A7420400E540040045420400A0
:1010F000BD420400FD4204001F43040035430400C8
:101100003D43040065430400734304003D43040071
:10111000534304008143040091430400AD430400A1
:10112000A1430400A543040000800040200001000A
:10113000A06F0220007002200C7002202470022098
:1011400030700220F5FFFFFF6D61696E0069646C0D
:1011500065000000843002202A2A2A2A2A20426FB1
:101160006F74696E67205A6570687972204F5320DA
:1011700076312E31332E39392D6E637332202A2A7F
:101180002A2A2A0A0000000039900400C9900400AD
:10119000998F0400559104005950040059500400DF
:1011A00059500400595004000992040001920400AF
:1011B00075630400C9640400A96504005D67040048
:1011C000696A040001690400D16B0400016D040028
:1011D000296F0400656F040015940400AD940400A9
:1011E000CD9404007D9504002D960400F59604002E
:1011F0006597040041980400DD980400C599040037
:1012000020000E00400008008000040000010200E1
:1012100000020200000401000000000060B0012094
:10122000C00F0000060000000012050000100100C1
:1012300041542B434D45453D310000004F4B0000CC
:10124000070000000600000004000000415425587B
:10125000504D4E473D302C220000000041542543A4
:101260004D4E473D332C302C35000000000000006F
:101270002D0000000C00000073000000330000008F
:10128000730000002D000000300000002D00000061
:101290002D000000390000002D0000002D0000008E
:1012A000160000003C0000009F130F492748EBB0D8
:1012B0007E95BF75899746ADA78240EE181265D717
:1012C000F2B1666326460000D6C239B039149FEFEA
:1012D000A38ED498ACB47ED0A24860F53CD06D808B
:1012E0007595C3367943072B303F7561595052D5F8
:1012F00061403581E8E377D5E68664297C2CA973C3
:10130000A53B420B4FAFADFA67855DCAC8348B2F42
:1013100016288F1C21B7BD398DA63AA6E19C5091A5
:10132000D40D087FDE9E5475AE40F8E2FA8EC67A80
:1013300091E743F03B30AB6E49E1426B665733CDEA
:101340002AC52923053A93F8AE40E8E2FA8EC67A18
:1013500091E743F03B30AB6E49E1470B665733CD25
:101360002AC52923053A11F877055E2136878BF2C5
:101370006182E8FC127BDE93931D76B1627336D1F5
:10138000A65C993250A3178F65636B65792E510067
:1013900002000000F81305006D8B0400618B04004F
:1013A000000000000000000000000000000000003D
:1013B000BD8B0400A58B0400918B0400718B04008D
:1013C00003000000F01305006D8B0400858B040002
:1013D000000000000000000000000000000000000D
:1013E000BD8B0400A58B0400918B0400718B04005D
:1013F00045435F4448000000454300002D2D2D2D3E
:101400002D454E44205055424C4943204B45592DC3
:101410002D2D2D2D0A0000002D2D2D2D2D4245475F
:10142000494E205055424C4943204B45592D2D2DB6
:101430002D2D0A00A9F20400ADF20400BDF2040053
:10144000C5F20400CDF20400D1F2040019F1040049
:1014500035F1040075F1040001F2040015F20400F6
:101460005DF20400718D0400918D0400D18D0400A3
:10147000D58E0400FD8E0400458F0400040000009A
:10148000E9920400000000000000000002000201D8
:10149000010000000000000000000000000000004B
:1014A000000000000000000000000000000000003C
:1014B00003000000A59B04000000000000000000E5
:1014C0004142434445464748494A4B4C4D4E4F5094
:1014D0005152535455565758595A61626364656660
:1014E0006768696A6B6C6D6E6F7071727374757614
:1014F0007778797A303132333435363738392B2FA3
:101500004B60D2273E3CCE3BF6B053CCB0061D65B7
:10151000BC86987655BDEBB3E7933AAAD835C65A40
:1015200096C298D84539A1F4A033EB2D817D03777D
:10153000F240A463E5E6BCF847422CE1F2D1176B18
:10154000F551BF376840B6CBCE5E316B5733CE2BEB
:10155000169E0F7C4AEBE78E9B7F1AFEE242E34F1A
:10156000512563FCC2CAB9F3849E17A7ADFAE6BC45
:10157000FFFFFFFFFFFFFFFF00000000FFFFFFFF77
:10158000FFFFFFFFFFFFFFFFFFFFFFFF0000000067
:10159000000000000000000001000000FFFFFFFF4E
:1015A0002A8648CE3D030107000000002A864886AF
:1015B000F70D010101000000A01505000800000062
:1015C0003016050030160500030000000000000082
:1015D000000000000000000000000000000000000B
:1015E000AC150500090000003C1605004C1605006E
:1015F0000100000050160500070000005816050005
:1016000068160500020000007816050005000000BD
:101610008016050088160500030000000000000089
:1016200000000000000000000000000000000000BA
:101630007365637032353672310000007273614534
:101640006E6372797074696F6E00000052534100CE
:101650002A8648CE3D02010069642D65635075629B
:101660006C69634B6579000047656E65726963203C
:101670004543206B657900002B8104010C000000BC
:1016800069642D65634448004543206B6579206695
:101690006F72204543444800637C777BF26B6FC5D3
:1016A0003001672BFED7AB76CA82C97DFA5947F065
:1016B000ADD4A2AF9CA472C0B7FD9326363FF7CC41
:1016C00034A5E5F171D8311504C723C31896059ADE
:1016D000071280E2EB27B27509832C1A1B6E5AA001
:1016E000523BD6B329E32F8453D100ED20FCB15BEC
:1016F0006ACBBE394A4C58CFD0EFAAFB434D338555
:1017000045F9027F503C9FA851A3408F929D38F528
:10171000BCB6DA2110FFF3D2CD0C13EC5F9744175F
:10172000C4A77E3D645D197360814FDC222A9088D6
:1017300046EEB814DE5E0BDBE0323A0A4906245C62
:10174000C2D3AC629195E479E7C8376D8DD54EA9C7
:101750006C56F4EA657AAE08BA78252E1CA6B4C693
:10176000E8DD741F4BBD8B8A703EB5664803F60EEC
:10177000613557B986C11D9EE1F8981169D98E94DB
:101780009B1E87E9CE5528DF8CA1890DBFE64268F4
:1017900041992D0FB054BB16C66363A5F87C7C84B9
:1017A000EE777799F67B7B8DFFF2F20DD66B6BBDF2
:1017B000DE6F6FB191C5C554603030500201010336
:1017C000CE6767A9562B2B7DE7FEFE19B5D7D762EA
:1017D0004DABABE6EC76769A8FCACA451F82829DE6
:1017E00089C9C940FA7D7D87EFFAFA15B25959EBDC
:1017F0008E4747C9FBF0F00B41ADADECB3D4D467D5
:101800005FA2A2FD45AFAFEA239C9CBF53A4A4F7FF
:10181000E47272969BC0C05B75B7B7C2E1FDFD1C58
:101820003D9393AE4C26266A6C36365A7E3F3F4136
:10183000F5F7F70283CCCC4F6834345C51A5A5F49E
:10184000D1E5E534F9F1F108E2717193ABD8D873C1
:10185000623131532A15153F0804040C95C7C7524D
:10186000462323659DC3C35E30181828379696A17A
:101870000A05050F2F9A9AB50E070709241212368A
:101880001B80809BDFE2E23DCDEBEB264E272769F4
:101890007FB2B2CDEA75759F1209091B1D83839E25
:1018A000582C2C74341A1A2E361B1B2DDC6E6EB27B
:1018B000B45A5AEE5BA0A0FBA45252F6763B3B4DC5
:1018C000B7D6D6617DB3B3CE5229297BDDE3E33EA3
:1018D0005E2F2F7113848497A65353F5B9D1D16825
:1018E00000000000C1EDED2C40202060E3FCFC1F57
:1018F00079B1B1C8B65B5BEDD46A6ABE8DCBCB461D
:1019000067BEBED97239394B944A4ADE984C4CD4E2
:10191000B05858E885CFCF4ABBD0D06BC5EFEF2A7F
:101920004FAAAAE5EDFBFB16864343C59A4D4DD75A
:1019300066333355118585948A4545CFE9F9F91009
:1019400004020206FE7F7F81A05050F0783C3C44A8
:10195000259F9FBA4BA8A8E3A25151F35DA3A3FE14
:10196000804040C0058F8F8A3F9292AD219D9DBCE3
:1019700070383848F1F5F50463BCBCDF77B6B6C102
:10198000AFDADA754221216320101030E5FFFF1A2B
:10199000FDF3F30EBFD2D26D81CDCD4C180C0C14DB
:1019A00026131335C3ECEC2FBE5F5FE1359797A28A
:1019B000884444CC2E17173993C4C45755A7A7F2AF
:1019C000FC7E7E827A3D3D47C86464ACBA5D5DE7CB
:1019D0003219192BE6737395C06060A01981819844
:1019E0009E4F4FD1A3DCDC7F44222266542A2A7EFC
:1019F0003B9090AB0B8888838C4646CAC7EEEE2995
:101A00006BB8B8D32814143CA7DEDE79BC5E5EE266
:101A1000160B0B1DADDBDB76DBE0E03B64323256B0
:101A2000743A3A4E140A0A1E924949DB0C06060A19
:101A30004824246CB85C5CE49FC2C25DBDD3D36E05
:101A400043ACACEFC46262A6399191A8319595A4DC
:101A5000D3E4E437F279798BD5E7E7328BC8C84312
:101A60006E373759DA6D6DB7018D8D8CB1D5D56470
:101A70009C4E4ED249A9A9E0D86C6CB4AC5656FA2B
:101A8000F3F4F407CFEAEA25CA6565AFF47A7A8EF3
:101A900047AEAEE9100808186FBABAD5F078788862
:101AA0004A25256F5C2E2E72381C1C2457A6A6F1E1
:101AB00073B4B4C797C6C651CBE8E823A1DDDD7C7B
:101AC000E874749C3E1F1F21964B4BDD61BDBDDC4D
:101AD0000D8B8B860F8A8A85E07070907C3E3E422B
:101AE00071B5B5C4CC6666AA904848D8060303050C
:101AF000F7F6F6011C0E0E12C26161A36A35355F5E
:101B0000AE5757F969B9B9D01786869199C1C158AE
:101B10003A1D1D27279E9EB9D9E1E138EBF8F8134D
:101B20002B9898B322111133D26969BBA9D9D97006
:101B3000078E8E89339494A72D9B9BB63C1E1E2244
:101B400015878792C9E9E92087CECE49AA5555FF66
:101B500050282878A5DFDF7A038C8C8F59A1A1F853
:101B6000098989801A0D0D1765BFBFDAD7E6E631FE
:101B7000844242C6D06868B8824141C3299999B06D
:101B80005A2D2D771E0F0F117BB0B0CBA85454FCEB
:101B90006DBBBBD62C16163AA5C6636384F87C7C55
:101BA00099EE77778DF67B7B0DFFF2F2BDD66B6BEE
:101BB000B1DE6F6F5491C5C5506030300302010132
:101BC000A9CE67677D562B2B19E7FEFE62B5D7D7E6
:101BD000E64DABAB9AEC7676458FCACA9D1F8282E2
:101BE0004089C9C987FA7D7D15EFFAFAEBB25959D8
:101BF000C98E47470BFBF0F0EC41ADAD67B3D4D4D1
